:020000020000FC
:0A0000000C941D050C9400000C94F4
:10000A0000000C9400000C9400000C9400000C9466
:10001A0000000C9400000C9400000C9400000C9456
:10002A0000000C9400000C94DD8D0C9400000C94DC
:10003A0000000C9400000C941A390C9400000C94E3
:10004A0000000C9400000C9400000C94CEC90C948F
:10005A00FCC90C9400000C9400000C94B1390C9467
:10006A0000000C9400000C9400000C9400000C9406
:10007A0000000C9400000C9400000C9400000C94F6
:10008A0000000C9400000C94000000000000010223
:10009A00030400060705E2BD4FB20FA68099938CB0
:1000AA00E07F8973C367B85C7A522049AA40103945
:1000BA005032512C08276622521EC51AA717EC1473
:1000CA008D127C10A90E0F0DAB0B1202010EFFFF51
:1000DA0013FFFFFFFF11161003FF0D0B0006FFFFB2
:1000EA000C00060209010D0B0711031405120E1864
:1000FA00160C17130408100F0A0017120B11090D1A
:10010A000508130714010C190410030215060A0E38
:10011A000F000000010101010000000000010101BF
:10012A0001000101000000000100FFFF00FFFFFFC6
:10013A0001FFFFFFFF02030405FFFF06FFFFFFFFAA
:10014A00FF00436F4465496E466F00C8020C0C00FD
:10015A00000FAA558A61707220323320323032364B
:10016A002032303A30393A3431000067010165648F
:10017A000000000101010202020303030404040552
:10018A000505060606070707414243414243414225
:10019A004341424341424341424341424341424334
:1001AA0000000000EF006A02900800000000000052
:1001BA000000000000000000000000000000000035
:1001CA0000000000000000000000000000006400C1
:1001DA002301C602D504820F0000000000000000BF
:1001EA000000000000000000000000000000000005
:1001FA00000000000000000000000000F000F00015
:10020A005402D203F60900000000000000000000BA
:10021A0000000000000000000000000000000000D4
:10022A00000000000000000000002A03C8032105A6
:10023A00E3064D100000000000000000000000006E
:10024A0000000000000000000000000000000000A4
:10025A0000000000000000000101FE0102FD01048F
:10026A00FB0108F701807F0140BF0120DF0110EF89
:10027A0000807F0040BF0020DF0010EF0001FE0079
:10028A0002FD0004FB0008F70B0A090C0D100E0F03
:10029A001B1A191C1D001E1F02060B0C0D0E110045
:1002AA0000004C01000043414E72783A2025303359
:1002BA00580A000043414E696E707574436E743D6E
:1002CA0025752121210A0043414E2D25753A2030FA
:1002DA000A0043414E2D25753A20310A0043414E0A
:1002EA002D25753A2025750A0043414E20257500B3
:1002FA0044656C61792074696D657220257500000A
:10030A00466163746F727944656661756C740A003C
:10031A00485038343432004572724C6F67506F73EC
:10032A003D25752C204E6F3D25750A004572723A9F
:10033A002025752025750A002575204F66660A0056
:10034A002575204F6E0A00466C6173682074696DCA
:10035A006572202575004850383434320043666788
:10036A0053756D3D253034580A0020557064617408
:10037A0065640A00485038343432207665722E207B
:10038A0025752E25752E2575206170722032332031
:10039A00323032362032303A30393A34310A005368
:1003AA00657269616C3A2025750A00596561723A6D
:1003BA00203230253032752C205765656B3A20255E
:1003CA00750A004857207665723A2025632C204F1B
:1003DA007074696F6E733A20253032580A00436C84
:1003EA006F636B3A202530386C580A0043666743BE
:1003FA00686B53756D3A202530345820004F4B0AEC
:10040A000020457272210A0043666756657245727A
:10041A00723A2025752028257529210A004545505C
:10042A007665724572723A2025752028257529212C
:10043A000A00526573746F7265436E743D257520A8
:10044A0025752025750A00446174614572723D253F
:10045A0030325820253032580A0048503834343265
:10046A000A004144436D696E4572726F725B25756D
:10047A005D3D25752121210A0000496E707574734E
:10048A003A002025753D257500496E2D313A202503
:10049A00750A00496E2D323A2025750A00496E2DDB
:1004AA00333A2025750A00496E2D343A2025750AFB
:1004BA0000496E2D25753A2025750A00496E412D91
:1004CA002575204F66663A2025755B6D565D0A00D4
:1004DA00496E412D2575204F6E3A2025755B6D5664
:1004EA005D0A0053776974636820257500416E615F
:1004FA006C6F6720332E257500416E616C6F672023
:10050A00342E257500004B65795061643D00426CBC
:10051A00696E6B3A2530325820253032580A004726
:10052A0072617968696C6C2043414E6F70656E0A1E
:10053A00004772617968696C6C204A313333390A31
:10054A00004850393634320A004E6F6E650A000090
:10055A004B65795061642E436F6E6E2025750A00D3
:10056A004B65795061642E4469736F6E6E6E2025F7
:10057A00750A00004F75745075736850756C6C3A43
:10058A002025750A004F7574486967685369646560
:10059A004F6E6C793A2025750A0043202532753A48
:1005AA00202534750043616C6962726174652000AC
:1005BA004F4B0A006F75747075742025752066613B
:1005CA00696C65642121210A002532753A20253596
:1005DA002E32665B415D0A002532753A204E6F2045
:1005EA00666565646261636B2C204F75742D257591
:1005FA000A002532753A20466565646261636B209C
:10060A006572726F722C204F75742D25750A004F12
:10061A007574707574207465737400426174742003
:10062A0063616C696220203A20257500416E616C15
:10063A006F672063616C69623A20333D25752C200F
:10064A00343D25750043616C6962726174696F6E2D
:10065A004D61736B3A2025580A0020202532753ADD
:10066A00202533752C202534692C202534692C202B
:10067A002534692C202534690042617474657279C5
:10068A00206661696C65642121210A00416E616CF2
:10069A006F67206661696C65642121210A00206EFA
:1006AA006F7420636F6D706C657465642121210A13
:1006BA00004F75745273744572725B25755D0A003A
:1006CA004F75742D25753A204F6E0A004F75742D9B
:1006DA0025753A205325752D3E25752C204F6E3DE4
:1006EA0025752C205365743D25750A004144433A0B
:1006FA00002025753D2575002020426174743D2532
:10070A0075004C6F77426174744F66663D2025759B
:10071A000A004C6F77426174744F6E3D2025753024
:10072A00300A0042617474657279536B697046428B
:10073A003A20252E31665B565D0A00426174746563
:10074A0072794642204F4B3A20252E31665B565D20
:10075A000A002020416E612D333D2025750020209E
:10076A00416E612D343D202575004F75742D257518
:10077A003A2025750A004F757420257520474E4486
:10078A002D31210A004F757420257520474E442DBE
:10079A0032210A004F7574202575206C696D6974C1
:1007AA00210A004F7574412D25753A205325752D60
:1007BA003E25752C204F6E3D25752C205365743DC2
:1007CA0025750A004F757420257520474E44210A65
:1007DA00004F7574202575204C696D6974210A00D3
:1007EA004F75742D25753A205325752D3E25752094
:1007FA005365743D25750A004F7574707574733AA4
:10080A000A002534753A2046423D25752041444365
:10081A003D25752025755B6D415D0A002534753AC5
:10082A002046423D25750A00526573657445727209
:10083A006F720A004F7574707574202575004F75B4
:10084A00742D25753A205325752C204F6E3D25753C
:10085A002025632C202575305B6D415D0A004F759C
:10086A00747075742067726F757020257500506FEB
:10087A00776572446F776E0A0057616B6555703AF7
:10088A002025750A00004F7574412D25753A2053AD
:10089A0025752D3E25752C204F6E3D25750A0000C5
:1008AA0043616C69622E2073746172742025755BD2
:1008BA00416D705D0A0054657374206F75740A0087
:1008CA0043616C69622E20626174740A0043616C30
:1008DA00696220616E6128352C3056207265662E59
:1008EA00290A0043616C69623F006330006331008A
:1008FA006333006336006332300063620063610071
:10090A00746573746F75740050617373776F726472
:10091A003F0050573A20272573270A0050573A209C
:10092A004E6F6E650A0050577265736574005057B2
:10093A007265736574202D204F4B0A004144433F72
:10094A0000496E7075743F004C6F61643F004850F7
:10095A007374617475733F0052526573746F726574
:10096A00005252204F4B0A0052657365740053655A
:10097A00744F75742025753D2025750A00526573DC
:10098A006574206572726F720A004F7074696F6EB7
:10099A003A20253032580A0052657365740A0000FD
:1009AA005365712025633A20004F66660A00256365
:1009BA000A0053657175656E6365202575002020F0
:1009CA004F4B0A0020204661696C65642121210A87
:1009DA00000056696E2D25753A2025750A0056695C
:1009EA00727475616C202575000057697065723ADA
:1009FA00205325752D3E5325750A000001002D4E02
:100A0A00414E00494E4600002D4E414E0000010065
:100A1A000200AA0200000700BC031A030000070034
:100A2A00C3036003000001004E0E060A0000000026
:100A3A00F894EE27EFBBF1E0F5BFE5BFE093740051
:100A4A00E09375008DE0A2E0BB27ED938A95E9F764
:100A5A0080EF9FE0A0E0B1E0ED930197E9F7E8E1CC
:100A6A00FAE0D0E0DBBF87919791009781F0A791D8
:100A7A00B79107901790C791D791BF01DBB7F001E3
:100A8A00CBBF07900D920197E1F7FB01EBCFE0E0B6
:100A9A00EEBBEFEEEDBFE0E1EEBFCCEBD3E00C94A2
:100AAA00D9360E9478DBAD014093D2035093D30329
:100ABA00A5E2B1E00E9447DDE07111F0E1E001C07A
:100ACA00E0E0AFECB3E0E170EE0F0E2EEC91ED7FBB
:100ADA00E029EC93A7ECB2E00E9447DDE093D10352
:100AEA00A8ECB2E00E9447DDE0935C04A091D10338
:100AFA00A13010F0AD3008F004C0E091CF03E460FB
:100B0A0003C0E091CF03EB7FE093CF03E1E0E093F2
:100B1A00D800FA01E436A0E0FA0741F4E2E1E093F2
:100B2A00E200ECE0E093E300E7E335C0ED37A0E054
:100B3A00FA0741F4EEE0E093E200ECE0E093E30030
:100B4A00E7E329C0E83CA0E0FA0741F4E8E0E093D3
:100B5A00E200ECE0E093E300E7E31DC0EA3FA0E037
:100B6A00FA0741F4E6E0E093E200ECE0E093E30008
:100B7A00E7E311C0E43FA1E0FA0711F4E6E005C09B
:100B8A00E83EA3E0FA0749F4E2E0E093E200E4E099
:100B9A00E093E300E3E1E093E40010E1103F88F41E
:100BAA001093ED002EEE30E0E8EFF0E02E173F074D
:100BBA0030F4D901E0E0EC932F5F3F4FF5CF105F9F
:100BCA00EDCFE091D800E260E093D80010E4103F46
:100BDA00A0F41093ED002EEE30E0E8EFF0E02E17CF
:100BEA003F0730F4D901E0E0EC932F5F3F4FF5CF98
:100BFA00E8E8E093EF00105FEACF0E947FDB2696D9
:100C0A00089564970E9478DBE091D003E03009F4FC
:100C1A0014C2E17089F0E0E0E093ED00E091EE00AB
:100C2A00E17551F0E091D003EE7FE093D003E0E06C
:100C3A00E093EE00E093EF00E091D003E27089F0D8
:100C4A00E0E1E093ED00E091EE00E17551F0E09112
:100C5A00D003ED7FE093D003E0E0E093EE00E09371
:100C6A00EF00E091D003E47089F0E0E2E093ED0058
:100C7A00E091EE00E17551F0E091D003EB7FE09353
:100C8A00D003E0E0E093EE00E093EF00E091D003C0
:100C9A00E87089F0E0E3E093ED00E091EE00E175A1
:100CAA0051F0E091D003E77FE093D003E0E0E093D6
:100CBA00EE00E093EF00A091D003AF3009F4BDC17C
:100CCA00A0915604E0915704EA1709F4B6C1A4EDBD
:100CDA00B3E0E0915604F0E0BD01ADE0B0E00E945F
:100CEA002DDCDB01AE0FBF1FEC91E071B1F041E0EA
:100CFA00A4EDB3E0E0915604F0E0BD01ADE0B0E050
:100D0A000E942DDCDB01AE0FBF1F11960E94EADCA8
:100D1A00EB8BFC8B6D8B7E8B13C040E0A4EDB3E0B4
:100D2A00E0915604F0E0BD01ADE0B0E00E942DDC98
:100D3A00DB01AE0FBF1F1196ED91FD91EF8BF88F7E
:100D4A00A4EDB3E0E0915604F0E0BD01ADE0B0E0FF
:100D5A000E942DDCDB01AE0FBF1FEC91EF700E2F4E
:100D6A00098F403019F0E98DE061E98FE091D003F5
:100D7A00E17009F051C0E0E0E093ED00E98DE09305
:100D8A00EF004030D1F0EB89EE0FEE0FEE0FE0935B
:100D9A00F000AB89BC89E5E00E94B3DBE093F10087
:100DAA00AB89BC898D899E89EDE00E94DBDBE093EB
:100DBA00F200E5E10E94DBDB0AC0EF89E295E07F01
:100DCA00EE0FE093F200EF89F88D0E9406DCE093C3
:100DDA00F30010E01017B0F4A4EDB3E0E09156046C
:100DEA00F0E0BD01ADE0B0E00E942DDCDB01AE0F0A
:100DFA00BF1F1596EE27A10FBE1FEC91E093FA00D4
:100E0A001F5FE8CFE98DE05CE093EF00E091D0034B
:100E1A00E160E093D00303C1E091D003E27009F0EE
:100E2A0051C0E0E1E093ED00E98DE093EF0040303E
:100E3A00D1F0EB89EE0FEE0FEE0FE093F000AB89E5
:100E4A00BC89E5E00E94B3DBE093F100AB89BC8981
:100E5A008D899E89EDE00E94DBDBE093F200E5E1FB
:100E6A000E94DBDB0AC0EF89E295E07FEE0FE09398
:100E7A00F200EF89F88D0E9406DCE093F30010E09F
:100E8A001017B0F4A4EDB3E0E0915604F0E0BD0110
:100E9A00ADE0B0E00E942DDCDB01AE0FBF1F15965E
:100EAA00EE27A10FBE1FEC91E093FA001F5FE8CF77
:100EBA00E98DE05CE093EF00E091D003E260E0931B
:100ECA00D003ADC0E091D003E47009F051C0E0E274
:100EDA00E093ED00E98DE093EF004030D1F0EB892B
:100EEA00EE0FEE0FEE0FE093F000AB89BC89E5E060
:100EFA000E94B3DBE093F100AB89BC898D899E899E
:100F0A00EDE00E94DBDBE093F200E5E10E94DBDB2F
:100F1A000AC0EF89E295E07FEE0FE093F200EF89D5
:100F2A00F88D0E9406DCE093F30010E01017B0F48D
:100F3A00A4EDB3E0E0915604F0E0BD01ADE0B0E00D
:100F4A000E942DDCDB01AE0FBF1F1596EE27A10F05
:100F5A00BE1FEC91E093FA001F5FE8CFE98DE05CD9
:100F6A00E093EF00E091D003E460E093D00357C030
:100F7A00E091D003E87009F051C0E0E3E093ED009E
:100F8A00E98DE093EF004030D1F0EB89EE0FEE0FE0
:100F9A00EE0FE093F000AB89BC89E5E00E94B3DB79
:100FAA00E093F100AB89BC898D899E89EDE00E94AE
:100FBA00DBDBE093F200E5E10E94DBDB0AC0EF89AC
:100FCA00E295E07FEE0FE093F200EF89F88D0E9440
:100FDA0006DCE093F30010E01017B0F4A4EDB3E0E0
:100FEA00E0915604F0E0BD01ADE0B0E00E942DDCD6
:100FFA00DB01AE0FBF1F1596EE27A10FBE1FEC91A6
:10100A00E093FA001F5FE8CFE98DE05CE093EF0020
:10101A00E091D003E860E093D00301C00EC0E091F4
:10102A005604EF5FE0935604E150A0915604AA30AB
:10103A0018F0E0E0E093560443CEE0E05E2F2E2F56
:10104A0030E4303F08F032C13093ED00E091EE0019
:10105A00E07209F41EC1E091EF00EF700E2EEE81EE
:10106A00E07FE029EE83EF70E93020F0EE81E07F47
:10107A00E860EE83E091EF00E07109F46DC0E09161
:10108A00F300FF2766277727EB8BFC8B6D8B7E8B14
:10109A00AB89BC898D899E89E8E00E94C4DBEB8B11
:1010AA00FC8B6D8B7E8BE091F200AB89BC898D89BC
:1010BA009E89FF2766277727EA2BFB2B682B792B3C
:1010CA00EB8BFC8B6D8B7E8BAB89BC898D899E8962
:1010DA00E8E00E94C4DBEB8BFC8B6D8B7E8BE0918E
:1010EA00F100AB89BC898D899E89FF2766277727FE
:1010FA00EA2BFB2B682B792BEB8BFC8B6D8B7E8B76
:10110A00AB89BC898D899E89E5E00E94C4DBEB8BA3
:10111A00FC8B6D8B7E8BE091F000F0E00E94FDDB92
:10112A00AB89BC898D899E896F2F660F660B762FD6
:10113A00EA2BFB2B682B792BEB8BFC8B6D8B7E8B35
:10114A00EE81E061EE83EB89FC896D897E89EF830C
:10115A00F88769877A871DC0E091F300F0E0EF8B8A
:10116A00F88F0E94F4DBEF8BF88FE091F200F0E049
:10117A00F595E7950E94FBDBAF89B88DEA2BFB2B2F
:10118A00EF8BF88FEE81EF7EEE83EF89F88DEF8398
:10119A00F88710E0EE81EF701E1758F4E12FF0E0A7
:1011AA00DE011B96AE0FBF1FE091FA00EC931F5FA2
:1011BA00F1CF2F5FE091CF03E17081F0E0EBF2E035
:1011CA0060E070E00E9405DDEB8DFC8D66277727D5
:1011DA000E9405DD84E00E94FFDA2896A091D103DF
:1011EA00A03069F0AF89B88D109749F4EE81EF709D
:1011FA00E23028F0E091D103AC85EA1709F017C074
:10120A00EB85F0E0E130A0E0FA0721F4E091CF03AA
:10121A00EB7F0BC0E230A0E0FA0721F0E038A0E053
:10122A00FA0729F4E091CF03E460E093CF03E09159
:10123A00CF03E47069F5DE0116960E945F1DE09106
:10124A00200AE27021F0DE0116960E940591E091D3
:10125A00AB07F0E0E130A0E0FA0729F4DE011696C8
:10126A000E94434915C0E230A0E0FA0721F0E330BA
:10127A00A0E0FA0729F4DE0116960E94335508C049
:10128A00E430A0E0FA0721F4DE0116960E94225DFE
:10129A0005C0E091EE00EE7039F05F5FE0E0E093A8
:1012AA00EE00E0E8E093EF00305FCBCE222319F4A2
:1012BA00552309F44DC0213078F0E091CE03E03097
:1012CA0041F4E0910B09E062E0930B09E0E0E0935E
:1012DA000609EEE1E093CE03A0915804B0915904B7
:1012EA00A13FEFEFBE0740F4A0915A04B0915B040E
:1012FA00A13FEFEFBE0760F1E0915804F091590465
:10130A00F695E795E0935804F0935904E0915A044E
:10131A00F0915B04F695E795E0935A04F0935B0429
:10132A00A0915804B0915904E22FF0E0EA0FFB1F94
:10133A00E0935804F0935904A0915A04B0915B04C5
:10134A00E52FF0E0EA0FFB1FE0935A04F0935B04E9
:10135A000E947FDB6A960895BA93AA9324970E9403
:10136A0078DBE091CF03E47009F07FC1E091630478
:10137A00E07821F0AA85BB850E945F1DAA85BB85FE
:10138A00EC91EF700E2F202FEC91E07151F031E0CB
:10139A00206111960E94EADCEE83FF8368877987D1
:1013AA0006C030E0AA85BB8511964D915C91E0910B
:1013BA00D003E17009F047C0E0E0E093ED0020932C
:1013CA00EF003030D1F0EE81EE0FEE0FEE0FE0932A
:1013DA00F000AE81BF81E5E00E94B3DBE093F1004B
:1013EA00AE81BF8188859985EDE00E94DBDBE093C1
:1013FA00F200E5E10E94DBDB0CC0E0E0E093F000E4
:10140A00E42FE295E07FEE0FE093F200FA010E94EA
:10141A0006DCE093F30010E0101758F4AA85BB85A8
:10142A001596EE27A10FBE1FEC91E093FA001F5FFD
:10143A00F3CFE22FE05CE093EF00E091D003E160AC
:10144A00E093D00312C1E091D003E27009F047C0E3
:10145A00E0E1E093ED002093EF003030D1F0EE812F
:10146A00EE0FEE0FEE0FE093F000AE81BF81E5E0E4
:10147A000E94B3DBE093F100AE81BF818885998534
:10148A00EDE00E94DBDBE093F200E5E10E94DBDBAA
:10149A000CC0E0E0E093F000E42FE295E07FEE0F6D
:1014AA00E093F200FA010E9406DCE093F30010E0F8
:1014BA00101758F4AA85BB851596EE27A10FBE1FF3
:1014CA00EC91E093FA001F5FF3CFE22FE05CE09328
:1014DA00EF00E091D003E260E093D003C6C0E09150
:1014EA00D003E47009F047C0E0E2E093ED002093F6
:1014FA00EF003030D1F0EE81EE0FEE0FEE0FE093F9
:10150A00F000AE81BF81E5E00E94B3DBE093F10019
:10151A00AE81BF8188859985EDE00E94DBDBE0938F
:10152A00F200E5E10E94DBDB0CC0E0E0E093F000B2
:10153A00E42FE295E07FEE0FE093F200FA010E94B9
:10154A0006DCE093F30010E0101758F4AA85BB8577
:10155A001596EE27A10FBE1FEC91E093FA001F5FCC
:10156A00F3CFE22FE05CE093EF00E091D003E46078
:10157A00E093D0037AC0E091D003E87009F047C045
:10158A00E0E3E093ED002093EF003030D1F0EE81FC
:10159A00EE0FEE0FEE0FE093F000AE81BF81E5E0B3
:1015AA000E94B3DBE093F100AE81BF818885998503
:1015BA00EDE00E94DBDBE093F200E5E10E94DBDB79
:1015CA000CC0E0E0E093F000E42FE295E07FEE0F3C
:1015DA00E093F200FA010E9406DCE093F30010E0C7
:1015EA00101758F4AA85BB851596EE27A10FBE1FC2
:1015FA00EC91E093FA001F5FF3CFE22FE05CE093F7
:10160A00EF00E091D003E860E093D0032EC0E091B0
:10161A005704EF5F1E2F1A3008F010E0E0915604CD
:10162A00E11759F4EF5FE0935604E150A091560494
:10163A00AA3018F0E0E0E0935604A4EDB3E0E0919C
:10164A005704F0E0BD01ADE0B0E00E942DDCE60FEA
:10165A00F71FFA93EA93EC85FD85FA93EA93ADE0D6
:10166A00B0E00E9465D4109357040E947FDB2C9649
:10167A0008951A930A938D011396ED91FD91A09105
:10168A00D203B091D303EA17FB0721F0F801A38133
:10169A00B48107DAE0910B09E17051F4E0910B098A
:1016AA00E160E0930B09E1E0E09306090E94173C30
:1016BA00F801E581EF70E93018F4D80115964CDE8F
:1016CA00099119910895A091CE03A13078F0E09183
:1016DA00CE03E150E093CE03E03041F4E0910B09F0
:1016EA00EF7DE0930B09E0E0E093060908951A9371
:1016FA00A4EAB5E00E9447DDE093330E11E116300B
:10170A0048F0A9EAB5E0EE27A10FBE1F0E9447DD07
:10171A00E03009F002C01150F2CFE12FE550E0931A
:10172A00340EE0E0E093350EABEBB5E00E9447DD06
:10173A00E093360EA0EFB5E00E9447DDE093370E46
:10174A00A5E2B6E00E9447DDE093380EAAE6B6E0CD
:10175A000E9447DDE093390EA091390EA13019F4A9
:10176A00E2E0E093390EE091390EE0933A0EABE6EF
:10177A00B6E00E943FDDE0933C0EF0933D0E60938D
:10178A003E0E70933F0EEFEFE0933B0EAFE6B6E0EE
:10179A000E9443DDE093400EF093410E309719F416
:1017AA00E0E0E0933A0EABE3B1E00E943FDD309710
:1017BA006040704011F4E0E00BC0AFE3B1E00E947A
:1017CA0047DDE093420EA091420EA63018F0E5E004
:1017DA00E093420E10E01330B0F5A4E4BEE0E12F2E
:1017EA00F0E0EE0FFF1FEA0FFB1F3196FF93EF9316
:1017FA00A2E7B6E0E12FF0E0BD01A5E1B0E00E946A
:10180A002DDCDB01AE0FBF1F14960E9447DDAF919E
:10181A00BF91EC93A4E4BEE0E12FF0E0EE0FFF1FCE
:10182A00AE0FBF1FEC91E078E560EC93A4E4BEE054
:10183A00E12FF0E0EE0FFF1FAE0FBF1FEC91EF7725
:10184A00EC931F5FC8CF1991089561970E9478DBC6
:10185A00E0916304E07421F40E947FDB67960895A7
:10186A00A0913A0EA13010F40C94DA15E0913A0ED8
:10187A00E150E0933A0EEF5FE0913A0EE03011F05A
:10188A000C94DA15E091390EE0933A0EE0913B0E92
:10189A00EF5FE0933B0EE150A0913B0EAF3018F0A2
:1018AA00E0E0E0933B0EEA85E07FE860EA87FE012C
:1018BA003F96FA93EA93E0E0EA93A8E0B0E00E9448
:1018CA0077D4E0913B0EF0E0309709F056C1E091F1
:1018DA00400EF091410EE17009F44BC100E0E09135
:1018EA009307E17009F00160E0919407E17009F053
:1018FA000260E0919507E17009F00460E0919607B3
:10190A00E17009F00860E0919707E17009F0006161
:10191A00E0919807E17009F00062E0919907E1709F
:10192A0009F00064E0919A07E17009F000680F87F6
:10193A0000E0E0919B07E17009F00160E0919C07EB
:10194A00E17009F00260E0919D07E17009F004601E
:10195A00E0919E07E17009F00860FE01709600832D
:10196A0000E0E0916A0DE07409F00160E091720D07
:10197A00E07409F00260E0917A0DE07409F0046005
:10198A00E091820DE07409F00860E0918A0DE0743C
:10199A0009F00061E091920DE07409F00062E091B3
:1019AA009A0DE07409F00064E091A20DE07409F068
:1019BA000068FE017196008300E0E091AA0DE074D0
:1019CA0009F00160E091B20DE07409F00260E09163
:1019DA00BA0DE07409F00460E091C20DE07409F0F8
:1019EA000860E091CA0DE07409F00061E091D20D3F
:1019FA00E07409F00062E091DA0DE07409F0006425
:101A0A00E091E20DE07409F00068FE01729600832D
:101A1A0000E0E0917704E07809F00160E091850444
:101A2A00E07809F00260E0919304E07809F004603C
:101A3A00E091A104E07809F00860E091AF04E07851
:101A4A0009F00061E091BD04E07809F00062E091DC
:101A5A00CB04E07809F00064E091D904E07809F059
:101A6A000068FE017396008300E0E091E704E078E5
:101A7A0009F00160E091F504E07809F00260E09174
:101A8A000305E07809F00460E0911105E07809F0B7
:101A9A000860E0911F05E07809F00061E0912D05EA
:101AAA00E07809F00062E0913B05E07809F0006413
:101ABA00E0914905E07809F00068FE017496008318
:101ACA0000E0E0915705E07809F00160E0916505D2
:101ADA00E07809F00260E0917305E07809F00460AB
:101AEA00E0918105E07809F00860E0918F05E078DF
:101AFA0009F00061E0919D05E07809F00062E0914B
:101B0A009D05E07809F00064E091B905E07809F0F4
:101B1A000068FE017596008300E0E091C705E07851
:101B2A0009F00160E091D505E07809F00260E091E2
:101B3A00E305E07809F00460E091F105E07809F046
:101B4A000860E091FF05E07809F00061E0910D0678
:101B5A00E07809F00062E0911B06E07809F0006481
:101B6A00E0912906E07809F00068FE017696008384
:101B7A00E2C7E1E0E0933B0E05C0E130A0E0FA07DE
:101B8A0009F0DCC0E091400EF091410EE27009F4D8
:101B9A00D1C0E0911C09E077E03321F4E0911C09FF
:101BAA00E47009F403C0E6E6EF870DC0E0911C0972
:101BBA00E295E770FF2766277727EC58FE4F6F4FAD
:101BCA006BBF06900F86E0912509E077E03321F498
:101BDA00E0912509E47009F403C0E6E6E88B0DC03C
:101BEA00E0912509E295E770FF2766277727EC58E9
:101BFA00FE4F6F4F6BBF0690088AE0912E09E0777F
:101C0A00E03321F4E0912E09E47009F403C0E6E61A
:101C1A00E98B0DC0E0912E09E295E770FF27662750
:101C2A007727EC58FE4F6F4F6BBF0690098AE091F9
:101C3A003709E077E03321F4E0913709E47009F4D9
:101C4A0003C0E6E6EA8B0DC0E0913709E295E7703A
:101C5A00FF2766277727EC58FE4F6F4F6BBF06901A
:101C6A000A8AE0914009E077E03321F4E0914009E3
:101C7A00E47009F403C0E6E6EB8B0DC0E09140097D
:101C8A00E295E770FF2766277727EC58FE4F6F4FDC
:101C9A006BBF06900B8AE0914909E077E03321F4A3
:101CAA00E0914909E47009F403C0E6E6EC8B0DC043
:101CBA00E0914909E295E770FF2766277727EC58F4
:101CCA00FE4F6F4F6BBF06900C8AE0915209E07786
:101CDA00E03321F4E0915209E47009F403C0E6E626
:101CEA00ED8B0DC0E0915209E295E770FF27662758
:101CFA007727EC58FE4F6F4F6BBF06900D8AE09125
:101D0A005B09E077E03321F4E0915B09E47009F4C0
:101D1A0003C0E6E6EE8B0DC0E0915B09E295E77041
:101D2A00FF2766277727EC58FE4F6F4F6BBF069049
:101D3A000E8A01C7E2E0E0933B0E05C0E230A0E064
:101D4A00FA0709F0DCC0E091400EF091410EE47010
:101D5A0009F4D1C0E0916409E077E03321F4E0911D
:101D6A006409E47009F403C0E6E6EF870DC0E09168
:101D7A006409E295E770FF2766277727EC58FE4F3C
:101D8A006F4F6BBF06900F86E0916D09E077E033E5
:101D9A0021F4E0916D09E47009F403C0E6E6E88BEA
:101DAA000DC0E0916D09E295E770FF276627772756
:101DBA00EC58FE4F6F4F6BBF0690088AE091760988
:101DCA00E077E03321F4E0917609E47009F403C086
:101DDA00E6E6E98B0DC0E0917609E295E770FF2708
:101DEA0066277727EC58FE4F6F4F6BBF0690098A1C
:101DFA00E0917F09E077E03321F4E0917F09E47014
:101E0A0009F403C0E6E6EA8B0DC0E0917F09E2958A
:101E1A00E770FF2766277727EC58FE4F6F4F6BBF97
:101E2A0006900A8AE0918809E077E03321F4E0918C
:101E3A008809E47009F403C0E6E6EB8B0DC0E09173
:101E4A008809E295E770FF2766277727EC58FE4F47
:101E5A006F4F6BBF06900B8AE0919109E077E033F0
:101E6A0021F4E0919109E47009F403C0E6E6EC8BF1
:101E7A000DC0E0919109E295E770FF276627772761
:101E8A00EC58FE4F6F4F6BBF06900C8AE0919A098F
:101E9A00E077E03321F4E0919A09E47009F403C091
:101EAA00E6E6ED8B0DC0E0919A09E295E770FF270F
:101EBA0066277727EC58FE4F6F4F6BBF06900D8A47
:101ECA00E091A309E077E03321F4E091A309E470FB
:101EDA0009F403C0E6E6EE8B0DC0E091A309E29592
:101EEA00E770FF2766277727EC58FE4F6F4F6BBFC7
:101EFA0006900E8A20C6E3E0E0933B0E05C0E3306D
:101F0A00A0E0FA0709F08EC0E091400EF091410E70
:101F1A00E87009F483C0E091AC09E077E03321F47A
:101F2A00E091AC09E47009F403C0E6E6EF870DC05E
:101F3A00E091AC09E295E770FF2766277727EC580E
:101F4A00FE4F6F4F6BBF06900F86E091B509E077A1
:101F5A00E03321F4E091B509E47009F403C0E6E640
:101F6A00E88B0DC0E091B509E295E770FF27662777
:101F7A007727EC58FE4F6F4F6BBF0690088AE091A7
:101F8A00EB09E295E770FF2766277727EC58FE4FA3
:101F9A006F4F6BBF0690098AE091EE09E295E770F0
:101FAA00FF2766277727EC58FE4F6F4F6BBF0690C7
:101FBA000A8AE091F109E295E770FF2766277727F9
:101FCA00EC58FE4F6F4F6BBF06900B8AE091F409F5
:101FDA00E295E770FF2766277727EC58FE4F6F4F89
:101FEA006BBF06900C8AE091F709E295E770FF272C
:101FFA0066277727EC58FE4F6F4F6BBF06900D8A06
:10200A00E091FA09E295E770FF2766277727EC58EF
:10201A00FE4F6F4F6BBF06900E8A8DC5E4E0E093CA
:10202A003B0E05C0E430A0E0FA0709F074C0E09165
:10203A00400EF091410EE07109F469C0E091FD098A
:10204A00E295E770FF2766277727EC58FE4F6F4F18
:10205A006BBF06900F86E091000AE295E770FF27B2
:10206A0066277727EC58FE4F6F4F6BBF0690088A9A
:10207A00E091030AE295E770FF2766277727EC5875
:10208A00FE4F6F4F6BBF0690098AE091060AE295F0
:10209A00E770FF2766277727EC58FE4F6F4F6BBF15
:1020AA0006900A8AE091090AE295E770FF276627F7
:1020BA007727EC58FE4F6F4F6BBF06900B8AE09163
:1020CA000C0AE295E770FF2766277727EC58FE4F40
:1020DA006F4F6BBF06900C8AE0910F0AE295E7708A
:1020EA00FF2766277727EC58FE4F6F4F6BBF069086
:1020FA000D8AE091120AE295E770FF276627772793
:10210A00EC58FE4F6F4F6BBF06900E8A14C5E5E080
:10211A00E0933B0E05C0E530A0E0FA0709F0B0C035
:10212A00E091400EF091410EE07209F4A5C0409191
:10213A002309509124094C3EE3E15E0738F4DA01A1
:10214A00E4E1F0E00E9473DC0E2F01C00FEF0F876D
:10215A00A0912809A63319F4E0E0E88B13C0409156
:10216A002C0950912D094C3EE3E15E0738F4DA015F
:10217A00E4E1F0E00E9473DC0E2F01C00FEFFE01D4
:10218A007096008340913509509136094C3EE3E13F
:10219A005E0738F4DA01E4E1F0E00E9473DC0E2F06
:1021AA0001C00FEFFE0171960083A0913A09A63390
:1021BA0019F4E0E0EA8B13C040913E0950913F09BF
:1021CA004C3EE3E15E0738F4DA01E4E1F0E00E9414
:1021DA0073DC0E2F01C00FEFFE017296008340914F
:1021EA004709509148094C3EE3E15E0738F4DA01A9
:1021FA00E4E1F0E00E9473DC0E2F01C00FEFFE0154
:10220A007396008340915009509151094C3EE3E185
:10221A005E0738F4DA01E4E1F0E00E9473DC0E2F85
:10222A0001C00FEFFE017496008340915909509145
:10223A005A094C3EE3E15E0738F4DA01E4E1F0E0E2
:10224A000E9473DC0E2F01C00FEFFE01759600830A
:10225A0040916209509163094C3EE3E15E0738F40C
:10226A00DA01E4E1F0E00E9473DC0E2F01C00FEF07
:10227A00FE01769600835FC4E6E0E0933B0E05C05C
:10228A00E630A0E0FA0709F0A2C0E091400EF09112
:10229A00410EE07409F497C040916B0950916C09A2
:1022AA004C3EE3E15E0738F4DA01E4E1F0E00E9433
:1022BA0073DC0E2F01C00FEF0F8740917409509104
:1022CA0075094C3EE3E15E0738F4DA01E4E1F0E037
:1022DA000E9473DC0E2F01C00FEFFE01709600837F
:1022EA0040917D0950917E094C3EE3E15E0738F446
:1022FA00DA01E4E1F0E00E9473DC0E2F01C00FEF77
:10230A00FE017196008340918609509187094C3EDF
:10231A00E3E15E0738F4DA01E4E1F0E00E9473DCFD
:10232A000E2F01C00FEFFE017296008340918F09B4
:10233A00509190094C3EE3E15E0738F4DA01E4E19A
:10234A00F0E00E9473DC0E2F01C00FEFFE017396BE
:10235A00008340919809509199094C3EE3E15E0748
:10236A0038F4DA01E4E1F0E00E9473DC0E2F01C0D8
:10237A000FEFFE01749600834091A1095091A209C2
:10238A004C3EE3E15E0738F4DA01E4E1F0E00E9452
:10239A0073DC0E2F01C00FEFFE017596008340918A
:1023AA00AA095091AB094C3EE3E15E0738F4DA0121
:1023BA00E4E1F0E00E9473DC0E2F01C00FEFFE0192
:1023CA0076960083B8C3E7E0E0933B0E05C0E7309A
:1023DA00A0E0FA0709F082C0E091400EF091410EA8
:1023EA00E07809F477C0A091AF09A63319F4E0E0C8
:1023FA00EF8711C04091B3095091B4094C3EE3E113
:10240A005E0738F4DA01E4E1F0E00E9473DC0E2F93
:10241A0001C00FEF0F87A091B809A63319F4E0E0C5
:10242A00E88B13C04091BC095091BD094C3EE3E1D1
:10243A005E0738F4DA01E4E1F0E00E9473DC0E2F63
:10244A0001C00FEFFE0170960083E091EB09E2955F
:10245A00E7702E2F223011F0233011F4EFE001C083
:10246A00E0E0E98BE091EE09E295E7702E2F223049
:10247A0011F0233011F4EFE0EA8BE091F109E295D3
:10248A00E7702E2F223011F0233011F4EFE0EB8B9E
:10249A00E091F409E295E7702E2F223011F02330F3
:1024AA0011F4EFE0EC8BE091F709E295E7702E2F3B
:1024BA00223011F0233011F4EFE0ED8BE091FA09AC
:1024CA00E295E7702E2F223011F0233011F4EFE05D
:1024DA00EE8B31C3E8E0E0933B0E05C0E830A0E0A4
:1024EA00FA0709F064C0E091400EF091410EF170D4
:1024FA0009F459C0E091FD09E295E7702E2F2230C8
:10250A0011F0233011F4EFE0EF87E091000AE29531
:10251A00E7702E2F223011F0233011F4EFE0E88B10
:10252A00E091030AE295E7702E2F223011F0233052
:10253A0011F4EFE0E98BE091060AE295E7702E2F9D
:10254A00223011F0233011F4EFE0EA8BE091090A0E
:10255A00E295E7702E2F223011F0233011F4EFE0CC
:10256A00EB8BE0910C0AE295E7702E2F223011F0E6
:10257A00233011F4EFE0EC8BE0910F0AE295E7705B
:10258A002E2F223011F0233011F4EFE0ED8BE09181
:10259A00120AE295E7702E2F223011F0233011F43F
:1025AA00EFE0EE8BC8C2E9E0E0933B0E05C0E930EC
:1025BA00A0E0FA0709F083C0E091400EF091410EC5
:1025CA00F27009F478C0A091300EE5E0EA9FA0010C
:1025DA005F87FE0170964083E0912D0EE98BE091B2
:1025EA002C0EEA8BE091BE09E077E03321F4E0910A
:1025FA00BE09E47009F403C0E6E6EB8B0DC0E09176
:10260A00BE09E295E770FF2766277727EC58FE4F49
:10261A006F4F6BBF06900B8AE091C709E077E033F2
:10262A0021F4E091C709E47009F403C0E6E6EC8BF3
:10263A000DC0E091C709E295E770FF276627772763
:10264A00EC58FE4F6F4F6BBF06900C8AE091D00991
:10265A00E077E03321F4E091D009E47009F403C093
:10266A00E6E6ED8B0DC0E091D009E295E770FF2711
:10267A0066277727EC58FE4F6F4F6BBF06900D8A7F
:10268A00E091D909E077E03321F4E091D909E470C7
:10269A0009F403C0E6E6EE8B0DC0E091D909E29594
:1026AA00E770FF2766277727EC58FE4F6F4F6BBFFF
:1026BA0006900E8A40C2EAE0E0933B0E05C0EA307B
:1026CA00A0E0FA0709F0A5C0E091400EF091410E92
:1026DA00F47009F49AC0A091C109A63319F4E0E094
:1026EA00EF8711C04091C5095091C6094C3EE3E1FC
:1026FA005E0738F4DA01E4E1F0E00E9473DC0E2FA1
:10270A0001C00FEF0F87A091CA09A63319F4E0E0C0
:10271A00E88B13C04091CE095091CF094C3EE3E1BA
:10272A005E0738F4DA01E4E1F0E00E9473DC0E2F70
:10273A0001C00FEFFE01709600834091D7095091B6
:10274A00D8094C3EE3E15E0738F4DA01E4E1F0E04F
:10275A000E9473DC0E2F01C00FEFFE0171960083F9
:10276A004091E0095091E1094C3EE3E15E0738F4FB
:10277A00DA01E4E1F0E00E9473DC0E2F01C00FEFF2
:10278A00FE0172960083A0911A09B0911B09E4E137
:10279A00F0E00E9473DCAF015B8BFE01749640830C
:1027AA00E091E209E077E03321F4E091E209E47094
:1027BA0009F403C0E6E6ED8B0DC0E091E209E2956B
:1027CA00E770FF2766277727EC58FE4F6F4F6BBFDE
:1027DA0006900D8AA091E509A63319F4E0E0EE8B84
:1027EA0013C04091E9095091EA094C3EE3E15E07C2
:1027FA0038F4DA01E4E1F0E00E9473DC0E2F01C044
:10280A000FEFFE017696008396C1EBE0E0933B0E54
:10281A0005C0EB30A0E0FA0709F06EC0E091400E67
:10282A00F091410EF87009F463C000E0E091EA0DFE
:10283A00E07409F00160E091F20DE07409F00260C1
:10284A00E091FA0DE07409F00460E091020EE07480
:10285A0009F008600F87E091150AE295E770FF27F3
:10286A0066277727EC58FE4F6F4F6BBF0690088A92
:10287A00E091180AE295E770FF2766277727EC5858
:10288A00FE4F6F4F6BBF0690098AE091150AE295D9
:10289A00E7702E2F223011F0233011F4EFE001C03F
:1028AA00E0E0EA8BE091180AE295E7702E2F2230D9
:1028BA0011F0233011F4EFE001C0E0E0EB8BE0917E
:1028CA00260AE17021F0E091270AE695EC8BE09167
:1028DA002E0AE17021F0E0912F0AE695ED8BE09146
:1028EA00360AE17021F0E091370AE695EE8B23C1B2
:1028FA00ECE0E0933B0E04C0EC30A0E0FA07C9F527
:10290A00E091400EF091410EF07179F1E2E0EF872B
:10291A00ECE0E88BA6E1B0E00E9447DDE98BA5E197
:10292A00B0E00E9447DDEA8BE0913E0AE17021F0B7
:10293A00E0913F0AE695EB8BE091460AE17021F0BF
:10294A00E091470AE695EC8BE0914E0AE17021F09E
:10295A00E0914F0AE695ED8BE091560AE17021F07D
:10296A00E091570AE695EE8BE6C0EDE0E0933B0E68
:10297A0005C0ED30A0E0FA0709F09FC0E091400ED3
:10298A00F091410EF07209F494C0E091430EEF5FAA
:10299A00E093430EE150EF8700E0E0912F0EE072E2
:1029AA0009F00160E0912F0EE07409F00260E091F5
:1029BA001509E17009F00460E0911509E27009F067
:1029CA000860E0911509E07209F00061E0911409CC
:1029DA00E07809F00062A5E3B1E00E9447DDA0912A
:1029EA00210EAE1708F00064A091CE03A13008F0C2
:1029FA000068FE0170960083E091190EE98BE09160
:102A0A00180EEA8BE0E01E2F0E2F31E0183060F42A
:102A1A00A3E01A9FF001ED5BF84FE081E27009F044
:102A2A00032B1F5F330FF2CFFE017396008300E082
:102A3A0018E031E0103160F4A3E01A9FF001ED5B79
:102A4A00F84FE081E27009F0032B1F5F330FF2CFDA
:102A5A00FE017496008300E010E131E0143160F465
:102A6A00A3E01A9FF001ED5BF84FE081E27009F0F4
:102A7A00032B1F5F330FF2CFFE0175960083E0E050
:102A8A001E2F0E2F31E0153080F4E12FAFE7B7E0AB
:102A9A00F0E00E94F6DBAE0FBF1F1396EC91E170D7
:102AAA0009F0032B1F5F330FEECFFE0176960083EA
:102ABA0042C0EEE0E0933B0E04C0EE30A0E0FA071D
:102ACA00D1F5E091400EF091410EF07479F1E09168
:102ADA008108F09182080E9408DCAF015F87FE013D
:102AEA0070964083E0918308F09184080E9408DC84
:102AFA00AF01598BFE017296408300E0E0911509FF
:102B0A00E47009F00160E0911509E87009F00260CB
:102B1A00E0911509E07109F00460E0911509E0728D
:102B2A0009F00860FE017396008305C0E0E0E093B7
:102B3A003B0E0C94660CA0913C0EB0913D0E809118
:102B4A003E0E90913F0EE0913B0EF0E06F2F660F24
:102B5A00660B762FEA0FFB1F681F791FEE83FF8330
:102B6A0068877987AE81BF8188859985A030E8E03A
:102B7A00BE07E0E08E07E0E09E0740F4EA85EF7EBC
:102B8A00EA87EE81FF81EB87FC870BC0EA85E0616B
:102B9A00EA87EE81FF8168857985EB87FC876D87F7
:102BAA007E87DE011A960E94B1090E947FDB679632
:102BBA00089564970E9478DBE0916304E07409F455
:102BCA0049C4EF81E07FE860EF83A091420EA13013
:102BDA0008F44FC0E091420EE150E093420EEF5FDD
:102BEA00E091420EE03009F044C0AFE3B1E00E9448
:102BFA0047DDE093420EABE3B1E00E943FDDEC8B90
:102C0A00FD8B6E8B7F8BAC89BD898E899F89A030A5
:102C1A00E8E0BE07E0E08E07E0E09E0740F4EF81BF
:102C2A00EF7EEF83EC89FD89E887F9870BC0EF8196
:102C3A00E061EF83EC89FD896E897F89E887F987EE
:102C4A006A877B87A9E3B1E00E9447DDEC87AAE3A4
:102C5A00B1E00E9447DDED87E2E0EE87ECE0EF8726
:102C6A00E88BE0E0E98BEA8BEB8BDE0117960E949A
:102C7A00B109A091330EA13008F421C1E091330EBD
:102C8A00E150E093330EE03009F019C1FE013C96A1
:102C9A00FA93EA93E0E0EA93A8E0B0E00E9477D4DE
:102CAA00A4EAB5E00E9447DDE093330EA5EAB5E059
:102CBA000E943FDDEC8BFD8B6E8B7F8BAC89BD89CF
:102CCA008E899F89A030E8E0BE07E0E08E07E0E049
:102CDA009E0740F4EF81EF7EEF83EC89FD89E88758
:102CEA00F9870BC0EF81E061EF83EC89FD896E897A
:102CFA007F89E887F9876A877B87A091340EA1309C
:102D0A0090F1E091350EEF5FE093350EE150A0911E
:102D1A00350EE091340EEA1718F4E1E0E093350E2F
:102D2A00E091350EEC87A9EAB5E0F0E03496AE0FF3
:102D3A00BF1F0E9447DD4E2F4F3010F0463208F079
:102D4A0012C0E42FF0E03F97A9E0B0E00E942DDC2A
:102D5A00ED5DF64FDF01ED91FD91DF01E4E1F0E079
:102D6A000E9473DCEB8BAEEAB5E00E9447DD4E2F82
:102D7A004F3010F0463208F012C0E42FF0E03F97CF
:102D8A00A9E0B0E00E942DDCED5DF64FDF01ED9188
:102D9A00FD91DF01E4E1F0E00E9473DCEA8BADEA29
:102DAA00B5E00E9447DD4E2F4F3010F0463208F052
:102DBA0012C0E42FF0E03F97A9E0B0E00E942DDCBA
:102DCA00ED5DF64FDF01ED91FD91DF01E4E1F0E009
:102DDA000E9473DCE98BACEAB5E00E9447DD4E2F16
:102DEA004F3010F0463208F012C0E42FF0E03F975F
:102DFA00A9E0B0E00E942DDCED5DF64FDF01ED9118
:102E0A00FD91DF01E4E1F0E00E9473DCE88BABEABC
:102E1A00B5E00E9447DD4E2F4F3010F0463208F0E1
:102E2A0012C0E42FF0E03F97A9E0B0E00E942DDC49
:102E3A00ED5DF64FDF01ED91FD91DF01E4E1F0E098
:102E4A000E9473DCEF87AAEAB5E00E9447DD4E2FA5
:102E5A004F3010F0463208F012C0E42FF0E03F97EE
:102E6A00A9E0B0E00E942DDCED5DF64FDF01ED91A7
:102E7A00FD91DF01E4E1F0E00E9473DCEE87A9EA4C
:102E8A00B5E00E9447DD4E2F4F3010F0463208F071
:102E9A0012C0E42FF0E03F97A9E0B0E00E942DDCD9
:102EAA00ED5DF64FDF01ED91FD91DF01E4E1F0E028
:102EBA000E9473DCED87DE0117960E94B109A0918A
:102ECA00360EA13008F47CC0E091360EE150E09352
:102EDA00360EEF5FE091360EE03009F071C0FE0168
:102EEA003C96FA93EA93E0E0EA93A8E0B0E00E9405
:102EFA0077D4ABEBB5E00E9447DDE093360EACEB3E
:102F0A00B5E00E943FDDEC8BFD8B6E8B7F8BAC892D
:102F1A00BD898E899F89A030E8E0BE07E0E08E0770
:102F2A00E0E09E0740F4EF81EF7EEF83EC89FD89B4
:102F3A00E887F9870BC0EF81E061EF83EC89FD89AF
:102F4A006E897F89E887F9876A877B87E0E00E2F99
:102F5A001E2F2E2F51E0103300F5A0ECB5E0EE271E
:102F6A00A10FBE1F0E9447DD4E2F403031F0A42F23
:102F7A000E94E03DE03009F0052B503859F4E22F69
:102F8A002F5FF0E0DE011C96EA0FFB1F008351E081
:102F9A0000E001C0550F1F5FDECFA0911A09B09162
:102FAA001B09AC39E3E6BE0728F4E4E6F0E00E9428
:102FBA0073DC01C0EFEFEA8BDE0117960E94B109BC
:102FCA00A091370EA13008F4B9C0E091370EE15054
:102FDA00E093370EEF5FE091370EE03009F0AEC0B4
:102FEA00A0EFB5E00E9447DDE093370EA1EFB5E010
:102FFA000E943FDDEC8BFD8B6E8B7F8BAC89BD898C
:10300A008E899F89A030E8E0BE07E0E08E07E0E005
:10301A009E0740F4EF81EF7EEF83EC89FD89E88714
:10302A00F9870BC0EF81E061EF83EC89FD896E8936
:10303A007F89E887F9876A877B87E0E00E2F1E2F52
:10304A002E2F51E0103308F06CC0A5EFB5E0EE2743
:10305A00A10FBE1F0E9447DD4E2F403009F451C018
:10306A004F3010F0463308F03AC0463210F5E42FDC
:10307A00F0E03F97A9E0B0E00E942DDCE45EF64F55
:10308A00E081E295E770EE83E42FF0E03F97A9E054
:10309A00B0E00E942DDCE45EF64FE081E47039F482
:1030AA00AE81A13021F0A43011F0A53009F4052B2E
:1030BA0015C0E42FF0E0B697A3E0B0E00E942DDC43
:1030CA00E551F64FE081E295E770EE83AE81A130DB
:1030DA0021F0A43011F0A53009F4052B12C04733B2
:1030EA0010F04C3308F007C0A42F0E947988E03012
:1030FA0009F0052B06C0A42F0E94E03DE03009F03C
:10310A00052B503859F4E22F2F5FF0E0DE011C96B0
:10311A00EA0FFB1F008351E000E001C0550F1F5F5B
:10312A0091CFE091300EF0E03196F595E795EA8B74
:10313A00E0E0EB8BDE0117960E94B109A091380EF0
:10314A00A13008F4BEC0E091380EE150E093380E89
:10315A00EF5FE091380EE03009F0B3C0FE013C9613
:10316A00FA93EA93E0E0EA93A8E0B0E00E9477D409
:10317A00A5E2B6E00E9447DDE093380EA6E2B6E08B
:10318A000E943FDDEC8BFD8B6E8B7F8BAC89BD89FA
:10319A008E899F89A030E8E0BE07E0E08E07E0E074
:1031AA009E0740F4EF81EF7EEF83EC89FD89E88783
:1031BA00F9870BC0EF81E061EF83EC89FD896E89A5
:1031CA007F89E887F9876A877B87E0E00E2F1E2FC1
:1031DA002E2F51E0103408F070C0AAE2B6E0EE27B4
:1031EA00A10FBE1F0E9447DD4E2F403009F455C083
:1031FA00103220F04F3010F0463308F03AC0463211
:10320A0010F5E42FF0E03F97A9E0B0E00E942DDC32
:10321A00E45EF64FE081E295E770EE83E42FF0E09A
:10322A003F97A9E0B0E00E942DDCE45EF64FE08112
:10323A00E47039F4AE81A13021F0A43011F0A53048
:10324A0009F4052B15C0E42FF0E0B697A3E0B0E02F
:10325A000E942DDCE551F64FE081E295E770EE839E
:10326A00AE81A13021F0A43011F0A53009F4052B6C
:10327A0014C0103220F0473310F04C3308F007C066
:10328A00A42F0E947988E03009F0052B06C0A42FEC
:10329A000E94E03DE03009F0052B503859F4E22F46
:1032AA002F5FF0E0DE011C96EA0FFB1F008351E05E
:1032BA0000E001C0550F1F5F8DCFDE0117960E94F7
:1032CA00B10910E0133008F0C5C0A4E4BEE0E12F54
:1032DA00F0E0EE0FFF1FAE0FBF1F11964C9140306A
:1032EA0009F4B6C0A4E4BEE0E12FF0E0EE0FFF1F40
:1032FA00AE0FBF1FEC91EF773E2FA42F0E94E03D47
:10330A000E2FA4E4BEE0E12FF0E0EE0FFF1FAE0F98
:10331A00BF1FEC91EE1FE0E0EE1FE1700E1799F06F
:10332A0031E0A4E4BEE0E12FF0E0EE0FFF1FAE0FA4
:10333A00BF1FE02FE170E795E0E0E7950E2EEC91D4
:10334A00EF77E029EC93313008F473C03150303014
:10335A0009F06FC0A1E7B6E00E9447DD3E2FA2E761
:10336A00B6E0E12FF0E0BD01A5E1B0E00E942DDC5E
:10337A00DB01AE0FBF1F0E943FDDEC8BFD8B6E8B16
:10338A007F8BAC89BD898E899F89A030E8E0BE0712
:10339A00E0E08E07E0E09E0740F4EF81EF7EEF83E6
:1033AA00EC89FD89E887F9870BC0EF81E061EF833B
:1033BA00EC89FD896E897F89E887F9876A877B8727
:1033CA00EF81E07FE860EF83A4E4BEE0E12FF0E064
:1033DA00EE0FFF1FAE0FBF1FEC91E07869F0A2E776
:1033EA00B6E0E12FF0E0BD01A5E1B0E00E942DDCDE
:1033FA00E60FF71F35960CC0A2E7B6E0E12FF0E022
:10340A00BD01A5E1B0E00E942DDCE60FF71F3D9655
:10341A00E88FF98FFE013C96FA93EA93EA8DFB8DC9
:10342A00FA93EA93A8E00E948529DE0117960E9482
:10343A00B109A4E4BEE0E12FF0E0EE0FFF1FAE0FEA
:10344A00BF1FE32FEF770E2EEC91E078E029EC9383
:10345A001F5F38CF0E947FDB6A9608951A93A4EA09
:10346A00B5E0E0E00E9463DDA5EAB5E0E0E0F0E067
:10347A0060E070E00E9453DD10E0123148F4A9EADE
:10348A00B5E0EE27A10FBE1F0E9463DD1F5FF5CFD7
:10349A00E1E7F6E0FA93EA93AAE60E94BA29E0E0A5
:1034AA00F8E4FA93EA93A0E5B0E00E945A2DABEB58
:1034BA00B5E0E0E00E9463DDACEBB5E0E0E0F0E00F
:1034CA0060E070E00E9453DD10E0103348F4A0EC95
:1034DA00B5E0EE27A10FBE1F0E9463DD1F5FF5CF87
:1034EA00A0EFB5E0E0E00E9463DDA1EFB5E0E0E027
:1034FA00F0E060E070E00E9453DD10E0103348F421
:10350A00A5EFB5E0EE27A10FBE1F0E9463DD1F5F86
:10351A00F5CFA5E2B6E0E0E00E9463DDA6E2B6E000
:10352A00E0E0F0E060E070E00E9453DD10E010346B
:10353A0048F4AAE2B6E0EE27A10FBE1F0E9463DD9F
:10354A001F5FF5CFAAE6B6E0E0E00E9463DDABE6D6
:10355A00B6E0E0E0F0E060E070E00E9453DDAFE644
:10356A00B6E0EFEFFFEF0E945BDDA2C21A93ADEB6C
:10357A00B2E00E9443DDDF010E945605A6ECB2E0EC
:10358A000E9447DDE170ABE0B9E0E1700E2EEC91EC
:10359A00EE7FE029EC93E0E0E0930609EDE5F4E044
:1035AA00FA93EA93E0E0EA93A6EEB2E00E9477D4B7
:1035BA00A1ECB2E00E9447DDE0935E04A0915E04B4
:1035CA00A53018F4E5E0E0935E04A6ECB2E00E94B0
:1035DA0047DDE695E170A3E6B4E0E170E795E0E047
:1035EA00E7950E2EEC91EF77E029EC93A2ECB2E08E
:1035FA000E943FDDE0935F04F093600460936104EE
:10360A0070936204E0E0E0936A0410E0143308F077
:10361A001DC2ACECB2E0E12FF0E0BD01AEE0B0E0DB
:10362A000E942DDCDB01AE0FBF1F1A960E9447DDF8
:10363A00E07809F409C2ABE6B4E0E12FF0E0BD019D
:10364A00AEE0B0E00E942DDCDB01AE0FBF1F1A9680
:10365A00EC91E068EC93ABE6B4E0E12FF0E0BD0159
:10366A00AEE0B0E00E942DDCE60FF71FFF93EF9368
:10367A00ACECB2E0E12FF0E0BD01AEE0B0E00E94B8
:10368A002DDCDB01AE0FBF1F0E943FDDAF91BF9162
:10369A00ED93FD936D937C93ABE6B4E0E12FF0E0FC
:1036AA00BD01AEE0B0E00E942DDCE60FF71F3496B4
:1036BA00FF93EF93ACECB2E0E12FF0E0BD01AEE096
:1036CA00B0E00E942DDCDB01AE0FBF1F14960E94F2
:1036DA0043DDAF91BF91ED93FC93ABE6B4E0E12FEC
:1036EA00F0E0BD01AEE0B0E00E942DDCE60FF71F6E
:1036FA003696FF93EF93ACECB2E0E12FF0E0BD0118
:10370A00AEE0B0E00E942DDCDB01AE0FBF1F1696C3
:10371A000E9443DDAF91BF91ED93FC93ABE6B4E019
:10372A00E12FF0E0BD01AEE0B0E00E942DDCE60F33
:10373A00F71F3896FF93EF93ACECB2E0E12FF0E07D
:10374A00BD01AEE0B0E00E942DDCDB01AE0FBF1F71
:10375A0018960E9443DDAF91BF91ED93FC93ABE6BF
:10376A00B4E0E12FF0E0BD01AEE0B0E00E942DDC54
:10377A00E60FF71F3A96FF93EF93ACECB2E0E12F16
:10378A00F0E0BD01AEE0B0E00E942DDCDB01AE0F3F
:10379A00BF1F1A960E9447DDEF70AF91BF91EF707D
:1037AA000E2EEC91E07FE029EC93ABE6B4E0E12F3A
:1037BA00F0E0BD01AEE0B0E00E942DDCE60FF71F9D
:1037CA003A96FF93EF93ACECB2E0E12FF0E0BD0143
:1037DA00AEE0B0E00E942DDCDB01AE0FBF1F1A96EF
:1037EA000E9447DDE295E770AF91BF91E770E295DD
:1037FA00E07F0E2EEC91EF78E029EC93ABE6B4E093
:10380A00E12FF0E0BD01AEE0B0E00E942DDCE60F52
:10381A00F71F3B96FF93EF93ACECB2E0E12FF0E099
:10382A00BD01AEE0B0E00E942DDCDB01AE0FBF1F90
:10383A001B960E9447DDEF70AF91BF91EF700E2E7D
:10384A00EC91E07FE029EC93ABE6B4E0E12FF0E005
:10385A00BD01AEE0B0E00E942DDCE60FF71F3B96FB
:10386A00FF93EF93ACECB2E0E12FF0E0BD01AEE0E4
:10387A00B0E00E942DDCDB01AE0FBF1F1B960E9439
:10388A0047DDE295EF70AF91BF91EF70E295E07F6F
:10389A000E2EEC91EF70E029EC93ABE6B4E0E12F49
:1038AA00F0E0BD01AEE0B0E00E942DDCE60FF71FAC
:1038BA003C96FF93EF93ACECB2E0E12FF0E0BD0150
:1038CA00AEE0B0E00E942DDCDB01AE0FBF1F1C96FC
:1038DA000E9447DDE170AF91BF91E1700E2EEC912D
:1038EA00EE7FE029EC93ABE6B4E0E12FF0E0BD0116
:1038FA00AEE0B0E00E942DDCE60FF71F3C96FF9386
:10390A00EF93ACECB2E0E12FF0E0BD01AEE0B0E045
:10391A000E942DDCDB01AE0FBF1F1C960E9447DD03
:10392A00E695E170AF91BF91E170EE0F0E2EEC912A
:10393A00ED7FE029EC93ABE6B4E0E12FF0E0BD01C6
:10394A00AEE0B0E00E942DDCE60FF71F3C96FF9335
:10395A00EF93ACECB2E0E12FF0E0BD01AEE0B0E0F5
:10396A000E942DDCDB01AE0FBF1F1C960E9447DDB3
:10397A00E695E695E370AF91BF91E370EE0FEE0F17
:10398A000E2EEC91E37FE029EC93ABE6B4E0E12F55
:10399A00F0E0BD01AEE0B0E00E942DDCE60FF71FBB
:1039AA003C96FF93EF93ACECB2E0E12FF0E0BD015F
:1039BA00AEE0B0E00E942DDCDB01AE0FBF1F1C960B
:1039CA000E9447DDE295E170AF91BF91E170E29507
:1039DA00E07F0E2EEC91EF7EE029EC93ABE6B4E0AB
:1039EA00E12FF0E0BD01AEE0B0E00E942DDCDB018A
:1039FA00AE0FBF1F1C96EC91EC70E43089F0ABE679
:103A0A00B4E0E12FF0E0BD01AEE0B0E00E942DDCB1
:103A1A00DB01AE0FBF1F1C96EC91EC70EC3081F409
:103A2A00ABE6B4E0E12FF0E0BD01AEE0B0E00E9409
:103A3A002DDCDB01AE0FBF1F1C96EC91E068EC9306
:103A4A00E12FEF5FE0936A041F5FE0CDE4E6F4E064
:103A5A00FA93EA93E0E4F1E0FA93EA93A5E00E948C
:103A6A008529E0916504F09166046091670470917C
:103A7A00680430976040704021F4E0916404EF7E5E
:103A8A0015C0E0916404E061E0936404F0E0F69507
:103A9A00E795E370F070E330A0E0FA0721F0E13037
:103AAA00A0E0FA0729F4E0916404E860E093640472
:103ABA0019910895BA93AA936D970E9478DBE0E072
:103ACA00EE8BABA1BCA1EC91E295E1703E2F3030B8
:103ADA00C1F01196ED91FD916D917D91ED8FFE8F63
:103AEA006F8F78A3E0915F04F091600460916104A4
:103AFA0070916204AD8DBE8D8F8D98A10E9425DCD8
:103B0A000CC0ABA1BCA111964D915C91A0915F0430
:103B1A00B0916004FA010E9413DCE88FE03099F159
:103B2A00ABA1BCA1EC91EF70E13038F0EBA1FCA1A4
:103B3A00A581A17011F00E94672BABA1BCA1EC91E9
:103B4A00EF70E63000F120E0E1E0EA8FE98F2732FA
:103B5A00D0F4ABA1BCA11596EA8DF0E0AE0FBF1F61
:103B6A00EC91A98DEA2319F0A22F0E941E71E98D0A
:103B7A00EE0FE98FE03029F4EA8DEF5FEA8FE1E09A
:103B8A00E98F2F5FE4CFE0916404E07109F43FC04C
:103B9A00303079F0E0916504F09166046091670431
:103BAA0070916804AD8DBE8D8F8D98A10E9425DC21
:103BBA0007C0A0916504B0916604FA010E9413DC63
:103BCA00E88FE03021F1EBA1FCA1A581A17071F091
:103BDA00E0916404E17021F0E0916404E77F03C09E
:103BEA00E0916404E860E09364040DC0E091640429
:103BFA00E17021F0E0916404E86003C0E09164049C
:103C0A00E77FE0936404E0915E04E0936904E09145
:103C1A006304EF70E23011F4E1E0EE8BA0916A04E4
:103C2A00A433A0F0EEEBF2E060E070E00E9405DD64
:103C3A00E0916A04FF27662777270E9405DD84E062
:103C4A000E94FFDA2896E4E3E0936A0420E0E09118
:103C5A006A042E1708F04FC5ABE6B4E0E22FF0E095
:103C6A00BD01AEE0B0E00E942DDCE60FF71F8F0128
:103C7A00E285E07809F43DC5303061F0D801ED9174
:103C8A00FD916D917D91AD8DBE8D8F8D98A10E9414
:103C9A0025DC07C0D801ED91FD91DF01FA010E94F0
:103CAA0013DCE88FE03009F424C5E0916304E07482
:103CBA0009F40DC5F801E485E07171F1ACECB2E0EC
:103CCA00E22FF0E0BD01AEE0B0E00E942DDCDB01A6
:103CDA00AE0FBF1F1C960E9447DDE295EF70E69576
:103CEA00E770ABA1BCA11596F0E0AE0FBF1FEC9137
:103CFA00EF93ACECB2E0E22FF0E0BD01AEE0B0E051
:103D0A000E942DDCDB01AE0FBF1F1D960E9447DD0E
:103D1A00AF91EA1709F0DBC4ABE6B4E0E22FF0E0BA
:103D2A00BD01AEE0B0E00E942DDCDB01AE0FBF1F8B
:103D3A001D96E0915E04EC93E0E0E9A3EAA3F801A2
:103D4A00E385EF70E13038F1ABA1BCA11596F8011B
:103D5A00E385F0E0EF70F0703197AE0FBF1FEC9182
:103D6A00F0E0E9A3FAA3F9A1E0E0E9A3FAA3ABA181
:103D7A00BCA11596F801E385F0E00E9404DCEF701F
:103D8A00F0703197AE0FBF1FEC91A9A1BAA1F0E074
:103D9A00EA2BFB2B0FC0ABA1BCA11596F801E3855A
:103DAA00F0E00E9404DCEF70F0703197AE0FBF1F95
:103DBA00EC91F0E0E9A3FAA3D8011896ED91FD91F0
:103DCA00A9A1BAA1EA23FB23E9A3FAA3F801E4858E
:103DDA00E17059F0F801A085B185FD01F695E795E6
:103DEA00A9A1BAA1EA17FB0708F00CC0D8011896D6
:103DFA00ED91FD91E095F095A9A1BAA1EA2BFB2BD3
:103E0A00E9A3FAA3F801E485E295EF70E695E69551
:103E1A00E170EF8BF801E485E17009F456C2E9A17B
:103E2A00FAA1EB8FFC8FF801E285F0E0EF70F070F9
:103E3A00E630A0E0FA0709F4C7C13097C9F4AB8DA0
:103E4A00BC8D00240A160B0624F4EB8DFC8DF29629
:103E5A0006C0AC8DAA232AF4EB8DFC8DF297EB8F6A
:103E6A00FC8FAB8DBC8DE4E6F0E00E9486DCAAC133
:103E7A00E130A0E0FA07C9F4AB8DBC8D00240A1624
:103E8A000B0624F4EB8DFC8D799606C0AC8DAA2323
:103E9A002AF4EB8DFC8D7997EB8FFC8FAB8DBC8D63
:103EAA00E2E3F0E00E9486DC8DC1E230A0E0FA078E
:103EBA00C9F4AB8DBC8D00240A160B0624F4EB8DD5
:103ECA00FC8D3A9606C0AC8DAA232AF4EB8DFC8DA4
:103EDA003A97EB8FFC8FAB8DBC8DE4E1F0E00E944A
:103EEA0086DC70C1E330A0E0FA07C9F4AB8DBC8D63
:103EFA0000240A160B0624F4EB8DFC8D359606C0B9
:103F0A00AC8DAA232AF4EB8DFC8D3597EB8FFC8FB1
:103F1A00AB8DBC8DEAE0F0E00E9486DC53C1E43050
:103F2A00A0E0FA07C9F4AB8DBC8D00240A160B0673
:103F3A0024F4EB8DFC8D339606C0AC8DAA232AF4AB
:103F4A00EB8DFC8D3397EB8FFC8FAB8DBC8DE5E051
:103F5A00F0E00E9486DC36C1E530A0E0FA07C9F439
:103F6A00AB8DBC8D00240A160B0624F4EB8DFC8D58
:103F7A00329606C0AC8DAA232AF4EB8DFC8D3297BB
:103F8A00EB8FFC8FAB8DBC8DE2E0F0E00E9486DC0B
:103F9A0019C1E730A0E0FA0741F5AB8DBC8D0024CA
:103FAA000A160B0674F4AF3FEFE3BE071CF0EFEFFF
:103FBA00FFE704C0EB8DFC8DEE0FFF1FEB8FFC8F2C
:103FCA0013C0AC8DAA2382F4AB8DBC8DE0E0F0EC7B
:103FDA00EA17FB071CF0E0E0F0E804C0EB8DFC8D6B
:103FEA00EE0FFF1FEB8FFC8FEFC0E830A0E0FA075F
:103FFA0061F5AB8DBC8D00240A160B0684F4A93931
:10400A00E9E1BE071CF0EFEFFFE706C0EB8DFC8D80
:10401A00A5E0B0E00E945BDCEB8FFC8F15C0AC8D95
:10402A00AA2392F4AB8DBC8DE7E6F6EEEA17FB07FE
:10403A001CF0E0E0F0E806C0EB8DFC8DA5E0B0E0F6
:10404A000E945BDCEB8FFC8FBFC0E930A0E0FA076F
:10405A0061F5AB8DBC8D00240A160B0684F4AC3CCA
:10406A00ECE0BE071CF0EFEFFFE706C0EB8DFC8D1E
:10407A00AAE0B0E00E945BDCEB8FFC8F15C0AC8D30
:10408A00AA2392F4AB8DBC8DE4E3F3EFEA17FB07A6
:10409A001CF0E0E0F0E806C0EB8DFC8DAAE0B0E091
:1040AA000E945BDCEB8FFC8F8FC0EA30A0E0FA073E
:1040BA0061F5AB8DBC8D00240A160B0684F4A63676
:1040CA00E6E0BE071CF0EFEFFFE706C0EB8DFC8DC4
:1040DA00A4E1B0E00E945BDCEB8FFC8F15C0AC8DD5
:1040EA00AA2392F4AB8DBC8DEAE9F9EFEA17FB0734
:1040FA001CF0E0E0F0E806C0EB8DFC8DA4E1B0E036
:10410A000E945BDCEB8FFC8F5FC0EB30A0E0FA070C
:10411A0061F5AB8DBC8D00240A160B0684F4AF380A
:10412A00E2E0BE071CF0EFEFFFE706C0EB8DFC8D67
:10413A00A2E3B0E00E945BDCEB8FFC8F15C0AC8D74
:10414A00AA2392F4AB8DBC8DE1E7FDEFEA17FB07DA
:10415A001CF0E0E0F0E806C0EB8DFC8DA2E3B0E0D5
:10416A000E945BDCEB8FFC8F2FC0EC30A0E0FA07DB
:10417A0059F5AB8DBC8D00240A160B0684F4A734BE
:10418A00E1E0BE071CF0EFEFFFE706C0EB8DFC8D08
:10419A00A4E6B0E00E945BDCEB8FFC8F15C0AC8D0F
:1041AA00AA2392F4AB8DBC8DE1E7FDEFEA17FB077A
:1041BA001CF0E0E0F0E806C0EB8DFC8DA4E6B0E070
:1041CA000E945BDCEB8FFC8FF801E285F0E00E9435
:1041DA0004DCE770F070309769F4F801A481B581C6
:1041EA00EB8DFC8DEA17FB0711F4E1E001C0E0E07A
:1041FA00EF8B6AC0E130A0E0FA0769F4F801A48104
:10420A00B581EB8DFC8DEA17FB0711F4E0E001C0E4
:10421A00E1E0EF8B59C0E230A0E0FA07D9F4EF8968
:10422A00E03061F0D8011696ED91FD91AB8DBC8D11
:10423A00EA17FB0714F0E0E0EF8B0BC0D8011496E5
:10424A00ED91FD91AB8DBC8DEA17FB0714F4E1E00B
:10425A00EF8B3AC0E330A0E0FA07D9F4EF89E030F7
:10426A0061F0D8011696ED91FD91AB8DBC8DAE171C
:10427A00BF0714F0E0E0EF8B0BC0D8011496ED9164
:10428A00FD91AB8DBC8DAE17BF0714F4E1E0EF8B47
:10429A001BC0E430A0E0FA07B9F4D8011496ED91F6
:1042AA00FD91AB8DBC8DAE17BF074CF0D8011696A9
:1042BA00ED91FD91AB8DBC8DEA17FB070CF402C0A2
:1042CA00E1E001C0E0E0EF8B75C1F801E285F0E0C2
:1042DA00EF70F070E630A0E0FA0709F4CCC030972E
:1042EA0061F4E9A1FAA1F296E9A3FAA3A9A1BAA1F4
:1042FA00E4E6F0E00E9473DCBCC0E130A0E0FA071B
:10430A0061F4E9A1FAA17996E9A3FAA3A9A1BAA14C
:10431A00E2E3F0E00E9473DCACC0E230A0E0FA070E
:10432A0061F4E9A1FAA13A96E9A3FAA3A9A1BAA16B
:10433A00E4E1F0E00E9473DC9CC0E330A0E0FA07FD
:10434A0061F4E9A1FAA13596E9A3FAA3A9A1BAA150
:10435A00EAE0F0E00E9473DC8CC0E430A0E0FA07E7
:10436A0061F4E9A1FAA13396E9A3FAA3A9A1BAA132
:10437A00E5E0F0E00E9473DC7CC0E530A0E0FA07DB
:10438A0041F4E9A1FAA13196E9A3FAA3F695E795D2
:10439A0070C0E730A0E0FA0781F4A9A1BAA1AF3F43
:1043AA00EFE7BE0728F4E9A1FAA1EE0FFF1F02C04A
:1043BA00EFEFFFEFE9A3FAA35EC0E830A0E0FA0747
:1043CA0079F4A9A1BAA1A333E3E3BE0720F4E5E097
:1043DA000E9455DC02C0EFEFFFEFE9A3FAA34BC03E
:1043EA00E930A0E0FA0779F4A9A1BAA1A939E9E16B
:1043FA00BE0720F4EAE00E9455DC02C0EFEFFFEFAF
:10440A00E9A3FAA338C0EA30A0E0FA0779F4A9A12F
:10441A00BAA1AC3CECE0BE0720F4E4E10E9455DC12
:10442A0002C0EFEFFFEFE9A3FAA325C0EB30A0E04B
:10443A00FA0779F4A9A1BAA1AE31E5E0BE0720F4E2
:10444A00E2E30E9455DC02C0EFEFFFEFE9A3FAA313
:10445A0012C0EC30A0E0FA0771F4A9A1BAA1AF38F2
:10446A00E2E0BE0720F4E4E60E9455DC02C0EFEF6A
:10447A00FFEFE9A3FAA3F801E285F0E00E9404DC69
:10448A00E770F070309769F4F801A481B581E9A169
:10449A00FAA1EA17FB0711F4E1E001C0E0E0EF8BB3
:1044AA0089C0E130A0E0FA0769F4F801A481B58176
:1044BA00E9A1FAA1EA17FB0711F0E0E001C0E1E087
:1044CA00EF8B78C0E230A0E0FA07D1F5F801E48575
:1044DA00E170D9F0EF89E03061F0D8011696ED91DC
:1044EA00FD91A9A1BAA1EA17FB0714F0E0E0EF8B4E
:1044FA000BC0D8011496ED91FD91A9A1BAA1EA17B2
:10450A00FB0714F4E1E0EF8B1AC0EF89E03061F0A9
:10451A00D8011696ED91FD91A9A1BAA1EA17FB0758
:10452A0010F0E0E0EF8B0BC0D8011496ED91FD91ED
:10453A00A9A1BAA1EA17FB0710F4E1E0EF8B3AC090
:10454A00E330A0E0FA07D9F4EF89E03061F0D8014E
:10455A001696ED91FD91A9A1BAA1AE17BF0710F069
:10456A00E0E0EF8B0BC0D8011496ED91FD91A9A163
:10457A00BAA1AE17BF0710F4E1E0EF8B1BC0E4301D
:10458A00A0E0FA07B9F4D8011496ED91FD91A9A11A
:10459A00BAA1AE17BF0748F0D8011696ED91FD9162
:1045AA00A9A1BAA1EA17FB0708F402C0E1E001C019
:1045BA00E0E0EF8BF801E485E27009F448C0F80105
:1045CA00E485E07419F4EF89E03009F43FC0F8019A
:1045DA00E485E078F1F0D8011C96EC91EF77EC9342
:1045EA00E0916304E073E03298F0E1EDF2E060E01C
:1045FA0070E00E9405DDE22FF0E031966F2F660F22
:10460A00660B762F0E9405DD84E00E94FFDA289669
:10461A001DC0D8011C96EC91E068EC93E09163040C
:10462A00E073E03298F0ECEDF2E060E070E00E94B6
:10463A0005DDE22FF0E031966F2F660F660B762FBD
:10464A000E9405DD84E00E94FFDA289633C0F80153
:10465A00E485EE1FE0E0EE1FE170AE2FEF89EA1766
:10466A0049F1D8011C96E170E795E0E0E7950E2E36
:10467A00EC91EF77E029EC93E0916304E073E03288
:10468A00C8F0E7EEF2E060E070E00E9405DDE22F9C
:10469A00F0E031966F2F660F660B762F0E9405DDCC
:1046AA00EF8DFF27662777270E9405DD88E00E94A5
:1046BA00FFDA2C96D8011C96EF89E170E295E07F2B
:1046CA00EE0FEE0F0E2EEC91EF7BE029EC93E091CA
:1046DA006304EF70E13059F0E0916304EF70AE2F9C
:1046EA00E22FF0E03396B0E0EA17FB0711F4E1E0BD
:1046FA00EE8B2F5FACCAE0916304EF70E23019F0E1
:10470A00EE89E030A1F1ABA1BCA1EC91EF70ED878D
:10471A00AD85A93010F0E8E0ED87ED85E85FEF831D
:10472A00E6E0E887ABA1BCA1EC91E07121F011961B
:10473A000E94EADC07C0ABA1BCA11196ED91FD91E4
:10474A0066277727E987FA876B877C87FE013E967B
:10475A00FA93EA93EDA1FEA13596FA93EA93A98911
:10476A00BB270E9465D4DE0116960E94CA9F0E944A
:10477A007FDBA59608951A930A93AFEBB2E00E94E5
:10478A0047DD0E2F003029F0A02F0E94E03DE030D7
:10479A0021F0E0916304E06403C0E0916304EF7BDD
:1047AA00E093630410E0E0916A041E1708F07DC0EC
:1047BA00ABE6B4E0E12FF0E0BD01AEE0B0E00E946C
:1047CA002DDCDB01AE0FBF1F1D96AC91A13008F4A2
:1047DA006AC0ABE6B4E0E12FF0E0BD01AEE0B0E0C4
:1047EA000E942DDCDB01AE0FBF1F1D96EC91E1503C
:1047FA00EC93ABE6B4E0E12FF0E0BD01AEE0B0E04F
:10480A000E942DDCDB01AE0FBF1F1D96EC91E0303C
:10481A0009F049C0ABE6B4E0E12FF0E0BD01AEE03B
:10482A00B0E00E942DDCDB01AE0FBF1F1C96EC919D
:10483A00F0E00E9408DCE370F070309781F4ABE698
:10484A00B4E0E12FF0E0BD01AEE0B0E00E942DDC63
:10485A00DB01AE0FBF1F1C96EC91EF7713C0E1305E
:10486A00A0E0FA0701F5ABE6B4E0E12FF0E0BD0104
:10487A00AEE0B0E00E942DDCDB01AE0FBF1F1C963C
:10488A00EC91E068EC93ABE6B4E0E12FF0E0BD0117
:10489A00AEE0B0E00E942DDCDB01AE0FBF1F1C961C
:1048AA00EC91EF7BEC931F5F7ECFA0916904A1305E
:1048BA0000F1E0916904E150E0936904EF5FE0914F
:1048CA006904E030B1F4E0916404F0E0F695E7950C
:1048DA00E370F070309721F4E0916404E77F07C039
:1048EA00E130A0E0FA0729F4E0916404E860E0937B
:1048FA0064040C948229A0971A93A1E4B1E0E0E041
:10490A00F0E060E070E00E9453DDADEBB2E0E4EF6E
:10491A00F1E00E945BDDAFEBB2E0E0E00E9463DD14
:10492A00A0ECB2E00E9463DDA8ECB2E0E0E10E94F4
:10493A0063DDA1ECB2E0E5E00E9463DDA2ECB2E047
:10494A00E0E0F0E060E070E00E9453DDA6ECB2E047
:10495A000E9447DDE1600E9463DDFE017196FA93D1
:10496A00EA93E0E0EA93A0E1B0E00E9477D4FE0186
:10497A003196FA93EA93E0E0EA93A0E1B0E00E946C
:10498A0077D410E0143308F046C1ACECB2E0E12F62
:10499A00F0E0BD01AEE0B0E00E942DDCDB01AE0F1D
:1049AA00BF1FE0E0F0E060E070E00E9453DDACEC95
:1049BA00B2E0E12FF0E0BD01AEE0B0E00E942DDCF4
:1049CA00DB01AE0FBF1F1496E0E0F0E00E945BDD52
:1049DA00ACECB2E0E12FF0E0BD01AEE0B0E00E9445
:1049EA002DDCDB01AE0FBF1F1696E0E0F0E00E945F
:1049FA005BDDACECB2E0E12FF0E0BD01AEE0B0E08F
:104A0A000E942DDCDB01AE0FBF1F1896EFEFFFEF00
:104A1A000E945BDDACECB2E0E12FF0E0BD01AEE05C
:104A2A00B0E00E942DDCDB01AE0FBF1F1A960E9478
:104A3A0047DDE07FE6600E9463DDACECB2E0E12F87
:104A4A00F0E0BD01AEE0B0E00E942DDCDB01AE0F6C
:104A5A00BF1F1A960E9447DDEF78E0620E9463DD6D
:104A6A00ACECB2E0E12FF0E0BD01AEE0B0E00E94B4
:104A7A002DDCDB01AE0FBF1F1A960E9447DDEF77D0
:104A8A000E9463DDACECB2E0E12FF0E0BD01AEE0E4
:104A9A00B0E00E942DDCDB01AE0FBF1F1C960E9406
:104AAA0047DDEE7F0E9463DDACECB2E0E12FF0E07F
:104ABA00BD01AEE0B0E00E942DDCDB01AE0FBF1FEE
:104ACA001B960E9447DDE07F0E9463DDACECB2E0FA
:104ADA00E12FF0E0BD01AEE0B0E00E942DDCDB0189
:104AEA00AE0FBF1F1B960E9447DDEF700E9463DD69
:104AFA00ACECB2E0E12FF0E0BD01AEE0B0E00E9424
:104B0A002DDCDB01AE0FBF1F1C960E9447DDED7F37
:104B1A000E9463DDACECB2E0E12FF0E0BD01AEE053
:104B2A00B0E00E942DDCDB01AE0FBF1F1C960E9475
:104B3A0047DDE37F0E9463DDACECB2E0E12FF0E0F9
:104B4A00BD01AEE0B0E00E942DDCDB01AE0FBF1F5D
:104B5A001C960E9447DDEF7E0E9463DDACECB2E05A
:104B6A00E12FF0E0BD01AEE0B0E00E942DDCDB01F8
:104B7A00AE0FBF1F1C960E9447DDEF710E9463DDD6
:104B8A00ACECB2E0E12FF0E0BD01AEE0B0E00E9493
:104B9A002DDCDB01AE0FBF1F1D96E0E00E9463DD36
:104BAA00FE017196FA93EA93E3EFF2E060E070E0B7
:104BBA000E9405DDE12FF0E031966F2F660F660B3C
:104BCA00762F0E9405DD84E00E94C4DA2A96E12F3E
:104BDA00F0E0A0EDBCE30E94F2DBEA0FFB1FFA93C0
:104BEA00EA93FE017396FA93EA93A0E10E94502C8D
:104BFA00E12FF0E0A0E1B0E40E94F4DBEA0FFB1F32
:104C0A00FA93EA93FE013396FA93EA93A8E00E9494
:104C1A00502C1F5FB7CE0E94BB1A1881A196089527
:104C2A001A93E3E4F7E0FA93EA93E0E0EA93ACE359
:104C3A00B0E00E9477D410E0143108F040C0AFE031
:104C4A00B7E0E12FF0E0BD01A6E0B0E00E942DDC64
:104C5A00DB01AE0FBF1F0E9447DDE03071F1A3E018
:104C6A001A9FF001ED5BF84FDF01EC91E160EC93E4
:104C7A00A3E01A9FF001ED5BF84FFF93EF93AFE0CB
:104C8A00B7E0E12FF0E0BD01A6E0B0E00E942DDC24
:104C9A00DB01AE0FBF1F12960E9443DDDF01EEE07B
:104CAA000E94B3DBE370AF91BF91E370E295E07FBE
:104CBA000E2EEC91EF7CE029EC931F5FBDCF19918A
:104CCA0008950E9478DB10E0143108F013C2A3E0C3
:104CDA001A9FF001ED5BF84FE081E17009F408C218
:104CEA00AFE0B7E0E12FF0E0BD01A6E0B0E00E943E
:104CFA002DDCDB01AE0FBF1F0E9447DDAE2F0E94E5
:104D0A00E03D0E2FA3E01A9FF001ED5BF84FE08122
:104D1A00F0E00E9404DCE370F070309709F07AC08A
:104D2A00003009F45BC01A9FF001ED5BF84FE08197
:104D3A00E47009F052C0AFE0B7E0E12FF0E0BD0146
:104D4A00A6E0B0E00E942DDCDB01AE0FBF1F129679
:104D5A000E9443DDFF73AF0100240416050688F4A0
:104D6A00A3E01A9FF001ED5BF84FDF01EC91E860D8
:104D7A00EC93A3E01A9FF001EC5BF84F4083518358
:104D8A002CC0A3E01A9FF001ED5BF84FDF01EC9114
:104D9A00E77FEC93A3E01A9FF001ED5BF84FDF0188
:104DAA00EC91E260EC93A3E01A9FF001EC5BF84F00
:104DBA00FF93EF93AFE0B7E0E12FF0E0BD01A6E08B
:104DCA00B0E00E942DDCDB01AE0FBF1F14960E94DB
:104DDA0043DDAF91BF91ED93FC931BC0A3E01A9FF3
:104DEA00F001EC5BF84FA0E0B0E0A083B183A3E050
:104DFA001A9FF001ED5BF84FDF01EC91E77FEC932E
:104E0A00A3E01A9FF001ED5BF84FDF01EC91ED7F13
:104E1A00EC931DC1E130A0E0FA0709F063C0A0914C
:104E2A00210EAB3008F413C1003041F4A3E01A9FFD
:104E3A00F001ED5BF84FE081E47009F452C0AFE095
:104E4A00B7E0E12FF0E0BD01A6E0B0E00E942DDC62
:104E5A00DB01AE0FBF1F12960E9443DDFF73AF0145
:104E6A0000240416050688F4A3E01A9FF001ED5BFE
:104E7A00F84FDF01EC91E860EC93A3E01A9FF00190
:104E8A00EC5BF84F408351832CC0A3E01A9FF001DA
:104E9A00ED5BF84FDF01EC91E860EC93A3E01A9F19
:104EAA00F001ED5BF84FDF01EC91E260EC93A3E0D7
:104EBA001A9FF001EC5BF84FFF93EF93AFE0B7E076
:104ECA00E12FF0E0BD01A6E0B0E00E942DDCDB019D
:104EDA00AE0FBF1F14960E9443DDAF91BF91ED93B1
:104EEA00FC93B5C0E230A0E0FA0709F05EC00030DA
:104EFA0041F0A3E01A9FF001ED5BF84FE081E47006
:104F0A0009F052C0AFE0B7E0E12FF0E0BD01A6E042
:104F1A00B0E00E942DDCDB01AE0FBF1F12960E948B
:104F2A0043DDFF73AF0100240416050688F4A3E0ED
:104F3A001A9FF001ED5BF84FDF01EC91E860EC930A
:104F4A00A3E01A9FF001EC5BF84F408351832CC019
:104F5A00A3E01A9FF001ED5BF84FDF01EC91E860E6
:104F6A00EC93A3E01A9FF001ED5BF84FDF01EC919F
:104F7A00E260EC93A3E01A9FF001EC5BF84FFF9319
:104F8A00EF93AFE0B7E0E12FF0E0BD01A6E0B0E0BB
:104F9A000E942DDCDB01AE0FBF1F14960E9443DD79
:104FAA00AF91BF91ED93FC9352C0E330A0E0FA07B2
:104FBA0009F04DC0A091210EAB3008F448C0003072
:104FCA0099F0A3E01A9FF001ED5BF84FDF01EC9135
:104FDA00E260EC93A3E01A9FF001EC5BF84FA0E0CB
:104FEA00B0E0A083B18333C0A3E01A9FF001ED5B68
:104FFA00F84FE081E47059F11A9FF001ED5BF84F28
:10500A00DF01EC91E77FEC93A3E01A9FF001ED5BDF
:10501A00F84FDF01EC91E260EC93A3E01A9FF001F4
:10502A00EC5BF84FFF93EF93AFE0B7E0E12FF0E0CE
:10503A00BD01A6E0B0E00E942DDCDB01AE0FBF1F70
:10504A0014960E9443DDAF91BF91ED93FC93A3E0C8
:10505A001A9FF001ED5BF84FDF01E02FE170EE0FD0
:10506A00EE0F0E2EEC91EB7FE029EC93AFE0B7E068
:10507A00E12FF0E0BD01A6E0B0E00E942DDCDB01EB
:10508A00AE0FBF1F11960E9447DD3E2F3030A1F0B0
:10509A00A3E01A9FF001ED5BF84FE081E87039F464
:1050AA001A9FF001ED5BF84FE081E27029F0A32F1F
:1050BA000E94E03DE03009F41BC0A3E01A9FF00112
:1050CA00ED5BF84FDF01EC91E77FEC93A3E01A9FC9
:1050DA00F001ED5BF84FDF01EC91ED7FEC93A3E07B
:1050EA001A9FF001EC5BF84FA0E0B0E0A083B18317
:1050FA001F5FEACD0E947FDB4AC11A9310E0143188
:10510A0008F069C0A3E01A9FF001ED5BF84FE08157
:10511A00E17061F01A9FF001EC5BF84FDF01ED914D
:10512A00FC91119700240E160F0608F052C0A3E056
:10513A001A9FF001EC5BF84FDF01ED91FD91319779
:10514A00FE93EE93A3E01A9FF001EC5BF84FDF01A8
:10515A00ED91FC9111973097E1F5A3E01A9FF001C8
:10516A00ED5BF84FE081E87059F11A9FF001ED5BB1
:10517A00F84FDF01EC91E77FEC93A3E01A9FF0016F
:10518A00EC5BF84FFF93EF93AFE0B7E0E12FF0E06D
:10519A00BD01A6E0B0E00E942DDCDB01AE0FBF1F0F
:1051AA0014960E9443DDAF91BF91ED93FC93A3E067
:1051BA001A9FF001ED5BF84FDF01EC91E26008C045
:1051CA00A3E01A9FF001ED5BF84FDF01EC91ED7F50
:1051DA00EC931F5F94CF0C942B2E60971A93FE01C9
:1051EA003196FA93EA93E0E0EA93A0E1B0E00E94F4
:1051FA0077D410E0143108F048C0FE013196FA93D2
:10520A00EA93E0E0EA93A6E0B0E00E9477D4AFE048
:10521A00B7E0E12FF0E0BD01A6E0B0E00E942DDC8E
:10522A00E60FF71FFA93EA93FE013396FA93EA938D
:10523A00A6E081D0FE013196FA93EA93EAEFF2E012
:10524A0060E070E00E9405DDE12FF0E031966F2FFB
:10525A00660F660B762F0E9405DD84E00E94C4DA91
:10526A002A96E12FF0E0A0E8B2E40E94F2DBEA0F0E
:10527A00FB1FFA93EA93FE013396FA93EA93A0E1AD
:10528A000E94502CA8951F5FB5CF1881619608958A
:10529A001A930A93EAE0F3E060E070E00E9405DD09
:1052AA0080E00E94FFDA24960FE010E0E5E4F1E0E6
:1052BA000E171F0738F4D801E0E00E9463DD0F5F84
:1052CA001F4FF4CF0E94E730A0E0B0E0E0E50E9473
:1052DA0063DDA1E0B0E0E3E40E9463DDA2E0B0E0B8
:1052EA00EDE40E9463DDA3E0B0E0E0E50E9463DD47
:1052FA00A4E0B0E0E0E00E9463DD0991199108950D
:10530A000E9478DB0A2F2E813F814885598510E05B
:10531A00101778F4E12FF0E0E40FF51F0F01D9011F
:10532A00EE27A10FBE1F0E9447DDD001EC931F5F3D
:10533A00EFCF0C94562D0E9478DB0A2F2E813F81E5
:10534A004885598510E0101778F4E12FF0E0E40F52
:10535A00F51F0F01D901EE27A10FBE1FEC91D00155
:10536A000E9463DD1F5FEFCF9CC30E947ADB0A2F86
:10537A002C813D8110E0101740F4D901EE27A10FCE
:10538A00BE1F0E9463DD1F5FF6CF0E9481DB269657
:10539A0008950E9478DB3A2F4E815F8110E0E32F57
:1053AA00F0E03197A12FB0E0AE17BF078CF4DA0115
:1053BA00EE27A10FBE1F0C91003051F0A885B985C8
:1053CA00EE27A10FBE1FE02F0E9463DD1F5FE7CF0C
:1053DA00A885B985EE27A10FBE1F0E9463DDE12FC4
:1053EA0060C30E9478DB3A2F4E815F8110E0E32F81
:1053FA00F0E03197A12FB0E0AE17BF0794F4DA01BD
:10540A00EE27A10FBE1F0E9447DD0E2F003049F084
:10541A00E12FA885B985F0E0EA0FFB1F00831F5F23
:10542A00E6CFA885B985EE27A10FBE1FEC93E12F21
:10543A0038C32E97D1500E947ADB10E0133030F532
:10544A00FE01E250FF4FFA93EA93E0E0F0E0FA93AC
:10545A00EA93A4E1B0E06CD1E03089F0E0911F0E4C
:10546A00EE7FE0931F0EFE01E250FF4FFA93EA939C
:10547A00ACEBB3E00E9487D4E03041F005C0E09184
:10548A001F0EE160E0931F0E1F5FD8CF133011F497
:10549A002CD194C0E0E0F0E0E093CC03F093CD038C
:1054AA0020E030E0283EE3E03E0708F059C0203D06
:1054BA00E3E03E0710F409E103C0E8EEE21B0E2F19
:1054CA00FE013496FA93EA93E091CA03F091CB0372
:1054DA0060E870E0AAE0B0E00E942DDCE60FF71F5A
:1054EA00FA93EA93EAE0E09FF001DF0121D1E0308C
:1054FA00A1F110E0101788F52F5F3F4FAAE01A9F1D
:10550A00F001DE011496AE0FBF1F1696EC91E03043
:10551A0021F1AAE01A9FF001DE011496AE0FBF1F17
:10552A00ED91FD91A091CC03B091CD03AE17BF07C9
:10553A0090F4AAE01A9FF001DE011496AE0FBF1F85
:10554A00ED91FC911197E093CC03F093CD03209356
:10555A00CA033093CB031F5FCDCF101708F0A2CF39
:10556A00ACECB3E0ED91FD913196FE93EE93A091F0
:10557A00CA03B091CB03A83EE3E0BE0728F0E0E0FF
:10558A00E093CA03E093CB03E1E2F3E060E070E06A
:10559A000E9405DDE091CA03F091CB0366277727C5
:1055AA000E9405DDE091CC03F091CD0366277727B1
:1055BA000E9405DD88E00E94FFDA2C960E9481DBBA
:1055CA006296DF5F08951A931A2F1A93E0E0EA931E
:1055DA00A0E0B0E001D03AC32A970E9478DB9D018F
:1055EA0008895989E6E3F3E060E070E00E9405DD8E
:1055FA00E52FFF27662777270E9405DDE02FFF2783
:10560A00662777270E9405DD88E00E94FFDA2C963C
:10561A00543638F0ACECB9E00E9443DD31960E9472
:10562A005BDDE091CC03F091CD03EE83FF83E09143
:10563A00F410F091F5106091F6107091F710E88768
:10564A00F9876A877B875C870D872E873F8710E0FB
:10565A001330A0F5E091CA03F091CB0360E870E043
:10566A00AAE0B0E00E942DDCE60FF71FFA93EA9356
:10567A00FE013896FA93EA93AAE00DD1E030E1F000
:10568A00ACECB3E0ED91FD913196FE93EE93AAEC6A
:10569A00B3E0ED91FD913196FE93EE93A091CA038A
:1056AA00B091CB03A83EE3E0BE0728F0E0E0E09328
:1056BA00CA03E093CB0302C01F5FCACF0E947FDBFD
:1056CA0062960895E1E0F0E0E093CC03F093CD0315
:1056DA00E0E0E093CA03E093CB03E0E8F0E0FA935A
:1056EA00EA93A0E1B7E2E1D108956497FE01FA9343
:1056FA00EA93E0E0EA93A4E1B0E00E9477D4FE01E5
:10570A00FA93EA93AAE1B3E080E090E00E94BFD462
:10571A00E2E0E887ECE0E987E0E0F0E0FA93EA9378
:10572A00FE013296FA93EA93A4E1B5D064960895FD
:10573A000E9478DBAD0110E01436C0F4A198EDB5F3
:10574A00E093160EE5E0EEBDEDB5E7FFFDCFE0E034
:10575A00EEBDEDB5E7FFFDCF0EB5A19A00FF06C07D
:10576A0080E991E00197F1F71F5FE6CF143659F40B
:10577A00E885F985FA93EA93E0E0EA93DA010E9470
:10578A0077D4E0E08EC1A198EDB5E093160EE3E080
:10579A00EEBDEDB5E7FFFDCFEF81F070EEBDEDB5E3
:1057AA00E7FFFDCFEE81EEBDEDB5E7FFFDCF20E0CF
:1057BA0030E02417350788F4EDB5E093160EE0E0E3
:1057CA00EEBDEDB5E7FFFDCFA885B985A20FB31FE2
:1057DA00EEB5EC932F5F3F4FECCFA19A61C10E94C7
:1057EA0078DB2A2F4E815F8110E01436C0F4A1982D
:1057FA00EDB5E093160EE5E0EEBDEDB5E7FFFDCFA2
:10580A00E0E0EEBDEDB5E7FFFDCF3EB5A19A30FF72
:10581A0006C080E991E00197F1F71F5FE6CF1436E1
:10582A0029F4A885B985E0E0EC933BC1213008F062
:10583A002150A198EDB5E093160EE3E0EEBDEDB56B
:10584A00E7FFFDCFE52FF070EEBDEDB5E7FFFDCF29
:10585A004EBDEDB5E7FFFDCF00E00217A0F4EDB5B0
:10586A00E093160EE0E0EEBDEDB5E7FFFDCFA885AB
:10587A00B985EE27A00FBE1FEEB5EC93EEB5E0306A
:10588A0011F00F5FEACFA19AA885B985EE27A00F7C
:10589A00BE1FEC9305C10E9478DB5A2F10E05130ED
:1058AA0008F47AC000E00436C0F4A198EDB5E0939C
:1058BA00160EE5E0EEBDEDB5E7FFFDCFE0E0EEBD8B
:1058CA00EDB5E7FFFDCF3EB5A19A30FF06C080E9EE
:1058DA0091E00197F1F70F5FE6CF043611F4E0E0AB
:1058EA00E0C0A198EDB5E093160EE6E0EEBDEDB589
:1058FA00E7FFFDCFA19A00000000A198EDB5E09363
:10590A00160EE5E0EEBDEDB5E7FFFDCFE0E0EEBD3A
:10591A00EDB5E7FFFDCF3EB5A19A31FF3AC0E88564
:10592A00EF77A0E8AE1B2A2F521708F4252FA1986B
:10593A00EDB5E093160EE2E0EEBDEDB5E7FFFDCF63
:10594A00E985F070EEBDEDB5E7FFFDCFE885EEBD68
:10595A00EDB5E7FFFDCF00E0021780F4EDB5E09367
:10596A00160EAE81BF81EE27A10FBE1FEC91EEBDD0
:10597A00EDB5E7FFFDCF0F5F1F5FEECFA19A521B78
:10598A00E22FF0E0A885B985EA0FFB1FE887F987BF
:10599A0002C0E0E086C083CF83C00E9478DB5A2F22
:1059AA0010E0513008F47CC000E00436C0F4A1983D
:1059BA00EDB5E093160EE5E0EEBDEDB5E7FFFDCFE0
:1059CA00E0E0EEBDEDB5E7FFFDCF3EB5A19A30FFB1
:1059DA0006C080E991E00197F1F70F5FE6CF043640
:1059EA0011F4E0E05EC0A198EDB5E093160EE6E092
:1059FA00EEBDEDB5E7FFFDCFA19A00000000A1982A
:105A0A00EDB5E093160EE5E0EEBDEDB5E7FFFDCF8F
:105A1A00E0E0EEBDEDB5E7FFFDCF3EB5A19A31FF5F
:105A2A003CC0E885EF77A0E8AE1B2A2F521708F48E
:105A3A00252FA198EDB5E093160EE2E0EEBDEDB587
:105A4A00E7FFFDCFE985F070EEBDEDB5E7FFFDCFCD
:105A5A00E885EEBDEDB5E7FFFDCF00E0021780F463
:105A6A00AE81BF81EE27A10FBE1F3C91EDB5E09339
:105A7A00160E3EBDEDB5E7FFFDCF0F5F1F5FEECF00
:105A8A00A19A303069F0521BE22FF0E0A885B9855F
:105A9A00EA0FFB1FE887F98702C0E0E002C081CF66
:105AAA00E1E00E947FDB2A9608950E9478DBAD012F
:105ABA0010E000240416050608F07BC000E0043656
:105ACA00C0F4A198EDB5E093160EE5E0EEBDEDB594
:105ADA00E7FFFDCFE0E0EEBDEDB5E7FFFDCF3EB558
:105AEA00A19A30FF06C080E991E00197F1F70F5FB4
:105AFA00E6CF043611F4E0E05DC0A198EDB5E0937D
:105B0A00160EE6E0EEBDEDB5E7FFFDCFA19A000067
:105B1A000000A198EDB5E093160EE5E0EEBDEDB5F7
:105B2A00E7FFFDCFE0E0EEBDEDB5E7FFFDCF3EB507
:105B3A00A19A31FF3BC0EE81EF77A0E8AE1B2A2F76
:105B4A00FA01B0E0EA17FB0708F4242FA198EDB593
:105B5A00E093160EE2E0EEBDEDB5E7FFFDCFEF8173
:105B6A00F070EEBDEDB5E7FFFDCFEE81EEBDEDB510
:105B7A00E7FFFDCF00E0021758F4EDB5E093160EEB
:105B8A00E0E0EEBDEDB5E7FFFDCF0F5F1F5FF3CF9E
:105B9A00A19AA22FBB274A1B5B0BE22FF0E0AE8132
:105BAA00BF81EA0FFB1FEE83FF8302C0E0E002C061
:105BBA0080CFE1E00E947FDB289608951A93EFE7F1
:105BCA00F7E0FA93EA93E0E0EA93A4E1B0E00E94F6
:105BDA0077D410E01530D0F5E12FAFE7B7E0F0E069
:105BEA000E94F6DBEA0FFB1F0F01ABEDB6E0E12FD7
:105BFA00F0E00E94F6DBAE0FBF1F0E9447DDD00126
:105C0A00EC93E12FAFE7B7E0F0E00E94F6DBEA0F92
:105C1A00FB1F33960F01ABEDB6E0E12FF0E00E94D7
:105C2A00F6DBAE0FBF1F13960E9447DDEE1FE0E0C2
:105C3A00EE1FE170D001E170EE0FEE0FEE0F0E2EA7
:105C4A00EC91E77FE029EC931F5FC4CF1991089587
:105C5A000E947ADB2A2F10E0153008F0CFC1E12F1D
:105C6A00AFE7B7E0F0E00E94F6DBAE0FBF1FAC91E2
:105C7A00A03081F0E12FAFE7B7E0F0E00E94F6DB59
:105C8A00AE0FBF1F1396EC91E695E695E695E17087
:105C9A002E1709F0B1C1E12FAFE7B7E0F0E00E949B
:105CAA00F6DBAE0FBF1FAC910E94E03DE03009F475
:105CBA0079C0E12FAFE7B7E0F0E00E94F6DBAE0F64
:105CCA00BF1F1396EC91E47009F06BC0E12FAFE7A8
:105CDA00B7E0F0E00E94F6DBAE0FBF1F1396EC911F
:105CEA00E160EC93E12FAFE7B7E0F0E00E94F6DB6A
:105CFA00AE0FBF1F1396EC91E460EC93E12FAFE770
:105D0A00B7E0F0E00E94F6DBEA0FFB1F33960F01C3
:105D1A00ABEDB6E0E12FF0E00E94F6DBAE0FBF1F5D
:105D2A0013960E9447DDEF77E13010F0E1E001C001
:105D3A00E0E0D001E170EE0F0E2EEC91ED7FE0294C
:105D4A00EC93E12FAFE7B7E0F0E00E94F6DBEA0F51
:105D5A00FB1F32960F01ABEDB6E0E12FF0E00E9497
:105D6A00F6DBAE0FBF1F13960E9447DDEF77D00117
:105D7A00EC93E12FAFE7B7E0F0E00E94F6DBEA0F21
:105D8A00FB1F31960F01ABEDB6E0E12FF0E00E9468
:105D9A00F6DBAE0FBF1F11960E9447DDD001EC93D0
:105DAA002BC12FC0E12FAFE7B7E0F0E00E94F6DB8E
:105DBA00AE0FBF1F1396EC91EB7FEC93E12FAFE789
:105DCA00B7E0F0E00E94F6DBAE0FBF1F1396EC912E
:105DDA00E270B9F4E12FAFE7B7E0F0E00E94F6DB3A
:105DEA00AE0FBF1F1396EC91EE7FEC93E12FAFE756
:105DFA00B7E0F0E00E94F6DBAE0FBF1F1196E0E0BD
:105E0A00EC93E12FAFE7B7E0F0E00E94F6DBAE0FCC
:105E1A00BF1F1196AC91A13008F4EEC0E12FAFE795
:105E2A00B7E0F0E00E94F6DBAE0FBF1F1196EC91CF
:105E3A00E150EC93E12FAFE7B7E0F0E00E94F6DB28
:105E4A00AE0FBF1F1196EC91E03009F0D5C0E12FDB
:105E5A00AFE7B7E0F0E00E94F6DBAE0FBF1F139684
:105E6A00EC91E17009F48CC0E2E4F3E060E070E0E8
:105E7A000E9405DDE12FF0E031966F2F660F660B69
:105E8A00762F0E9405DD84E00E94FFDA2896E12F32
:105E9A00AFE7B7E0F0E00E94F6DBAE0FBF1F139644
:105EAA00EC91EE7FEC93E12FAFE7B7E0F0E00E94D0
:105EBA00F6DBAE0FBF1F1396EC91E27009F442C0F5
:105ECA00E12FAFE7B7E0F0E00E94F6DBAE0FBF1FAD
:105EDA001296AC91A130A8F1E12FAFE7B7E0F0E05C
:105EEA000E94F6DBAE0FBF1F1296EC91E150EC93C5
:105EFA00E12FAFE7B7E0F0E00E94F6DBAE0FBF1F7D
:105F0A001296AC91A130E8F0ABEDB6E0E12FF0E0EB
:105F1A000E94F6DBAE0FBF1F12960E9447DD0E2FBE
:105F2A00E295EF70E695E6953E2F031BE6950E1B6C
:105F3A00E12FAFE7B7E0F0E00E94F6DBEA0FFB1FC4
:105F4A0001831DC0ABEDB6E0E12FF0E00E94F6DB65
:105F5A00AE0FBF1F12960E9447DD0E2FE295EF701B
:105F6A00E695E6953E2F031BE6950E1BE12FAFE75C
:105F7A00B7E0F0E00E94F6DBEA0FFB1F01833CC0AA
:105F8A00EAE4F3E060E070E00E9405DDE12FF0E072
:105F9A0031966F2F660F660B762F0E9405DD84E01F
:105FAA000E94FFDA2896E12FAFE7B7E0F0E00E94FF
:105FBA00F6DBAE0FBF1F1396EC91E160EC93ABEDED
:105FCA00B6E0E12FF0E00E94F6DBAE0FBF1F11969C
:105FDA000E9447DD0E2FE295EF70E695E6953E2F7B
:105FEA00031BE6950E1BE12FAFE7B7E0F0E00E9436
:105FFA00F6DBEA0FFB1F01831F5F2ECED5C1609728
:10600A001A93FE013196FA93EA93E0E0EA93A0E14B
:10601A00B0E00E9477D410E0153008F069C0ABED0B
:10602A00B6E0E12FF0E00E94F6DBAE0FBF1FE0E022
:10603A000E9463DDABEDB6E0E12FF0E00E94F6DBF3
:10604A00AE0FBF1F1196E5E00E9463DDABEDB6E02F
:10605A00E12FF0E00E94F6DBAE0FBF1F1296E5E0DB
:10606A000E9463DDABEDB6E0E12FF0E00E94F6DBC3
:10607A00AE0FBF1F13960E9447DDE0780E9463DDD2
:10608A00ABEDB6E0E12FF0E00E94F6DBAE0FBF1FEA
:10609A0013960E9447DDEF770E9463DDFE01319679
:1060AA00FA93EA93E1E5F3E060E070E00E9405DD2F
:1060BA00E12FF0E031966F2F660F660B762F0E9464
:1060CA0005DD84E00E94C4DA2A96E12FF0E0A0EB15
:1060DA00B1E40E94F2DBEA0FFB1FFA93EA93FE0196
:1060EA003396FA93EA93A0E10E94502C1F5F94CF53
:1060FA0065DD32C1E0E0E2B9EFEFE1B9E1E0E5B92F
:10610A00E7EFE4B9E8E1E8B9EFE1E7B9E0E2EBB9D2
:10611A00E8EBEAB9E2E0EEB9EEE7EDB9E0E8E093E0
:10612A006A00E0E0E1BBA091220EA33430F0EFE078
:10613A00E0937E00E0EFE0BB08C0E7E0E0937E007A
:10614A00E8EFE0BBE0E8E5BFE5BFE7E0E4BBEFE18D
:10615A00E3BBE1E5ECBDE1E0EDBDE6E0E093C200C2
:10616A00E8E9E093C100E0E0E093C500E3E0E093F2
:10617A00C400EDE0E4BDE0E0E6BDEFE4E7BDE2E047
:10618A00E0936E000895E0E0E093210E0E942A3920
:10619A000E9448650E9463880E94F03C0E94BB1AD4
:1061AA000E947C0B0BDD0E9415260E94A7D10E943B
:1061BA0021CA0E940CCC0E947C0B0E94E98D0E948D
:1061CA00AE47089560971A9310E01A3048F4A8E190
:1061DA00B1E0EE27A10FBE1F0E9463DD1F5FF5CF5E
:1061EA00A6E2B1E00E9447DDE07F0E9463DDA6E2FD
:1061FA00B1E00E9447DDEF7E0E9463DDA6E2B1E0D6
:10620A000E9447DDE0620E9463DDA5E2B1E0E0E0C2
:10621A000E9463DDA7E2B1E00E9463DDA8E2B1E07B
:10622A000E9463DDA9E2B1E00E9463DDAAE2B1E067
:10623A000E9463DDABE2B1E00E9463DDACE2B1E053
:10624A000E9463DDADE2B1E0E4E10E9463DDAEE20B
:10625A00B1E0E0E00E9463DDAFE2B1E00E9463DDFD
:10626A00A0E3B1E00E9463DDA1E3B1E00E9463DD37
:10627A00FE013196FA93EA93E0E0EA93A0E1B0E0F6
:10628A000E9477D4FE013196FA93EA93A3ECB3E025
:10629A000E94B2D4E0E0F8E3FA93EA93FE0133965F
:1062AA00FA93EA93A0E10E94502CE0E0E983E0E04F
:1062BA00F6E4FA93EA93FE013396FA93EA93A1E09D
:1062CA000E94502CA2E3B1E0EEE1F0E0FF700F0172
:1062DA000E9443DDE070F07FE029F1290E945BDD36
:1062EA00A4E3B1E0E0E00E9463DDA5E3B1E0EAE007
:1062FA000E9463DDA6E3B1E0E0E80E9463DDA7E364
:10630A00B1E00E9463DDE9E3F1E0FA93EA93A7E0E2
:10631A000E94BA290E94B6860E94C4880E94B64684
:10632A000E9480240E94331A6ADE0E94F2280E9488
:10633A0027D40E948CCB0E94A4D00E94359D0E9433
:10634A00D1840E943B490E94672B1DDFA8E0B0E080
:10635A00E3E00E9463DD6BD11881619608950E9483
:10636A007ADBA89522E231E000E010E02E3CE9E079
:10637A003E0748F4D9010E9447DDF0E00E0F1F1FC7
:10638A002F5F3F4FF3CFE7E6F3E060E070E00E9453
:10639A0005DDF801662777270E9405DD84E00E9463
:1063AA00FFDA2896A895F8010E9481DB24960895C1
:1063BA00EF97EF9726970E9478DBE091240EED7F06
:1063CA00E093240EEB7FE093240EE77FE093240E04
:1063DA00E0E0E093260EA8E0B0E00E9447DDE3305B
:1063EA00B1F5E091240EE260E093240EA2E2B1E05E
:1063FA000E9447DDE13039F5E091240EE460E09334
:10640A00240EADDFAF01A3E2B1E00E9443DDE887CD
:10641A00F987E985F0E0F0E04E1B5F0BE885F98526
:10642A00F0E0F0E04E1B5F0BE885F985E417F5070D
:10643A0031F4E091240EE860E093240E03C0E4E016
:10644A00E093260E03C0E2E0E093260E03C0E1E0EB
:10645A00E093260E30E040E050E0E2E2F1E0EE8325
:10646A00FF83AE81BF81AE3CE9E0BE0708F04BC0B6
:10647A00EEECF9E0EA1BFB0BE138A0E0FA0710F0BA
:10648A0010E804C0AE81EEECEA1B1E2FFE013A961C
:10649A00FA93EA93E2E2F1E0A0E0B8E20E9415DDA5
:1064AA00EA1BFB0BA885B985EA0FFB1FFA93EA934F
:1064BA00A12FBB270E949D2B303071F4AA85A130F1
:1064CA0031F0E091260EE061E093260E1CC0EB85C8
:1064DA00FC85E887F98731E000E0011760F4E02FD6
:1064EA00F0E0DE011A96AE0FBF1FEC91F0E04E0FFE
:1064FA005F1F0F5FF2CFA895EE81FF81E058FF4F33
:10650A00EE83FF83AECF313009F08BC0E985F0E02E
:10651A00F0E04E1B5F0BE885F985F0704E1B5F0BB0
:10652A00E885F985E417F50709F076C0E091240EAD
:10653A00E87009F070C0AFEFBFE00E9447DDEF5F7F
:10654A000E9463DDE091260EE064E093260EE2E20B
:10655A00F1E0EE83FF83AE81BF81AE3CE9E0BE0786
:10656A00B8F5EEECF9E0EA1BFB0BE138A0E0FA071C
:10657A0010F010E804C0AE81EEECEA1B1E2FFE01FB
:10658A003A96FA93EA93E2E2F1E0A0E0B8E20E94D6
:10659A0015DDEA1BFB0BA885B985EA0FFB1FFA93E9
:1065AA00EA93A12FBB270E949D2BEE81FF81FA93CC
:1065BA00EA93FE013C96FA93EA93A12F0E94A0293E
:1065CA00A895EE81FF81E058FF4FEE83FF83C3CF8A
:1065DA00C6DEAF01A3E2B1E00E9443DDE887F98796
:1065EA00E985F0E0F0E04E1B5F0BE885F985F0E005
:1065FA00F0E04E1B5F0BE885F985E417F50731F4E7
:10660A00E091240EE860E093240E05C0E091260E86
:10661A00E068E093260E05C0E091260EE062E09362
:10662A00260E0E947FDBEF96EF962C960895EF9741
:10663A00EF9724970E9478DBE4E7F3E060E070E0EC
:10664A000E9405DD80E00E94FFDA2496A2E2B1E012
:10665A00E1E00E9463DDA3E2B1E0E0E0F0E00E9445
:10666A005BDD7DDEAF01A3E2B1E00E9443DDEE8394
:10667A00FF83EF81F0E0F0E04E1B5F0BEE81FF81BC
:10668A00F0E0F0E04E1B5F0BA3E2B1E0FA010E94DA
:10669A005BDD22E231E02E3CE9E03E0760F5EEECFC
:1066AA00F9E0E21BF30BE138A0E0FA0710F010E87A
:1066BA0003C0EEECE21B1E2FFE013896FA93EA9312
:1066CA003A932A93A12F0E948529E2E2F1E0A0E001
:1066DA00B8E20E9415DDEA1BFB0BE20FF31FFA93E7
:1066EA00EA93FE013A96FA93EA93A12F0E94502C5C
:1066FA0020583F4FD0CFE091240EE460E093240E5F
:10670A00E860E093240EE0E0E093260EE091240E88
:10671A00E07129F0E091240EE160E093240E0E94DA
:10672A007FDBEF96EF962A960895EF97EF972297D9
:10673A000E9478DB4A2F403039F5A4E1B0E0E3E764
:10674A000E9463DDA3E2B0E0E1E00E9463DDA4E21F
:10675A00B0E0E0E0F0E00E945BDD20E030E004E140
:10676A0010E0E8E1F1E00E171F0748F4D8010E9493
:10677A0047DDF0E02E0F3F1F0F5F1F4FF2CFA4E25D
:10678A00B0E0F9010E945BDD00E010E00430E1E0D6
:10679A001E0748F5E4E0F1E0E01BF10BE138A0E068
:1067AA00FA0710F050E803C0E4E0E01B5E2FFE0198
:1067BA003696FA93EA93E4E1F0E0E00FF11FFA93D8
:1067CA00EA93A52F0E948529F801E058F140FA932F
:1067DA00EA93FE013896FA93EA93A52F0E94502C69
:1067EA0000581F4FD3CF0E947FDBEF96EF96289673
:1067FA0008950E9478DB20E030E004E110E0E8E14F
:10680A00F1E00E171F0748F4D8010E9447DDF0E0B7
:10681A002E0F3F1F0F5F1F4FF2CFA4E2B0E00E947E
:10682A0043DDAF01E52FF0E0F0E02E1B3F0BFA014C
:10683A00F0E0F0E02E1B3F0B4217530711F4E1E0A2
:10684A0001C0E0E00E947FDB26960895EF97EF975C
:10685A0025970E9478DBE0E0DE01A957BF4FEC9351
:10686A00DE01A957BF4FAC91AA3020F5A8E1B1E0EB
:10687A00FE01E957FF4FE081F0E0AE0FBF1F0E9413
:10688A0047DDDE01A857BF4FEC93DE01A857BF4F83
:10689A00AC91A03210F0AB3730F0A8E1B1E0E0E003
:1068AA000E9463DD07C0DE01A957BF4FEC91EF5F7D
:1068BA00EC93D6CFE091240EEF7EE093240EE0E035
:1068CA00DE01A957BF4FEC93DE01A957BF4FAC9128
:1068DA00A53038F5A0E0B0E00E9447DDE035C1F40C
:1068EA00A1E0B0E00E9447DDE33491F4A2E0B0E019
:1068FA000E9447DDED3461F4A3E0B0E00E9447DD79
:10690A00E03531F4A4E0B0E00E9447DDE03009F060
:10691A0001C007C0DE01A957BF4FEC91EF5FEC93AE
:10692A00D3CFDE01A957BF4FAC91A53039F40E94ED
:10693A004D29E091250EE160E093250EA3E2B0E037
:10694A000E9447DDE03061F4A4E2B0E00E9443DD3A
:10695A00309731F4A2E2B0E00E9447DDEF3109F04E
:10696A0008C0E091250EE260E093250EA0E0DDDE8E
:10697A000EC03FDFE03031F0E091240EE061E09399
:10698A00240E05C0E091250EE460E093250EE0E0B8
:10699A00DE01AA57BF4FEC93E0E0F0E08F019F01C0
:1069AA000430E1E01E0708F061C0E4E0F1E0E01B1A
:1069BA00F10BE138A0E0FA0710F0E0E802C0E4E0E9
:1069CA00E01BDE01A857BF4FEC93FE013696FA93FF
:1069DA00EA93F801E058F140FA93EA93DE01A457EA
:1069EA00BF4FAC91BB270E949D2BFE01EA57FF4F78
:1069FA00E081E030A9F4AE81A33719F4AD89A13062
:106A0A0009F008C04E895F89E1E0DE01AA57BF4F4D
:106A1A00EC9306C0E091250EE860E093250E26C0AF
:106A2A00E0E0DE01A957BF4FEC93FE01E857FF4FA4
:106A3A00E081DE01A957BF4FAC91AE17A0F4FE0169
:106A4A00E957FF4FE081F0E0DE011696AE0FBF1F57
:106A5A00EC91F0E02E0F3F1FDE01A957BF4FEC91DA
:106A6A00EF5FEC93E2CF00581F4F9ACFE52FF0E08B
:106A7A00F0E02E1B3F0BFA01F0E0F0E02E1B3F0B7B
:106A8A00DE01AA57BF4FAC91A13019F44217530740
:106A9A0009F059C0E091240EE07109F053C0E09169
:106AAA00250EE061E093250E00E010E00430E1E0FD
:106ABA001E0798F5EEECF9E0E01BF10BE138A0E0D7
:106ACA00FA0710F0E0E802C0EEECE01BDE01A8577E
:106ADA00BF4FEC93FE013696FA93EA93F801E05819
:106AEA00F140FA93EA93DE01A457BF4FAC91BB275A
:106AFA000E949D2BE4E1F0E0E00FF11FFA93EA9384
:106B0A00FE013896FA93EA93DE01A457BF4FAC917F
:106B1A000E94A02900581F4FC9CF6BDEE03069F0F0
:106B2A00E091240EE061E093240EAEEFBFE00E94F4
:106B3A0047DDEF5F0E9463DD05C0E091250EE0624C
:106B4A00E093250E17C0E091250EE064E093250E30
:106B5A00E091240EE07171F0A1E0E7DDADEFBFE056
:106B6A000E9447DDEF5F0E9463DDE091250EE06839
:106B7A00E093250E0E947FDBEF96EF962B96089501
:106B8A00EEE7F3E060E070E00E9405DDE2E0F0E0AD
:106B9A0060E070E00E9405DDECE0F0E060E070E0AB
:106BAA000E9405DD0E9405DD8CE00E94FFDA6096F6
:106BBA00E9EAF3E060E070E00E9405DDA5E1B0E0FB
:106BCA000E9443DD662777270E9405DD84E00E9444
:106BDA00FFDA2896E5EBF3E060E070E00E9405DD5D
:106BEA00A7E1B0E00E9447DDFF27662777270E94CA
:106BFA0005DDA8E1B0E00E9447DDFF276627772779
:106C0A000E9405DD88E00E94FFDA2C96EDECF3E0A5
:106C1A0060E070E00E9405DDE091220EFF27662702
:106C2A0077270E9405DDAAE1B0E00E9447DDFF2731
:106C3A00662777270E9405DD88E00E94FFDA2C96F6
:106C4A00E8EEF3E060E070E00E9405DDE091F41008
:106C5A00F091F5106091F6107091F7100E9405DD21
:106C6A0084E00E94FFDA2896E091240EE27009F48B
:106C7A0044C0E091240EE47031F1E6EFF3E060E005
:106C8A0070E00E9405DDA3E2B1E00E9443DD6627C1
:106C9A0077270E9405DD84E00E94FFDA2896E091BA
:106CAA00240EE87029F0E7E0F4E060E070E004C048
:106CBA00EBE0F4E060E070E00E9405DD80E00E9415
:106CCA00FFDA249619C0E2E1F4E060E070E00E9485
:106CDA0005DDA2E2B1E00E9447DDFF27662777279C
:106CEA000E9405DDE1E0F0E060E070E00E9405DD71
:106CFA0088E00E94FFDA2C9619C0E7E2F4E060E02F
:106D0A0070E00E9405DDA8E0B0E00E9447DDFF27A1
:106D1A00662777270E9405DDE3E0F0E060E070E097
:106D2A000E9405DD88E00E94FFDA2C96ECE3F4E08D
:106D3A0060E070E00E9405DDAFEFBFE00E9447DD32
:106D4A00FF27662777270E9405DDADEFBFE00E9487
:106D5A0047DDFF27662777270E9405DDAEEFBFE0F4
:106D6A000E9447DDFF27662777270E9405DD8CE012
:106D7A000E94FFDA6096E1E5F4E060E070E00E94CC
:106D8A0005DDE091250EFF27662777270E9405DD9E
:106D9A00E091260EFF27662777270E9405DD88E007
:106DAA000E94FFDA2C960895ABE0B0E00E9447DD1E
:106DBA00E093220EACE0B0E00E9447DDE093230EA0
:106DCA0099D90E94C29E7894A1E00E94AE3A0E948C
:106DDA001E2AA8953BDDECDAE091240EE07121F041
:106DEA00E091240EE87009F405C0E091240EE160F8
:106DFA00E093240EC8D9A091F010B091F1108091BF
:106E0A00F2109091F310AA3AE5E5BE07E0E08E078A
:106E1A00EFEF9E0719F4E4B7E0FF1AC0EAEAF5E5D6
:106E2A0060E07FEFE093F010F093F1106093F210BE
:106E3A007093F310E0E0F0E060E070E8E093F410A3
:106E4A00F093F5106093F6107093F710E093F81032
:106E5A00A2E3B1E00E9443DDFF70E093180EF093C5
:106E6A00190EA091180EB091190E1A9730F4EAE093
:106E7A00F0E0E093180EF093190EE4B7E3FF04C0B4
:106E8A00A091F810A03009F002C0A4E006C0E4B74F
:106E9A00E2FF02C0A5E001C0A2E00E94E82AE0E009
:106EAA00E4BFE093F810E4E6F4E060E070E00E94EA
:106EBA0005DD80E00E94FFDA2496F09A0DD2E09177
:106ECA001409E87FE260E0931409E0916304EF7C1F
:106EDA00E062E0936304E2E0E093690DE0E0E093AE
:106EEA001C0EA2E3B1E00E9443DDFF70339770F4F9
:106EFA00A2E3B1E0E3E0F0E0FF700F010E9443DD9E
:106F0A00E070F07FE029F1290E945BDDE091250E17
:106F1A00E03049F0EAE0EA93E0E0EA93A091250E36
:106F2A00BB270E94F12AE091260EE03049F0EBE0FF
:106F3A00EA93E0E0EA93A091260EBB270E94F12A89
:106F4A00A091770AA03071F4A091620BE091630BD3
:106F5A00EA1741F4A0917A00A03021F4A0911C0E06
:106F6A00A03009F005C0E1E0E3BF8895E0E0E3BFA7
:106F7A00A091280EA13060F0E091280EE150E09334
:106F8A00280EEF5FE091240EE07211F40E942A0CA1
:106F9A000E940606A0913608A43028F00E943C40C0
:106FAA00E0E0E0933608A0911C0EA13008F439C144
:106FBA00E0911C0EE150E0931C0EEF5FE5E0E093D8
:106FCA00280EA0E0F799A1E0E1E0EA2711F4F7988A
:106FDA0001C0F79AF79BE6C00E94ADCE0E94BDD2CF
:106FEA00E091240EE072D9F4E091AB07F0E0E130D1
:106FFA00A0E0FA0719F40E94F94A11C0E230A0E0B1
:10700A00FA0721F0E330A0E0FA0719F40E948A5740
:10701A0006C0E430A0E0FA0711F40E94FB5DA1E08B
:10702A000E942D2EA0E020FCA1E0E1E0EA27E894EE
:10703A00EE2309F0689420F820FE0FC00E9480CA4F
:10704A000E946626E0910A0EE07439F0E0910A0E79
:10705A00EF7BE0930A0E0E94E392A0914A0EA430BD
:10706A0030F4E0914A0EEF5FE0934A0E92C0E0E0FE
:10707A00E0934A0EA0E021FCA1E0E1E0EA27E894CF
:10708A00EE2309F0689421F821FE83C0A895A09107
:10709A00210EAF3F30F4E091210EEF5FE093210E15
:1070AA00E150A091270EA13060F0E091270EE15047
:1070BA00E093270EEF5FE091270EE03011F4A0E095
:1070CA0034DBA091170EA13030F0E091170EE15099
:1070DA00E093170E17C0E4E0E093170EABE0B9E0B7
:1070EA000A2EEC91E295E170A1E0EA27A02DE17069
:1070FA00E295E07F0E2EEC91EF7EE029EC93E0E042
:10710A00E0930609A0913508A03131F4DED00E943F
:10711A00E3920E94A67511C0E0913308EF70E13046
:10712A0060F0A3E3B8E080E0EFE00E9439DDE0918F
:10713A003308E061E093330801C0CED00E94B9CD94
:10714A000E9429450E94C0230E94E9D3A0E00E9420
:10715A002D2E0E94DE150E948228E091AB07F0E0F6
:10716A00E130A0E0FA0711F40E94FD510E94CD9E81
:10717A000E94680BA0914B0EA93030F4E0914B0E9F
:10718A00EF5FE0934B0E05C0E0E0E0934B0E0E94E8
:10719A0033CEE0910A0EEF7BE0930A0E0E94C8718B
:1071AA000E94173CE0911D0EF0911E0E7096E0931E
:1071BA001D0EF0931E0EA0911D0EB0911E0EA5334A
:1071CA00ECE0BE07E0F0E0911D0EF0911E0EE553D3
:1071DA00FC40E0931D0EF0931E0EA4EFB0E1ED917A
:1071EA00FD916D917D91EF5FFF4F6F4F7F4F7E93C2
:1071FA006E93FE93EE930E9407890E942484E09185
:10720A003308E07121F0A0913508A03109F009C0D6
:10721A00E0913308EF7EE093330857D00E94A675B9
:10722A005BD00E942B9F8CCEFFCFEA93EFB7EA93F5
:10723A00E1E0E0931B0EE0911C0EEF5FE0931C0E61
:10724A00E150E991EFBFE99118950E947ADB10E0CD
:10725A001731B8F5A2E3B0E0E12FF0E0BD01AAE0F2
:10726A00B0E00E942DDCDB01AE0FBF1F0E9443DDA0
:10727A000E9406DC9F012030E1E03E0788F0ECE640
:10728A00F4E060E070E00E9405DDF90166277727E7
:10729A000E9405DD84E00E94FFDA28962FEF30E095
:1072AA00A5ECB8E0E12FFF2766277727EC5FFE4FB2
:1072BA006F4F6BBFE691F0E0EA0FFB1F20831F5F61
:1072CA00C7CF0E9481DB24960895E6E8E0937A000E
:1072DA00E0E0E09332080895E6E8E0937A00E0E01F
:1072EA00E8B9E0937C00E0933408E0933508E1E0E4
:1072FA00E0933208E1E4F8E0FA93EA93E0E0EA93F3
:10730A00A0E4B0E00E9477D4E5E8F8E0FA93EA93C3
:10731A00E0E0EA93A0E2B0E00E9477D4E5EAF8E080
:10732A00FA93EA93E0E0EA93A0E2B0E00E9477D40D
:10733A00E5EEF8E0FA93EA93E0E0EA93A0E2B0E03F
:10734A000E9477D4EEECE0937A00E0913308E07F74
:10735A00E560E093330808950A921A928A93AA93F1
:10736A00BA93EA93FA93EFB7EA93E0913208F0E01E
:10737A00E130A0E0FA0739F4EFECE0937A00E2E0BA
:10738A00E0933208DCC0E230A0E0FA0709F0D7C087
:10739A0046B0E0913408EF5FE0933408E150E091A1
:1073AA003408EF71E0933408E8B9A0913408A931A0
:1073BA00D0F4EEECE0937A00A091220EA33460F0B0
:1073CA00A0913408A83010F0A83110F0E0E001C014
:1073DA00E3E0E0937C0003C0E0E0E0937C00E1E0BE
:1073EA00E09332081CC0A0913408AE3139F4E1E0D0
:1073FA00E0937C0080E58A95F1F70EC0A0913408ED
:10740A00AF3139F4E2E0E0937C0080E58A95F1F748
:10741A0003C0E0E0E0937C00EFECE0937A00E091B7
:10742A003408E770E0934C0EA7E3B8E0F0E0EA0F07
:10743A00FB1F4082E0914C0EE03031F4E0913608B7
:10744A00EF5FE0933608E150A5E8B8E0E091340830
:10745A00F0E0AE0FBF1FEC91E429EC93A5EAB8E087
:10746A00E0913408F0E0EA0FFB1F0F01A081E42D40
:10747A00E095EA2BD001EC93A0913508A03108F0F1
:10748A005EC0A5ECB8E0E0913408F0E0AE0FBF1F93
:10749A00EC91E0934C0EE0917800F0917900A09184
:1074AA004C0EB0E0AE17BF0798F4A1E4B8E0E09143
:1074BA003408F0E0EE0FFF1FEA0FFB1F0F01DF0198
:1074CA00ED91FD91DF01E0917800F091790011C012
:1074DA00A1E4B8E0E0913408F0E0EE0FFF1FEA0FF4
:1074EA00FB1F0F01DF01ED91FD91DF01E0914C0ED1
:1074FA00F0E0EA0FFB1FD001ED93FC93A091340852
:10750A00AA3140F4A0917800B0917900A03FE3E05D
:10751A00BE0708F40AC0A5EEB8E0E0913408F0E02E
:10752A00AE0FBF1FEC91EF5FEC93E0913408E030AF
:10753A0031F4E0913508EF5FE0933508E150E991C5
:10754A00EFBFF991E991B991A9918991199009909F
:10755A0018951A931A2F103041F05C988BE08A958F
:10756A00F1F75C9A8BE08A95F1F72898EDB5E093EC
:10757A00160EE0E4EEBDEDB5E7FFFDCFE5E0EEBDAA
:10758A00EDB5E7FFFDCFE8E0EEBDEDB5E7FFFDCFD6
:10759A00289AE0910B09ED7FE0930B09A6ECB2E083
:1075AA000E9447DDE170ABE0B9E0E1700E2EEC918C
:1075BA00EE7FE029EC93EBE0F9E0DF01F49B02C0F7
:1075CA00F59B01C002C0E1E001C0E0E0E170E7958F
:1075DA00E0E0E7950E2EEC91EF77E029EC932898FE
:1075EA00EDB5E093160EE0E4EEBDEDB5E7FFFDCF95
:1075FA00EAE0EEBDEDB5E7FFFDCFE0910B09EEBD88
:10760A00EDB5E7FFFDCF289AA091220EA334A0F092
:10761A002898EDB5E093160EE0E4EEBDEDB5E7FF70
:10762A00FDCFE6E0EEBDEDB5E7FFFDCFECE0EEBD48
:10763A00EDB5E7FFFDCF13C02898EDB5E093160E20
:10764A00E0E4EEBDEDB5E7FFFDCFE6E0EEBDEDB55A
:10765A00E7FFFDCFE4E0EEBDEDB5E7FFFDCF289AE9
:10766A002898EDB5E093160EE0E4EEBDEDB5E7FF20
:10767A00FDCFE0E0EEBDEDB5E7FFFDCFECE0EEBDFE
:10768A00EDB5E7FFFDCF289A2898EDB5E093160EE1
:10769A00E2E4EEBDEDB5E7FFFDCFEAE0EEBDEDB504
:1076AA00E7FFFDCFE0E0EEBDEDB5E7FFFDCF289A9D
:1076BA002898EDB5E093160EE2E4EEBDEDB5E7FFCE
:1076CA00FDCFE0E0EEBDEDB5E7FFFDCFE0E0EEBDBA
:1076DA00EDB5E7FFFDCF289A2898EDB5E093160E91
:1076EA00E4E4EEBDEDB5E7FFFDCFEAE0EEBDEDB5B2
:1076FA00E7FFFDCFE0E0EEBDEDB5E7FFFDCF289A4D
:10770A002898EDB5E093160EE4E4EEBDEDB5E7FF7B
:10771A00FDCFE0E0EEBDEDB5E7FFFDCFE0E0EEBD69
:10772A00EDB5E7FFFDCF289AE0911009E062E093FA
:10773A001009A298EDB5E093160EE0E4EEBDEDB5A2
:10774A00E7FFFDCFE5E0EEBDEDB5E7FFFDCFE8E0F1
:10775A00EEBDEDB5E7FFFDCFA29AA298EDB5E09395
:10776A00160EE0E4EEBDEDB5E7FFFDCFEAE0EEBDB3
:10777A00EDB5E7FFFDCFE0911009EEBDEDB5E7FFEE
:10778A00FDCFA29AA298EDB5E093160EE0E4EEBD05
:10779A00EDB5E7FFFDCFE0E0EEBDEDB5E7FFFDCFCC
:1077AA00EFE1EEBDEDB5E7FFFDCFA29AE2E1F9E028
:1077BA00DF01F29B02C0F39B01C002C0E1E001C0FD
:1077CA00E0E0E170EE0F0E2EEC91ED7FE029EC93F4
:1077DA00A298EDB5E093160EE2E4EEBDEDB5E7FF33
:1077EA00FDCFEAE0EEBDEDB5E7FFFDCFE09112096E
:1077FA00EEBDEDB5E7FFFDCFA29AA298EDB5E093F5
:10780A00160EE2E4EEBDEDB5E7FFFDCFE0E0EEBD1A
:10781A00EDB5E7FFFDCFECEFEEBDEDB5E7FFFDCF30
:10782A00A29AC7C1A0910609A13030F0E0910609D9
:10783A00E150E093060918C0E3E6E09306092898A8
:10784A00EDB5E093160EE0E4EEBDEDB5E7FFFDCF32
:10785A00EAE0EEBDEDB5E7FFFDCFE0910B09EEBD25
:10786A00EDB5E7FFFDCF289AA0910709A13038F0BE
:10787A00E0910709E150E0930709EF5F18C0E3E6DA
:10788A00E09307092898EDB5E093160EE2E4EEBD01
:10789A00EDB5E7FFFDCFEAE0EEBDEDB5E7FFFDCFC1
:1078AA00E0910D09EEBDEDB5E7FFFDCF289AA09155
:1078BA000809A13038F0E0910809E150E09308097D
:1078CA00EF5F18C0E3E6E09308092898EDB5E09366
:1078DA00160EE4E4EEBDEDB5E7FFFDCFEAE0EEBD3E
:1078EA00EDB5E7FFFDCFE0910E09EEBDEDB5E7FF7F
:1078FA00FDCF289AA0910909A13038F0E091090931
:10790A00E150E0930909EF5F2DC0E3E6E09309092E
:10791A00A298EDB5E093160EE0E4EEBDEDB5E7FFF3
:10792A00FDCFEAE0EEBDEDB5E7FFFDCFE09110092E
:10793A00EEBDEDB5E7FFFDCFA29AA298EDB5E093B3
:10794A00160EE0E4EEBDEDB5E7FFFDCFE0E0EEBDDB
:10795A00EDB5E7FFFDCFE0910F09EEBDEDB5E7FF0D
:10796A00FDCFA29AA0910A09A13038F0E0910A0944
:10797A00E150E0930A09EF5F2DC0E3E6E0930A09BC
:10798A00A298EDB5E093160EE2E4EEBDEDB5E7FF81
:10799A00FDCFEAE0EEBDEDB5E7FFFDCFE0911209BC
:1079AA00EEBDEDB5E7FFFDCFA29AA298EDB5E09343
:1079BA00160EE2E4EEBDEDB5E7FFFDCFE0E0EEBD69
:1079CA00EDB5E7FFFDCFE0911109EEBDEDB5E7FF9B
:1079DA00FDCFA29A08951A93F298F398F498F5981D
:1079EA00E0917E00E97FE0937E00E3E9F7E0FA9315
:1079FA00EA93E0E0EA93ACE0B0E00E9477D410E0CA
:107A0A001C3008F04EC0E12FF0E0ED56F84F0F01A0
:107A1A00ABE0B2E0EE27A10FBE1F0E9447DDE37084
:107A2A00D001E370EE0FEE0F0E2EEC91E37FE0290A
:107A3A00EC93E12FF0E0ED56F84F0F01ABE0B2E026
:107A4A00EE27A10FBE1F0E9447DDE695E695E1707D
:107A5A00D001E170EE0F0E2EEC91ED7FE029EC9350
:107A6A00E12FF0E0ED56F84FE081F0E00E9408DCEB
:107A7A00E370F070309741F4123011F0133011F4C2
:107A8A00F49A01C0F29A0BC0E130A0E0FA0739F487
:107A9A00123011F0133011F4F59A01C0F39A1F5FF6
:107AAA00AFCFE0919507EC70E83031F0AFE1B2E08A
:107ABA000E9447DDE37051F0E0917E00E260E093BE
:107ACA007E00E1E0E0933F08F59AF498E09196078A
:107ADA00EC70E83031F0AFE1B2E00E9447DDEC70C3
:107AEA0051F0E0917E00E460E0937E00E1E0E093F3
:107AFA004008F59AF498E2E1F9E0DF01F29B02C04E
:107B0A00F39B01C002C0E1E001C0E0E0E170EE0FCA
:107B1A000E2EEC91ED7FE029EC93E0E0E0930A0968
:107B2A00EBE0F9E0DF01F49B02C0F59B01C002C063
:107B3A00E1E001C0E0E0E170E795E0E0E7950E2EB4
:107B4A00EC91EF77E029EC93E0E0E093060931C08D
:107B5A001A93E4E8F4E060E070E00E9405DD80E05A
:107B6A000E94FFDA249610E01C3000F5ECE8F4E0FD
:107B7A0060E070E00E9405DDE12FF0E031966F2FA2
:107B8A00660F660B762F0E9405DDE12FF0E0ED56B9
:107B9A00F84FE081E170FF27662777270E9405DD0D
:107BAA0088E00E94FFDA2C961F5FDECFAAE00E94CF
:107BBA00089F199108950E947ADB3A2FE091240ECA
:107BCA00E17009F44FC2373310F03C3308F006C0B5
:107BDA00E32FF0E0F797E55EF54F3081313059F445
:107BEA00A0912C0EB0912D0EA037E7E1BE0710F040
:107BFA00E1E039C237C2333010F03F3008F008C034
:107C0A00E32FF0E03397ED56F84FE081E1702BC295
:107C1A003F3010F0363308F03CC03632E8F4E32F38
:107C2A00F0E03F97A9E0B0E00E942DDCE45EF64F59
:107C3A00E081E17079F0E32FF0E03F97A9E0B0E04E
:107C4A000E942DDCE45EF64FE081E077E03410F428
:107C5A00E1E001C0E0E007C2E32FF0E0B697A3E05D
:107C6A00B0E00E942DDCE551F64FE081E17079F039
:107C7A00E32FF0E0B697A3E0B0E00E942DDCE551D7
:107C8A00F64FE081E077E03410F4E1E001C0E0E093
:107C9A00EAC13C3310F0303708F014C0ABE6B4E068
:107CAA00E32FF0E0FC97BD01AEE0B0E00E942DDCCE
:107CBA00DB01AE0FBF1F1C96EC91EE1FE0E0EE1F3A
:107CCA00E170D1C1303710F0343808F011C0AAE69B
:107CDA00BDE0E32FF0E0E057F0400E94F4DBAE0F86
:107CEA00BF1FEC91E295EF70E695E695E170BBC196
:107CFA00343810F0383908F00EC0E32FF0E0E458B9
:107D0A00F040A3E0B0E00E942DDCED5BF84FE0818B
:107D1A00E695E170A8C1383910F03D3908F00EC077
:107D2A00E32FF0E0E859F040AFE7B7E00E94F6DB56
:107D3A00AE0FBF1F1396EC91E17095C13D39B9F4AE
:107D4A00E0910A0EEF70E33079F0E0910A0EEF70DD
:107D5A00E43051F0E0910A0EEF70E13029F0E09141
:107D6A000A0EEF70E63011F4E1E07DC17BC13E39C5
:107D7A0069F4E0910A0EEF70E53029F0E0910A0EFD
:107D8A00EF70E23011F4E1E06EC16CC13F3910F0DE
:107D9A00373B08F06FC0E32FEF591E2FFF276627E6
:107DAA007727E658FE4F6F4F6BBF0691E12FFF27EB
:107DBA0066277727EE56FE4F6F4F6BBF1691113429
:107DCA0049F5A3E00A9FF001E05AF54FE081E07F10
:107DDA00E03111F4E1E047C1A3E00A9FF001E05A63
:107DEA00F54FE081E07FE03288F00A9FF001E05A27
:107DFA00F54FE081E770E33041F00A9FF001E05A65
:107E0A00F54FE081E770E43009F401C002C0E1E017
:107E1A002AC12FC0123401F5A3E00A9FF001E05AEB
:107E2A00F54FE081E07FE03211F4E1E01CC1A3E00C
:107E3A000A9FF001E05AF54FE081E07FE03340F01D
:107E4A000A9FF001E05AF54FE081E770E43009F04B
:107E5A0002C0E1E008C10DC0133459F4A3E00A9F3F
:107E6A00F001E05AF54FE081E07FE03311F4E1E000
:107E7A00FAC0F8C03A3B10F0363C08F009C0E32FCC
:107E8A00EA5B0E2FF0E0E156F84FE081E170EBC0BB
:107E9A00373C10F03F3D08F0BEC0E091AB07F0E080
:107EAA00E130A0E0FA0709F04CC03F3C88F4E32F28
:107EBA00E75C1E2FA1E0B0E00E94A2DBA091B5070B
:107ECA00B0E0EA23FB23309711F0E1E0CCC038C0E0
:107EDA00333D88F4E32FEF5C1E2FA1E0B0E00E944F
:107EEA00A2DBA091B607B0E0EA23FB23309711F09A
:107EFA00E1E0B9C025C03B3D88F4E32FE35D1E2FC6
:107F0A00A1E0B0E00E94A2DBA091CE07B0E0EA2394
:107F1A00FB23309711F0E1E0A6C012C03F3D80F488
:107F2A00E32FEB5D1E2FA1E0B0E00E94A2DBA0913F
:107F3A00CF07B0E0EA23FB23309711F0E1E093C0CA
:107F4A0069C0E230A0E0FA0721F0E330A0E0FA07C6
:107F5A0089F4A2EDB7E0E32FF0E0E75CF0400E947D
:107F6A00F6DBAE0FBF1F1296EC91E17011F0E1E063
:107F7A007AC050C0E430A0E0FA0709F04BC03F3C99
:107F8A0088F4E32FE75C1E2FA1E0B0E00E94A2DB99
:107F9A00A091B307B0E0EA23FB23309711F0E1E0A8
:107FAA0062C038C0333D88F4E32FEF5C1E2FA1E096
:107FBA00B0E00E94A2DBA091B607B0E0EA23FB235F
:107FCA00309711F0E1E04FC025C03B3D88F4E32F24
:107FDA00E35D1E2FA1E0B0E00E94A2DBA091DB07C7
:107FEA00B0E0EA23FB23309711F0E1E03CC012C075
:107FFA003F3D80F4E32FEB5D1E2FA1E0B0E00E942D
:10800A00A2DBA091DE07B0E0EA23FB23309711F050
:10801A00E1E029C027C03F3D39F4E0912F0EE0721C
:10802A0011F0E1E020C01EC0303E39F4E0912F0E7D
:10803A00E07411F0E1E017C015C0323059F4A5E33D
:10804A00B1E00E9447DDA091210EAE1710F0E1E0E9
:10805A000AC008C0313E31F4E0916404E87011F0BE
:10806A00E1E001C0E0E00E9481DB249608952397B5
:10807A000E9478DBF39904C0F59902C022FE01C080
:10808A0003C0689422F8DCC4F09B10C0E091930707
:10809A00E1704E2FE0919407E170E887E09195072F
:1080AA00E170EF83E0919607E170EE8322FE48C00B
:1080BA00E0919307EC7009F042C0E0919307E295D2
:1080CA00EF701E2F489B02C0F19B01C01FC01230E7
:1080DA0010F41F5F1AC01230B9F4E0919307E270EE
:1080EA0071F0E0919307E17021F0E0919307EE7F40
:1080FA0003C0E0919307E160E093930705C0E09124
:10810A009307E160E09393071FE00EC01B3010F065
:10811A0011500AC0E0919307E27029F4E0919307A5
:10812A00EE7FE093930710E0E12FEF70E295E07F96
:10813A000E2EE0919307EF70E029E093930745C074
:10814A00E0919307EC70E43009F03FC0E0919307A7
:10815A00E295EF701E2F489B0FC01B3010F0115094
:10816A000AC0E0919307E27029F4E0919307EE7F49
:10817A00E093930710E01EC0123010F41F5F1AC07C
:10818A001230B9F4E0919307E27071F0E09193072D
:10819A00E17021F0E0919307EE7F03C0E09193072D
:1081AA00E160E093930705C0E0919307E160E093F3
:1081BA0093071FE0E12FEF70E295E07F0E2EE0912A
:1081CA009307EF70E029E093930722FE4AC0E091FB
:1081DA009407EC7009F044C0E0919407E295EF70BF
:1081EA001E2F499B02C0F19B01C021C0123010F41E
:1081FA001F5F1CC01230C9F4E0919407E27081F04D
:10820A00E0919407E17031F0A4E9B7E0EC91EE7FD8
:10821A00EC9305C0E0919407E160E093940705C0F0
:10822A00E0919407E160E09394071FE00EC01B30D1
:10823A0010F011500AC0E0919407E27029F4A4E901
:10824A00B7E0EC91EE7FEC9310E0A4E9B7E0E12F00
:10825A00EF70E295E07F0E2EEC91EF70E029EC933F
:10826A0047C0E0919407EC70E43009F041C0E09116
:10827A009407E295EF701E2F499B0FC01B3010F038
:10828A0011500AC0E0919407E27029F4A4E9B7E01A
:10829A00EC91EE7FEC9310E020C0123010F41F5FD7
:1082AA001CC01230C9F4E0919407E27081F0E091A9
:1082BA009407E17031F0A4E9B7E0EC91EE7FEC931A
:1082CA0005C0E0919407E160E093940705C0E0914E
:1082DA009407E160E09394071FE0A4E9B7E0E12F77
:1082EA00EF70E295E07F0E2EEC91EF70E029EC93AF
:1082FA00E0919507EC70E83009F03FC0E091810801
:10830A00F091820834960E9406DC5E2FE091950770
:10831A00E295EF701E2FA9E1B2E00E9447DD3E2FE1
:10832A00AAE1B2E00E9447DD2E2F321728F5E0912C
:10833A009507E17089F0351768F0143010F41F5F63
:10834A0008C0143031F4A5E9B7E0EC91EE7FEC9364
:10835A0010E001C010E010C0521768F0123010F49B
:10836A001F5F08C0123031F4E0919507E160E09395
:10837A00950710E001C010E085C022FE47C0E091D9
:10838A009507EC7009F041C0E0919507E295EF700E
:10839A001E2F799B0FC01B3010F011500AC0E091BC
:1083AA009507E27029F4A5E9B7E0EC91EE7FEC932A
:1083BA0010E020C0123010F41F5F1CC01230C9F444
:1083CA00E0919507E27081F0E0919507E17031F054
:1083DA00A5E9B7E0EC91EE7FEC9305C0E091950733
:1083EA00E160E093950705C0E0919507E160E093AD
:1083FA0095071FE0A5E9B7E0E12FEF70E295E07F6E
:10840A000E2EEC91EF70E029EC9347C0E0919507AE
:10841A00EC70E43009F041C0E0919507E295EF7005
:10842A001E2F799B21C0123010F41F5F1CC012301E
:10843A00C9F4E0919507E27081F0E0919507E17047
:10844A0031F0A5E9B7E0EC91EE7FEC9305C0E0913D
:10845A009507E160E093950705C0E0919507E16013
:10846A00E09395071FE00EC01B3010F011500AC0B0
:10847A00E0919507E27029F4A5E9B7E0EC91EE7F67
:10848A00EC9310E0A5E9B7E0E12FEF70E295E07F09
:10849A000E2EEC91EF70E029EC93E0919607EC70C8
:1084AA00E83009F03FC0E0918308F09184083496DF
:1084BA000E9406DC5E2FE0919607E295EF701E2F70
:1084CA00ADE1B2E00E9447DD3E2FAEE1B2E00E948C
:1084DA0047DD2E2F321728F5E0919607E17089F0D3
:1084EA00351768F0143010F41F5F08C0143031F4E7
:1084FA00A6E9B7E0EC91EE7FEC9310E001C010E042
:10850A0010C0521768F0123010F41F5F08C0123002
:10851A0031F4E0919607E160E093960710E001C01C
:10852A0010E085C022FE47C0E0919607EC7009F082
:10853A0041C0E0919607E295EF701E2F7A9B0FC01B
:10854A001B3010F011500AC0E0919607E27029F42E
:10855A00A6E9B7E0EC91EE7FEC9310E020C0123070
:10856A0010F41F5F1CC01230C9F4E0919607E27044
:10857A0081F0E0919607E17031F0A6E9B7E0EC915D
:10858A00EE7FEC9305C0E0919607E160E0939607D1
:10859A0005C0E0919607E160E09396071FE0A6E91F
:1085AA00B7E0E12FEF70E295E07F0E2EEC91EF70CD
:1085BA00E029EC9347C0E0919607EC70E43009F0AB
:1085CA0041C0E0919607E295EF701E2F7A9B21C079
:1085DA00123010F41F5F1CC01230C9F4E0919607E4
:1085EA00E27081F0E0919607E17031F0A6E9B7E018
:1085FA00EC91EE7FEC9305C0E0919607E160E09381
:10860A00960705C0E0919607E160E09396071FE0A0
:10861A000EC01B3010F011500AC0E0919607E270AC
:10862A0029F4A6E9B7E0EC91EE7FEC9310E0A6E915
:10863A00B7E0E12FEF70E295E07F0E2EEC91EF703C
:10864A00E029EC93F09B5FC0E0919307E170E41797
:10865A0091F0E3E9F4E060E070E00E9405DDE0916A
:10866A009307E170FF27662777270E9405DD84E0DC
:10867A000E94FFDA2896E0919407E170A885EA172C
:10868A0091F0EDE9F4E060E070E00E9405DDE09130
:10869A009407E170FF27662777270E9405DD84E0AB
:1086AA000E94FFDA2896E0919507E170AF81EA17F8
:1086BA0091F0E7EAF4E060E070E00E9405DDE09105
:1086CA009507E170FF27662777270E9405DD84E07A
:1086DA000E94FFDA2896E0919607E170AE81EA17C8
:1086EA0091F0E1EBF4E060E070E00E9405DDE091DA
:1086FA009607E170FF27662777270E9405DD84E049
:10870A000E94FFDA289654E05C3008F028C1E52F71
:10871A00F0E0ED56F84FE081E1704E2F22FE85C061
:10872A00E52FF0E0ED56F84FE081EC7009F07CC0DF
:10873A00A7E3B8E0E52FFF2766277727EC56FF4F18
:10874A006F4F6BBFE691F0E0AE0FBF1FEC91E07286
:10875A000E2FF19B02C000E011C0A7E3B8E0E52F9D
:10876A00FF2766277727EC56FF4F6F4F6BBFE691BF
:10877A00F0E0AE0FBF1FEC91E0720E2FE52FF0E094
:10878A00ED56F84FE081E295EF701E2F003061F14F
:10879A00123010F41F5F27C0123021F5E52FF0E0E8
:1087AA00ED56F84FE081E270B1F0E52FF0E0ED56BA
:1087BA00F84FE081E17039F0A52FB0E0AD56B84F1F
:1087CA00EC91EE7F06C0A52FB0E0AD56B84FEC9104
:1087DA00E160EC9307C0A52FB0E0AD56B84FEC911D
:1087EA00E160EC931FE013C01B3010F011500FC072
:1087FA00E52FF0E0ED56F84FE081E27039F4A52F4D
:10880A00B0E0AD56B84FEC91EE7FEC9310E0A52F97
:10881A00B0E0AD56B84FE12FEF70E295E07F0E2E33
:10882A00EC91EF70E029EC9370C0E52FF0E0ED5683
:10883A00F84FE081EC70E43009F067C0A7E3B8E0D4
:10884A00E52FFF2766277727EC56FF4F6F4F6BBF41
:10885A00E691F0E0AE0FBF1FEC91E0720E2FE52F0C
:10886A00F0E0ED56F84FE081E295EF701E2F0030F0
:10887A00A1F01B3010F011500FC0E52FF0E0ED56BB
:10888A00F84FE081E27039F4A52FB0E0AD56B84F49
:10889A00EC91EE7FEC9310E02BC0123010F41F5FC6
:1088AA0027C0123021F5E52FF0E0ED56F84FE081B0
:1088BA00E270B1F0E52FF0E0ED56F84FE081E1709B
:1088CA0039F0A52FB0E0AD56B84FEC91EE7F06C057
:1088DA00A52FB0E0AD56B84FEC91E160EC9307C01C
:1088EA00A52FB0E0AD56B84FEC91E160EC931FE0D4
:1088FA00A52FB0E0AD56B84FE12FEF70E295E07FBB
:10890A000E2EEC91EF70E029EC93F09B26C0E52F38
:10891A00F0E0ED56F84FE081E170E417F1F0EBEB8F
:10892A00F4E060E070E00E9405DDE52FF0E03196AA
:10893A006F2F660F660B762F0E9405DDE52FF0E09C
:10894A00ED56F84FE081E170FF27662777270E94EE
:10895A0005DD88E00E94FFDA2C965F5FD5CEF39B97
:10896A0006C0F29904C0F59B02C0F49B01C002C084
:10897A00E89414C0F39906C0F29B04C0F59902C0AA
:10898A00F49901C002C0689409C0A0E022FCA1E0E9
:10899A00E1E0EA27E894EE2309F0689422F8F39BD1
:1089AA0002C0F29901C021C0A2E1B9E0E0E022FCD4
:1089BA00E1E0E170EE0F0E2EEC91ED7FE029EC93F1
:1089CA00A298EDB5E093160EE2E4EEBDEDB5E7FF31
:1089DA00FDCFEAE0EEBDEDB5E7FFFDCFE09112096C
:1089EA00EEBDEDB5E7FFFDCFA29AF59B02C0F49963
:1089FA0001C026C0E3E6E0930609ABE0B9E0E0E097
:108A0A0022FCE1E0E170E795E0E0E7950E2EEC91BB
:108A1A00EF77E029EC932898EDB5E093160EE0E4A1
:108A2A00EEBDEDB5E7FFFDCFEAE0EEBDEDB5E7FF40
:108A3A00FDCFE0910B09EEBDEDB5E7FFFDCF289A1A
:108A4A000E947FDB2996089524970E9478DBAFE184
:108A5A00B2E00E9447DDE3703E2F303009F4B9C01E
:108A6A00A0E2B2E00E9447DD2E2FA1E2B2E00E940E
:108A7A0047DD5E2F313029F4E0918108F0918208B8
:108A8A0004C0E0918308F091840834960E9408DCBF
:108A9A00E887F98710E0163008F09BC0A2E2B2E03E
:108AAA00EE27A10FBE1F0E9447DD0E2F013008F4EA
:108ABA008EC0F0E0EE83FF83EE0FFF1FEE83FF838D
:108ACA00E12FF0E0E156F84FE081E17009F443C08C
:108ADA00E22FF0E0A885B985AE0FBF1FEE27A50FDC
:108AEA00BE1FEE81FF81AE17BF0778F0E22FF0E0DC
:108AFA00AE81BF81AE0FBF1FE52FF0E0EA0FFB1F6B
:108B0A00A885B985EA17FB0728F5F09B1CC0E6EC97
:108B1A00F4E060E070E00E9405DDE12FF0E03196BC
:108B2A006F2F660F660B762F0E9405DDA889B9891B
:108B3A00EAE00E9455DC662777270E9405DD88E077
:108B4A000E94FFDA2C96A12FB0E0A156B84FEC9103
:108B5A00EE7FEC933CC0E22FF0E0A885B985AE0F1A
:108B6A00BF1FEE81FF81AE17BF0758F0E22FF0E07A
:108B7A00AE81BF81EA0FFB1FA885B985EA17FB07FB
:108B8A0008F425C0F09B1CC0EAEDF4E060E070E058
:108B9A000E9405DDE12FF0E031966F2F660F660B1C
:108BAA00762F0E9405DDA889B989EAE00E9455DC82
:108BBA00662777270E9405DD88E00E94FFDA2C9657
:108BCA00A12FB0E0A156B84FEC91E160EC931F5F82
:108BDA0062CFAFE1B2E00E9447DDE695E695E37029
:108BEA003E2F303009F4B9C0A0E2B2E00E9447DD5E
:108BFA002E2FA1E2B2E00E9447DD5E2F313029F428
:108C0A00E0918108F091820804C0E0918308F09114
:108C1A00840834960E9408DCE887F98716E01C303D
:108C2A0008F09BC0A2E2B2E0EE27A10FBE1F0E948D
:108C3A0047DD0E2F013008F48EC0F0E0EE83FF838B
:108C4A00EE0FFF1FEE83FF83E12FF0E0E156F84FAE
:108C5A00E081E17009F443C0E22FF0E0A885B9850C
:108C6A00AE0FBF1FEE27A50FBE1FEE81FF81AE1705
:108C7A00BF0778F0E22FF0E0AE81BF81AE0FBF1FD1
:108C8A00E52FF0E0EA0FFB1FA885B985EA17FB0775
:108C9A0028F5F09B1CC0E6ECF4E060E070E00E946E
:108CAA0005DDE12FF0E031966F2F660F660B762F08
:108CBA000E9405DDA889B989EAE00E9455DC662789
:108CCA0077270E9405DD88E00E94FFDA2C96A12F03
:108CDA00B0E0A156B84FEC91EE7FEC933CC0E22F86
:108CEA00F0E0A885B985AE0FBF1FEE81FF81AE17F0
:108CFA00BF0758F0E22FF0E0AE81BF81EA0FFB1FF9
:108D0A00A885B985EA17FB0708F425C0F09B1CC0A3
:108D1A00EAEDF4E060E070E00E9405DDE12FF0E0AA
:108D2A0031966F2F660F660B762F0E9405DDA88994
:108D3A00B989EAE00E9455DC662777270E9405DD9B
:108D4A0088E00E94FFDA2C96A12FB0E0A156B84F16
:108D5A00EC91E160EC931F5F62CF0E947FDB2A9661
:108D6A00089560971A93FE013196FA93EA93E0E028
:108D7A00EA93A0E1B0E00E9477D410E01C3008F03A
:108D8A003FC0ABE0B2E0EE27A10FBE1F0E9447DD55
:108D9A00EC7F0E9463DDABE0B2E0EE27A10FBE1FBD
:108DAA000E9447DDEB7F0E9463DDFE013196FA9354
:108DBA00EA93EDEEF4E060E070E00E9405DDE12F59
:108DCA00F0E031966F2F660F660B762F0E9405DD55
:108DDA0084E00E94C4DA2A96E12FF0E0A0EDBAE31B
:108DEA000E94F2DBEA0FFB1FFA93EA93FE01339625
:108DFA00FA93EA93A0E10E94502CA8951F5FBECF78
:108E0A00A7E1B2E0E0E00E9463DDA8E1B2E0EAEFA8
:108E1A000E9463DDA9E1B2E0E4E60E9463DDAAE113
:108E2A00B2E0E6E90E9463DDABE1B2E0E0E00E9475
:108E3A0063DDACE1B2E0EAEF0E9463DDADE1B2E0EE
:108E4A00E4E60E9463DDAEE1B2E0E6E90E9463DD9A
:108E5A00AFE1B2E00E9447DDEC7F0E9463DDAFE143
:108E6A00B2E00E9447DDE37F0E9463DDAFE1B2E03A
:108E7A000E9447DDEF700E9463DDA0E2B2E0E8E104
:108E8A000E9463DDA1E2B2E0E2E00E9463DDE2E279
:108E9A00F2E0FA93EA93ACE00E94BA2910E01630A5
:108EAA0008F054C0FE013196FA93EA93E7EFF4E032
:108EBA0060E070E00E9405DDE12FF0E031966F2F4F
:108ECA00660F660B762F0E9405DD84E00E94C4DAE5
:108EDA002A96E12FF0E0A0E4B5E40E94F2DBEA0F63
:108EEA00FB1FFA93EA93FE013396FA93EA93A0E101
:108EFA000E94502CFE013196FA93EA93E3E0F5E0E2
:108F0A0060E070E00E9405DDE12FF0E031966F2FFE
:108F1A00660F660B762F0E9405DD84E00E94C4DA94
:108F2A002A96E12FF0E03696A0E4B5E40E94F2DB3F
:108F3A00EA0FFB1FFA93EA93FE013396FA93EA9338
:108F4A00A0E10E94502CA8951F5FA9CF18816196B5
:108F5A0008950E9478DBEBEAF7E0FA93EA93E0E0FF
:108F6A00EA93A7E8B0E00E9477D4A8E3B1E00E94B0
:108F7A0047DDE093AB07E0E1F5E060E070E00E94D6
:108F8A0005DD80E00E94FFDA2496E091AB07F0E06D
:108F9A00E130A0E0FA0709F028C100E0023008F049
:108FAA0007C1AAE7B8E0E02FF0E0BD01A1E7B0E011
:108FBA000E942DDCDB01AE0FBF1F0E9447DDE030AF
:108FCA0009F4F4C0ACEAB7E0E02FF0E0BD01A9E192
:108FDA00B0E00E942DDCE60FF71FFF93EF93AAE79C
:108FEA00B8E0E02FF0E0BD01A1E7B0E00E942DDC7F
:108FFA00DB01AE0FBF1F11960E9447DDE295EF70AD
:10900A00AF91BF91EF770E2EEC91E078E029EC93C7
:10901A00ACEAB7E0E02FF0E0BD01A9E1B0E00E94C0
:10902A002DDCDB01AE0FBF1F1296E5E0EC9331E0B9
:10903A00E0E01E2F5E2F2E2F183008F040C0AAE75E
:10904A00B8E0E02FF0E0BD01A1E7B0E00E942DDC1E
:10905A00DB01AE0FBF1F1E96E12FF0E00E94F4DB8A
:10906A00AE0FBF1F16960E9447DDF0E0F695E79512
:10907A00E370F070E130A0E0FA0721F0E330A0E0FD
:10908A00FA0709F4232BAAE7B8E0E02FF0E0BD01C4
:10909A00A1E7B0E00E942DDCDB01AE0FBF1F1E96D8
:1090AA00E12FF0E00E94F4DBAE0FBF1F16960E947C
:1090BA0047DDE17009F0532B1F5F330FBDCFACEAD8
:1090CA00B7E0E02FF0E0BD01A9E1B0E00E942DDC9D
:1090DA00E60FF71F2187ACEAB7E0E02FF0E0BD0109
:1090EA00A9E1B0E00E942DDCE60FF71F558331E0BD
:1090FA00E0E05E2F2E2F1C3008F040C0AAE7B8E04F
:10910A00E02FF0E0BD01A1E7B0E00E942DDCDB0119
:10911A00AE0FBF1F1E96E12FF0E00E94F4DBAE0FE8
:10912A00BF1F16960E9447DDF0E0F695E795E370BB
:10913A00F070E130A0E0FA0721F0E330A0E0FA078E
:10914A0009F4232BAAE7B8E0E02FF0E0BD01A1E77C
:10915A00B0E00E942DDCDB01AE0FBF1F1E96E12F8F
:10916A00F0E00E94F4DBAE0FBF1F16960E9447DDA7
:10917A00E17009F0532B1F5F330FBDCFACEAB7E0A4
:10918A00E02FF0E0BD01A9E1B0E00E942DDCE60F7E
:10919A00F71F2287ACEAB7E0E02FF0E0BD01A9E1B2
:1091AA00B0E00E942DDCE60FF71F56830F5FF6CE64
:1091BA00E8E1F5E060E070E00E9405DDAAE7B8E0CA
:1091CA000E9447DDFF27662777270E9405DDABEE61
:1091DA00B8E00E9447DDFF27662777270E9405DD52
:1091EA0088E00E94FFDA2C963DC0E230A0E0FA0740
:1091FA0069F4E9E2F5E060E070E00E9405DD80E0F4
:10920A000E94FFDA24960E94B1532CC0E330A0E0FA
:10921A00FA0769F4EBE3F5E060E070E00E9405DD2F
:10922A0080E00E94FFDA24960E94B1531BC0E4300A
:10923A00A0E0FA0769F4EBE4F5E060E070E00E9470
:10924A0005DD80E00E94FFDA24960E94115C0AC0C4
:10925A00E3E5F5E060E070E00E9405DD80E00E9451
:10926A00FFDA24960E947FDB26960895E0E0E093D9
:10927A00AB07A8E3B1E00E9463DD0895BA93AA930D
:10928A0023970E9478DBA985BA85EC91E07109F0F1
:10929A00A7C1E985FA85A181EFE7EA233E2F30309D
:1092AA0009F49EC100E0023008F09AC1AAE7B8E0CA
:1092BA00E02FF0E0BD01A1E7B0E00E942DDCDB0168
:1092CA00AE0FBF1F0E9447DD3E1709F087C1ACEA07
:1092DA00B7E0E02FF0E0BD01A9E1B0E00E942DDC8B
:1092EA00DB01AE0FBF1F1296EAE0EC93E985FA851F
:1092FA00A181B281E7E00E94B3DBEE83F0E0EE30B9
:10930A00A0E0FA0709F46AC1E330A0E0FA0709F01D
:10931A0065C1ACEAB7E0E02FF0E0BD01A9E1B0E039
:10932A000E942DDCDB01AE0FBF1FEC91E07889F5BE
:10933A00ACEAB7E0E02FF0E0BD01A9E1B0E00E949D
:10934A002DDCDB01AE0FBF1FEC91E068EC93ACEAB9
:10935A00B7E0E02FF0E0BD01A9E1B0E00E942DDC0A
:10936A00DB01AE0FBF1F1196E0E0EC93EAE5F5E0F2
:10937A0060E070E00E9405DDE02FF0E031966F2F8B
:10938A00660F660B762F0E9405DD84E00E94FFDAE5
:10939A002896ACEAB7E0E02FF0E0BD01A9E1B0E021
:1093AA000E942DDCDB01AE0FBF1F1296E1E1EC93A8
:1093BA00ACEAB7E0E02FF0E0BD01A9E1B0E00E941D
:1093CA002DDCE60FF71F4185ACEAB7E0E02FF0E0AD
:1093DA00BD01A9E1B0E00E942DDCDB01AE0FBF1F89
:1093EA001796EC91E887ACEAB7E0E02FF0E0BD0110
:1093FA00A9E1B0E00E942DDCDB01AE0FBF1F15967C
:10940A00EC91EF83E985FA85258110E051E0183067
:10941A0008F5E52FAF81EA2391F0E52FE22349F021
:10942A00E52FA885EA2321F44527E52FEA2BE887CB
:10943A0005C0E52FE095A885EA23E88708C0E52F4F
:10944A00E22311F0452B03C0E52FE0954E231F5F61
:10945A00550FDDCFACEAB7E0E02FF0E0BD01A9E19E
:10946A00B0E00E942DDCDB01AE0FBF1F1996AC9154
:10947A004A17D9F0ACEAB7E0E02FF0E0BD01A9E164
:10948A00B0E00E942DDCE60FF71F4187ACEAB7E097
:10949A00E02FF0E0BD01A9E1B0E00E942DDCDB0184
:1094AA00AE0FBF1F1396E0E0EC93ACEAB7E0E02FF3
:1094BA00F0E0BD01A9E1B0E00E942DDCE60FF71F44
:1094CA003796A885A083ACEAB7E0E02FF0E0BD01AB
:1094DA00A9E1B0E00E942DDCE60FF71F4285ACEA55
:1094EA00B7E0E02FF0E0BD01A9E1B0E00E942DDC79
:1094FA00DB01AE0FBF1F1896EC91E887ACEAB7E024
:10950A00E02FF0E0BD01A9E1B0E00E942DDCDB0113
:10951A00AE0FBF1F1696EC91EF83E985FA85268177
:10952A0010E051E0143008F5E52FAF81EA2391F0FD
:10953A00E52FE22349F0E52FA885EA2321F4452700
:10954A00E52FEA2BE88705C0E52FE095A885EA23F1
:10955A00E88708C0E52FE22311F0452B03C0E52F69
:10956A00E0954E231F5F550FDDCFACEAB7E0E02F41
:10957A00F0E0BD01A9E1B0E00E942DDCDB01AE0FF5
:10958A00BF1F1A96AC914A17D9F0ACEAB7E0E02FA0
:10959A00F0E0BD01A9E1B0E00E942DDCE60FF71F63
:1095AA004287ACEAB7E0E02FF0E0BD01A9E1B0E004
:1095BA000E942DDCDB01AE0FBF1F1396E0E0EC9397
:1095CA00ACEAB7E0E02FF0E0BD01A9E1B0E00E940B
:1095DA002DDCE60FF71F3896A885A0830F5F63CEB0
:1095EA000E947FDB2B9608956F970E9478DBE091AB
:1095FA006304E07409F4F8C640E0423008F0F4C6A7
:10960A00ACEAB7E0E42FF0E0BD01A9E1B0E00E94C6
:10961A002DDCDB01AE0FBF1F1296AC91A13008F40E
:10962A00E1C6ACEAB7E0E42FF0E0BD01A9E1B0E0A1
:10963A000E942DDCDB01AE0FBF1FEC91EF775E2F8E
:10964A00ACEAB7E0E42FF0E0BD01A9E1B0E00E9486
:10965A002DDCDB01AE0FBF1F1396AC91A13080F059
:10966A00ACEAB7E0E42FF0E0BD01A9E1B0E00E9466
:10967A002DDCDB01AE0FBF1F1396EC91E150A7C49E
:10968A00ACEAB7E0E42FF0E0BD01A9E1B0E00E9446
:10969A002DDCDB01AE0FBF1F1396E4E0EC93FE0155
:1096AA003C96FA93EA93E0E0EA93A6E0B0E00E94DF
:1096BA0077D4FE013696FA93EA93E0E0EA93A6E0BD
:1096CA00B0E00E9477D420E0E1E0EE8BE0E1ED8BA0
:1096DA00251708F003C400E030E0AAE7B8E0E42F59
:1096EA00F0E0BD01A1E7B0E00E942DDCDB01AE0F86
:1096FA00BF1F1E96E22FF0E00E94F4DBAE0FBF1FE1
:10970A0015960E9447DD1E2FA12F0E9480853E2FAD
:10971A003030E9F4AAE7B8E0E42FF0E0BD01A1E7B0
:10972A00B0E00E942DDCDB01AE0FBF1F1E96E22FB8
:10973A00F0E00E94F4DBAE0FBF1F14960E9447DDD3
:10974A001E2F103021F0A12F0E9480853E2F30302D
:10975A00E9F4AAE7B8E0E42FF0E0BD01A1E7B0E040
:10976A000E942DDCDB01AE0FBF1F1E96E22FF0E038
:10977A000E94F4DBAE0FBF1F13960E9447DD1E2F17
:10978A00103021F0A12F0E9480853E2F303009F43D
:10979A00C4C0E32FF0E0E130A0E0FA0729F5AAE718
:1097AA00B8E0E42FF0E0BD01A1E7B0E00E942DDCB3
:1097BA00DB01AE0FBF1F1C960E9447DDE295E770E2
:1097CA000E2FAAE7B8E0E42FF0E0BD01A1E7B0E070
:1097DA000E942DDCDB01AE0FBF1F1C960E9447DDE5
:1097EA00EE1FE0E0EE1F96C0E230A0E0FA07F9F4BF
:1097FA00AAE7B8E0E42FF0E0BD01A1E7B0E00E94DB
:10980A002DDCDB01AE0FBF1F1C960E9447DDE770FF
:10981A000E2FAAE7B8E0E42FF0E0BD01A1E7B0E01F
:10982A000E942DDCDB01AE0FBF1F1C966EC0E33019
:10983A00A0E0FA0729F5AAE7B8E0E42FF0E0BD01B5
:10984A00A1E7B0E00E942DDCDB01AE0FBF1F1B9623
:10985A000E9447DDE295E7700E2FAAE7B8E0E42FF1
:10986A00F0E0BD01A1E7B0E00E942DDCDB01AE0F04
:10987A00BF1F1B960E9447DDEE1FE0E0EE1F4AC0A5
:10988A00E430A0E0FA07F9F4AAE7B8E0E42FF0E040
:10989A00BD01A1E7B0E00E942DDCDB01AE0FBF1FC6
:1098AA001B960E9447DDE7700E2FAAE7B8E0E42F67
:1098BA00F0E0BD01A1E7B0E00E942DDCDB01AE0FB4
:1098CA00BF1F1B9622C0E530A0E0FA0729F5AAE7D8
:1098DA00B8E0E42FF0E0BD01A1E7B0E00E942DDC82
:1098EA00DB01AE0FBF1F1D960E9447DDE7700E2FEA
:1098FA00AAE7B8E0E42FF0E0BD01A1E7B0E00E94DA
:10990A002DDCDB01AE0FBF1F1D960E9447DDE695D9
:10991A00E695E695E170EF8BF0C0AAE7B8E0E42F90
:10992A00F0E0BD01A1E7B0E00E942DDCDB01AE0F43
:10993A00BF1F1E96E22FF0E00E94F4DBAE0FBF1F9E
:10994A0012960E9447DD1E2F103029F0A12F0E9487
:10995A00E03DE03009F42EC0AAE7B8E0E42FF0E0D9
:10996A00BD01A1E7B0E00E942DDCDB01AE0FBF1FF5
:10997A001E96E22FF0E00E94F4DBAE0FBF1F17968F
:10998A000E9447DDE295E7700E2FAAE7B8E0E42FC0
:10999A00F0E0BD01A1E7B0E00E942DDCDB01AE0FD3
:1099AA00BF1F1E96E22FF0E00E94F4DBAE0FBF1F2E
:1099BA0017969CC0AAE7B8E0E42FF0E0BD01A1E742
:1099CA00B0E00E942DDCDB01AE0FBF1F1E96E22F16
:1099DA00F0E00E94F4DBAE0FBF1F11960E9447DD34
:1099EA001E2F103029F0A12F0E94E03DE03009F42B
:1099FA0032C0AAE7B8E0E42FF0E0BD01A1E7B0E089
:109A0A000E942DDCDB01AE0FBF1F1E96E22FF0E095
:109A1A000E94F4DBAE0FBF1F17960E9447DDE77066
:109A2A000E2FAAE7B8E0E42FF0E0BD01A1E7B0E00D
:109A3A000E942DDCDB01AE0FBF1F1E96E22FF0E065
:109A4A000E94F4DBAE0FBF1F17960E9447DDE69512
:109A5A00E695E69550C0AAE7B8E0E42FF0E0BD012C
:109A6A00A1E7B0E00E942DDCDB01AE0FBF1F1E96FE
:109A7A00E22FF0E00E94F4DBAE0FBF1F0E9447DD29
:109A8A001E2F103029F0A12F0E94E03DE03009F48A
:109A9A0034C0AAE7B8E0E42FF0E0BD01A1E7B0E0E6
:109AAA000E942DDCDB01AE0FBF1F1E96E22FF0E0F5
:109ABA000E94F4DBAE0FBF1F16960E9447DDE295A7
:109ACA00E7700E2FAAE7B8E0E42FF0E0BD01A1E7A6
:109ADA00B0E00E942DDCDB01AE0FBF1F1E96E22F05
:109AEA00F0E00E94F4DBAE0FBF1F16960E9447DD1E
:109AFA00EE1FE0E0EE1FE170EF8BEF89E03009F432
:109B0A00C9C0E02FF0E0E130A0E0FA0781F4283084
:109B1A0028F4EE89AE81EA2BEE8308C0FE0137965F
:109B2A000F01E081AE89EA2BD001EC93B2C0E2309A
:109B3A00A0E0FA0771F4243018F4FE01379602C047
:109B4A00FE0138960F01E081AD89EA2BD001EC9332
:109B5A00A0C0E330A0E0FA0771F4283018F4FE013F
:109B6A00399602C0FE013A960F01E081AE89EA2BCE
:109B7A00D001EC938EC0E430A0E0FA07E9F4283073
:109B8A0028F4EE89AE81EA2BEE8308C0FE013796EF
:109B9A000F01E081AE89EA2BD001EC93243018F44E
:109BAA00FE01379602C0FE0138960F01E081AD89A9
:109BBA00EA2BD001EC936DC0E530A0E0FA07D9F4A6
:109BCA00243018F4FE01379602C0FE0138960F01C0
:109BDA00E081AD89EA2BD001EC93283018F4FE011C
:109BEA00399602C0FE013A960F01E081AE89EA2B4E
:109BFA00D001EC934EC0E630A0E0FA07E9F4283031
:109C0A0028F4EE89AE81EA2BEE8308C0FE0137966E
:109C1A000F01E081AE89EA2BD001EC93283018F4C9
:109C2A00FE01399602C0FE013A960F01E081AE8923
:109C3A00EA2BD001EC932DC0E730A0E0FA0749F5F2
:109C4A00283028F4EE89AE81EA2BEE8308C0FE01A3
:109C5A0037960F01E081AE89EA2BD001EC932430CC
:109C6A0018F4FE01379602C0FE0138960F01E08112
:109C7A00AD89EA2BD001EC93283018F4FE0139960D
:109C8A0002C0FE013A960F01E081AE89EA2BD001AB
:109C9A00EC9312C1593008F047C0E02FF0E0E130F0
:109CAA00A0E0FA0729F4EE89AC85EA2BEC873BC0E1
:109CBA00E230A0E0FA0719F4FE013D962EC0E33027
:109CCA00A0E0FA0741F1E430A0E0FA0739F4EE899E
:109CDA00AC85EA2BEC87FE013D961FC0E530A0E07B
:109CEA00FA0789F0E630A0E0FA0729F4EE89AC8594
:109CFA00EA2BEC8710C0E730A0E0FA07A1F4EE895E
:109D0A00AC85EA2BEC87FE013D960F01E081AE8916
:109D1A00EA2BD001EC93FE013E960F01E081AE8959
:109D2A00EA2BD001EC93C8C0E02FF0E0E130A0E0CC
:109D3A00FA0781F4283028F4EE89AC85EA2BEC87FF
:109D4A0008C0FE013D960F01E081AE89EA2BD001E1
:109D5A00EC93B2C0E230A0E0FA0771F4243018F4B0
:109D6A00FE013D9602C0FE013E960F01E081AD89DB
:109D7A00EA2BD001EC93A0C0E330A0E0FA0771F41B
:109D8A00283018F4FE013F9602C0FE0170960F01BA
:109D9A00E081AE89EA2BD001EC938EC0E430A0E0DA
:109DAA00FA07E9F4283028F4EE89AC85EA2BEC8727
:109DBA0008C0FE013D960F01E081AE89EA2BD00171
:109DCA00EC93243018F4FE013D9602C0FE013E9643
:109DDA000F01E081AD89EA2BD001EC936DC0E5302B
:109DEA00A0E0FA07D9F4243018F4FE013D9602C027
:109DFA00FE013E960F01E081AD89EA2BD001EC937A
:109E0A00283018F4FE013F9602C0FE0170960F0139
:109E1A00E081AE89EA2BD001EC934EC0E630A0E097
:109E2A00FA07E9F4283028F4EE89AC85EA2BEC87A6
:109E3A0008C0FE013D960F01E081AE89EA2BD001F0
:109E4A00EC93283018F4FE013F9602C0FE0170968A
:109E5A000F01E081AE89EA2BD001EC932DC0E730E7
:109E6A00A0E0FA0749F5283028F4EE89AC85EA2BF8
:109E7A00EC8708C0FE013D960F01E081AE89EA2B0E
:109E8A00D001EC93243018F4FE013D9602C0FE0185
:109E9A003E960F01E081AD89EA2BD001EC93283080
:109EAA0018F4FE013F9602C0FE0170960F01E08190
:109EBA00AE89EA2BD001EC93EE89EE0FEE8BED8999
:109ECA00EE0FED8BEE89E03011F4E1E0EE8BED89D7
:109EDA00E03011F4E1E0ED8B2F5FFACBACEAB7E0AA
:109EEA00E42FF0E0BD01A9E1B0E00E942DDCE60F0D
:109EFA00F71F3B96FA93EA93FE013E96FA93EA938A
:109F0A00A6E0B0E00E944CD4E03029F1ACEAB7E018
:109F1A00E42FF0E0BD01A9E1B0E00E942DDCE60FDC
:109F2A00F71F3B96FA93EA93FE013E96FA93EA9359
:109F3A00A6E0B0E00E9465D4ACEAB7E0E42FF0E016
:109F4A00BD01A9E1B0E00E942DDCDB01AE0FBF1F0D
:109F5A005796E0E0EC93ACEAB7E0E42FF0E0BD01FD
:109F6A00A9E1B0E00E942DDCE60FF71F7196FA9383
:109F7A00EA93FE013896FA93EA93A6E0B0E00E94CB
:109F8A004CD4E03029F1ACEAB7E0E42FF0E0BD01AF
:109F9A00A9E1B0E00E942DDCE60FF71F7196FA9353
:109FAA00EA93FE013896FA93EA93A6E0B0E00E949B
:109FBA0065D4ACEAB7E0E42FF0E0BD01A9E1B0E076
:109FCA000E942DDCDB01AE0FBF1F5896E0E0EC9338
:109FDA00ACEAB7E0E42FF0E0BD01A9E1B0E00E94ED
:109FEA002DDCDB01AE0FBF1F1496AC91A13088F0B7
:109FFA00ACEAB7E0E42FF0E0BD01A9E1B0E00E94CD
:10A00A002DDCDB01AE0FBF1F1496EC91E150EC93EF
:10A01A0024C1ACEAB7E0E42FF0E0BD01A9E1B0E069
:10A02A000E942DDCDB01AE0FBF1F5796AC91A13009
:10A03A0080F0ACEAB7E0E42FF0E0BD01A9E1B0E0BE
:10A04A000E942DDCDB01AE0FBF1F5896AC91A130E8
:10A05A0008F403C1ACEAB7E0E42FF0E0BD01A9E1DE
:10A06A00B0E00E942DDCDB01AE0FBF1F1496E4E6C0
:10A07A00EC93AAE7B8E0E42FF0E0BD01A1E7B0E075
:10A08A000E942DDCDB01AE0FBF1F17960E9447DD31
:10A09A00AE2F0E94E03DE03081F1AAE7B8E0E42F5C
:10A0AA00F0E0BD01A1E7B0E00E942DDCDB01AE0FBC
:10A0BA00BF1F18960E9447DDEC8BAAE7B8E0E42F91
:10A0CA00F0E0BD01A1E7B0E00E942DDCDB01AE0F9C
:10A0DA00BF1F1A960E9447DDE295EF70EB8BAAE745
:10A0EA00B8E0E42FF0E0BD01A1E7B0E00E942DDC6A
:10A0FA00DB01AE0FBF1F199671C0AAE7B8E0E42FC3
:10A10A00F0E0BD01A1E7B0E00E942DDCDB01AE0F5B
:10A11A00BF1F14960E9447DDAE2F0E94E03DE0303B
:10A12A0079F1AAE7B8E0E42FF0E0BD01A1E7B0E0D9
:10A13A000E942DDCDB01AE0FBF1F15960E9447DD82
:10A14A00EC8BAAE7B8E0E42FF0E0BD01A1E7B0E0AC
:10A15A000E942DDCDB01AE0FBF1F1A960E9447DD5D
:10A16A00EF70EB8BAAE7B8E0E42FF0E0BD01A1E7BE
:10A17A00B0E00E942DDCDB01AE0FBF1F16962EC089
:10A18A00AAE7B8E0E42FF0E0BD01A1E7B0E00E9441
:10A19A002DDCDB01AE0FBF1F12960E9447DDEC8B50
:10A1AA00AAE7B8E0E42FF0E0BD01A1E7B0E00E9421
:10A1BA002DDCDB01AE0FBF1F11960E9447DDEF7049
:10A1CA00EB8BAAE7B8E0E42FF0E0BD01A1E7B0E02D
:10A1DA000E942DDCDB01AE0FBF1F13960E9447DDE4
:10A1EA00EA8BE88DE07FE160E88FEF7EE88FAAE7EF
:10A1FA00B8E0E42FF0E0BD01A1E7B0E00E942DDC59
:10A20A00DB01AE0FBF1F0E9447DDF0E0F460E98F6B
:10A21A00FA8FEA89ED8FDE0158960E94B109E88D1E
:10A22A00E07FE260E88FAAE7B8E0E42FF0E0BD0142
:10A23A00A1E7B0E00E942DDCDB01AE0FBF1F0E9438
:10A24A0047DDF0E0F560E98FFA8FEC89ED8FEB8955
:10A25A00EE8FDE0158960E94B109593010F0E6E0FF
:10A26A0001C0E3E0EF700E2EE88DE07FE029E88F71
:10A27A00EF7EE88FACEAB7E0E42FF0E0BD01A9E198
:10A28A00B0E00E942DDCDB01AE0FBF1F5796AC91E8
:10A29A00A13088F0ACEAB7E0E42FF0E0BD01A9E113
:10A2AA00B0E00E942DDCDB01AE0FBF1F5796EC9188
:10A2BA00E150EC933BC0ACEAB7E0E42FF0E0BD011B
:10A2CA00A9E1B0E00E942DDCDB01AE0FBF1F57965B
:10A2DA00EAEFEC93AAE7B8E0E42FF0E0BD01A1E7CA
:10A2EA00B0E00E942DDCDB01AE0FBF1F0E9447DDEC
:10A2FA00F0E0F260E98FFA8FFE017D96FA93EA9315
:10A30A00ACEAB7E0E42FF0E0BD01A9E1B0E00E94B9
:10A31A002DDCE60FF71F3B96FA93EA93A6E0B0E02E
:10A32A000E9465D4DE0158960E94B109ACEAB7E0F2
:10A33A00E42FF0E0BD01A9E1B0E00E942DDCDB01D1
:10A34A00AE0FBF1F5896AC91A13088F0ACEAB7E0C7
:10A35A00E42FF0E0BD01A9E1B0E00E942DDCDB01B1
:10A36A00AE0FBF1F5896EC91E150EC933BC0ACEA9C
:10A37A00B7E0E42FF0E0BD01A9E1B0E00E942DDCD6
:10A38A00DB01AE0FBF1F5896EAEFEC93AAE7B8E0DD
:10A39A00E42FF0E0BD01A1E7B0E00E942DDCDB0173
:10A3AA00AE0FBF1F0E9447DDF0E0F360E98FFA8F1E
:10A3BA00FE017D96FA93EA93ACEAB7E0E42FF0E067
:10A3CA00BD01A9E1B0E00E942DDCE60FF71F7196EE
:10A3DA00FA93EA93A6E0B0E00E9465D4DE015896AB
:10A3EA000E94B1094F5F09C90E947FDBA5960895B3
:10A3FA002D970E947ADBE0916304E07409F4A8C106
:10A40A0000E0023008F0A4C1AAE7B8E0E02FF0E0CB
:10A41A00BD01A1E7B0E00E942DDCDB01AE0FBF1F3A
:10A42A000E9447DDE03081F4ACEAB7E0E02FF0E0CB
:10A43A00BD01A9E1B0E00E942DDCDB01AE0FBF1F18
:10A44A001296E0E0EC9382C1ACEAB7E0E02FF0E0CC
:10A45A00BD01A9E1B0E00E942DDCDB01AE0FBF1FF8
:10A46A001296AC91A13008F46CC0ACEAB7E0E02FC8
:10A47A00F0E0BD01A9E1B0E00E942DDCDB01AE0FE6
:10A48A00BF1F1296EC91E150EC93ACEAB7E0E02FD3
:10A49A00F0E0BD01A9E1B0E00E942DDCDB01AE0FC6
:10A4AA00BF1F1196AC91A13088F0ACEAB7E0E02F5B
:10A4BA00F0E0BD01A9E1B0E00E942DDCDB01AE0FA6
:10A4CA00BF1F1196EC91E150EC933AC0ACEAB7E0A9
:10A4DA00E02FF0E0BD01A9E1B0E00E942DDCDB0134
:10A4EA00AE0FBF1F1196E2E3EC93EC81E07FE860C8
:10A4FA00EC83EF7EEC83AAE7B8E0E02FF0E0BD0141
:10A50A00A1E7B0E00E942DDCDB01AE0FBF1F0E9465
:10A51A0047DDF0E0F660ED83FE83EBE2E987E0E0F9
:10A52A00EA87E8E1EB87E5E0EC87E4EFED87E1E035
:10A53A00EE87E0E0EF87E88BDE0114960E94B1090E
:10A54A0005C1ACEAB7E0E02FF0E0BD01A9E1B0E057
:10A55A000E942DDCDB01AE0FBF1FEC91E07809F4FD
:10A56A00C8C0ACEAB7E0E02FF0E0BD01A9E1B0E075
:10A57A000E942DDCDB01AE0FBF1FEC91EF773E2F5F
:10A58A00ACEAB7E0E02FF0E0BD01A9E1B0E00E943B
:10A59A002DDCDB01AE0FBF1FEC91EF77EC93EAE6FF
:10A5AA00F5E060E070E00E9405DDE02FF0E0319612
:10A5BA006F2F660F660B762F0E9405DD84E00E94DE
:10A5CA00FFDA289621E010E0131708F047C0AAE73F
:10A5DA00B8E0E02FF0E0BD01A1E7B0E00E942DDC79
:10A5EA00DB01AE0FBF1F1E96E12FF0E00E94F4DBE5
:10A5FA00AE0FBF1F16960E9447DDF0E0F695E7956D
:10A60A00E370F070309799F4ACEAB7E0E02FF0E02D
:10A61A00BD01A9E1B0E00E942DDCE60FF71F3996D3
:10A62A000F01A081E22FE095EA23D00113C0E130A7
:10A63A00A0E0FA0781F4ACEAB7E0E02FF0E0BD0150
:10A64A00A9E1B0E00E942DDCDB01AE0FBF1F199615
:10A65A00EC91E22BEC931F5F220FB6CF21E0131788
:10A66A0008F047C0AAE7B8E0E02FF0E0BD01A1E793
:10A67A00B0E00E942DDCDB01AE0FBF1F1E96E12F5A
:10A68A00F0E00E94F4DBAE0FBF1F16960E9447DD72
:10A69A00F0E0F695E795E370F070309799F4ACEA3C
:10A6AA00B7E0E02FF0E0BD01A9E1B0E00E942DDCA7
:10A6BA00E60FF71F3A960F01A081E22FE095EA23F1
:10A6CA00D00113C0E130A0E0FA0781F4ACEAB7E0A8
:10A6DA00E02FF0E0BD01A9E1B0E00E942DDCDB0132
:10A6EA00AE0FBF1F1A96EC91E22BEC931F5F220F5D
:10A6FA00B6CFACEAB7E0E02FF0E0BD01A9E1B0E0E7
:10A70A000E942DDCDB01AE0FBF1F1296EAE0EC932C
:10A71A00EC81E07FE260EC83EF7EEC83E0E0ED83A6
:10A72A00EE83E1E0E987AAE7B8E0E02FF0E0BD01B7
:10A73A00A1E7B0E00E942DDCDB01AE0FBF1F0E9433
:10A74A0047DDEA87DE0114960E94B1090F5F59CEF0
:10A75A000E9481DB619608950E947ADB10E0133033
:10A76A0008F081C0AEEAB7E0E12FF0E0BD01ACE04D
:10A77A00B0E00E942DDCE60FF71F3196FF93EF93AE
:10A78A00AAE7B8E0E12FF0E0BD01AAE0B0E00E943C
:10A79A002DDCDB01AE0FBF1F0E9447DDAF91BF91D9
:10A7AA00EC93AEEAB7E0E12FF0E0BD01ACE0B0E037
:10A7BA000E942DDCE60FF71F3296FF93EF93AAE76C
:10A7CA00B8E0E12FF0E0BD01AAE0B0E00E942DDC84
:10A7DA00DB01AE0FBF1F11960E9447DDAF91BF91FB
:10A7EA00EC93AEEAB7E0E12FF0E0BD01ACE0B0E0F7
:10A7FA000E942DDCE60FF71F3596FF93EF93AAE729
:10A80A00B8E0E12FF0E0BD01AAE0B0E00E942DDC43
:10A81A00DB01AE0FBF1F12960E9447DDAF91BF91B9
:10A82A00EC93AEEAB7E0E12FF0E0BD01ACE0B0E0B6
:10A83A000E942DDCE60FF71F3696FF93EF93AAE7E7
:10A84A00B8E0E12FF0E0BD01AAE0B0E00E942DDC03
:10A85A00DB01AE0FBF1F15960E9447DDAF91BF9176
:10A86A00EC931F5F7CCFE091B007E093BD07A09106
:10A87A00B007E091BC07EA0FE093C907A091C907A6
:10A88A00E091C807EA0FE093AD0710E0183108F02D
:10A89A00E1C0E0E03E2F0E2FA8E9B8E0E12FF0E09A
:10A8AA00BD01ACE0B0E00E942DDCDB01AE0FBF1FA2
:10A8BA0011960E9447DDE03009F031E0A8E9B8E0DE
:10A8CA00E12FF0E0BD01ACE0B0E00E942DDCDB013D
:10A8DA00AE0FBF1F12960E9447DDE03009F03260CA
:10A8EA00A8E9B8E0E12FF0E0BD01ACE0B0E00E94D9
:10A8FA002DDCDB01AE0FBF1F15960E9447DDE0304D
:10A90A0009F03460A8E9B8E0E12FF0E0BD01ACE05D
:10A91A00B0E00E942DDCDB01AE0FBF1F16960E942D
:10A92A0047DDE03009F03860A8E9B8E0E12FF0E04F
:10A93A00BD01ACE0B0E00E942DDCDB01AE0FBF1F11
:10A94A0019960E9447DDE03009F03061A8E9B8E0C5
:10A95A00E12FF0E0BD01ACE0B0E00E942DDCDB01AC
:10A96A00AE0FBF1F1A960E9447DDE03009F0306231
:10A97A00A8E9B8E0E12FF0E0BD01ACE0B0E00E9448
:10A98A002DDCDB01AE0FBF1F13960E9447DDE030BE
:10A99A0009F000E1A8E9B8E0E12FF0E0BD01ACE080
:10A9AA00B0E00E942DDCDB01AE0FBF1F17960E949C
:10A9BA0047DDE03009F00062A8E9B8E0E12FF0E0F5
:10A9CA00BD01ACE0B0E00E942DDCDB01AE0FBF1F81
:10A9DA001B960E9447DDE03009F00064A2EDB7E063
:10A9EA00E12FF0E00E94F6DBEA0FFB1F0283A2EDE3
:10A9FA00B7E0E12FF0E00E94F6DBEA0FFB1F33839A
:10AA0A00A2EDB7E0E12FF0E00E94F6DBEA0FFB1FB0
:10AA1A003296FF93EF93A8E9B8E0E12FF0E0BD0189
:10AA2A00ACE0B0E00E942DDCDB01AE0FBF1F0E943C
:10AA3A0047DDE295EF70E695E695E170AF91BF913B
:10AA4A00E170EE0FEE0F0E2EEC91EB7FE029EC9306
:10AA5A001F5F1CCF0E9481DB24960895BA93AA93A4
:10AA6A0025970E9478DBE091AB07F0E0E230A0E0A6
:10AA7A00FA0739F4AB85BC85EC91E07109F02AC17B
:10AA8A000AC0E330A0E0FA0731F4AB85BC85EC914B
:10AA9A00E07109F41FC1E091AB07F0E0E230A0E0F9
:10AAAA00FA0729F0E330A0E0FA0709F013C110E031
:10AABA00133008F00FC1AEEAB7E0E12FF0E0BD01B4
:10AACA00ACE0B0E00E942DDCE60FF71F22812130B6
:10AADA0008F4FDC0AEEAB7E0E12FF0E0BD01ACE05A
:10AAEA00B0E00E942DDCE60FF71F3181A091AB0781
:10AAFA00A23089F4E32FF0E0E058FE4F0F01AB8556
:10AB0A00BC851196ED91FC911197E015F10509F0BC
:10AB1A00DFC0E1E007C0EB85FC85E181E31709F0BE
:10AB2A00D7C0E3E0EA87AEEAB7E0E12FF0E0BD0183
:10AB3A00ACE0B0E00E942DDCDB01AE0FBF1FEC9150
:10AB4A00E03079F4AEEAB7E0E12FF0E0BD01ACE025
:10AB5A00B0E00E942DDCDB01AE0FBF1F1496EFEFB1
:10AB6A00EC93AEEAB7E0E12FF0E0BD01ACE0B0E073
:10AB7A000E942DDCDB01AE0FBF1FECE0EC93AEEAC6
:10AB8A00B7E0E12FF0E0BD01ACE0B0E00E942DDCBF
:10AB9A00E60FF71F5381E0E04E2FE8870E2F42178A
:10ABAA0008F094C0A091AB07A230A1F4003069F478
:10ABBA0007E0AB85BC851596E885EF5FE887E1502D
:10ABCA00F0E0AE0FBF1FEC9103C00150E985E69596
:10ABDA00E98714C0003069F403E0AB85BC8515969B
:10ABEA00E885EF5FE887E150F0E0AE0FBF1FEC9118
:10ABFA0004C00150E985E695E695E987A2EDB7E03C
:10AC0A00E52FF0E00E94F6DBAE0FBF1F1296EC9123
:10AC1A00E47009F43FC0A2EDB7E0E52FF0E00E942E
:10AC2A00F6DBAE0FBF1F1296EC91E170EF83A2ED37
:10AC3A00B7E0E52FF0E00E94F6DBAE0FBF1F1296D9
:10AC4A00EC91E695E170EE83EA85A985EA23E13085
:10AC5A0069F4EE81E03049F4E1E0EE83EF81E0301F
:10AC6A0011F0E0E001C0E1E0EF8302C0E0E0EE8332
:10AC7A00A2EDB7E0E52FF0E00E94F6DBAE0FBF1FB2
:10AC8A001296EE81E170EE0F0E2EEC91ED7FE02927
:10AC9A00EC9309C0EA85A985EA23E13011F4E1E0E1
:10ACAA0001C0E0E0EF83A2EDB7E0E52FF0E00E94FB
:10ACBA00F6DBAE0FBF1F1296EF81E1700E2EEC91FC
:10ACCA00EE7FE029EC934F5F5F5F69CF03C002C05C
:10ACDA001F5FEECE0E947FDB2D9608952D970E946E
:10ACEA007ADB1A2F09893A89EC81E061EC83E07FEB
:10ACFA00E860EC83F32FE0E066277727E060F060F6
:10AD0A006F6E7861DF01CB01E0915C04FF27662753
:10AD1A007727EA2BFB2B682B792BED83FE836F8336
:10AD2A007887E02FEF5FE987A2EDB7E0E12FF0E047
:10AD3A000E94F6DBAE0FBF1FEC91EA87A2EDB7E0E7
:10AD4A00E12FF0E00E94F6DBAE0FBF1F1196EC91E7
:10AD5A00EB87C9C02D970E9478DB4A2FEE81EF7EE0
:10AD6A00EE83E07FE860EE83EC89F0E0E050FE4F8E
:10AD7A00EF83F887FE013B96FA93EA93E0E0EA93C1
:10AD8A00A8E0B0E00E9477D451E020E031E0E0E0B2
:10AD9A000E2F1E2F141708F04BC030E0333008F086
:10ADAA0042C0503051F4E02F0F5FF0E0DE011B96F5
:10ADBA00EA0FFB1F208351E020E0E32FF0E03097F9
:10ADCA0069F4A2EDB7E0EB89F0E00E94F6DBAE0F82
:10ADDA00BF1FEC91EF7009F0252B22C0E130A0E0F3
:10ADEA00FA0769F4A2EDB7E0EB89F0E00E94F6DB1E
:10ADFA00AE0FBF1FEC91E07F09F0252B11C0E230A6
:10AE0A00A0E0FA0769F4A2EDB7E0EB89F0E00E944E
:10AE1A00F6DBAE0FBF1F1196EC91E03009F0252B3F
:10AE2A00550F3F5FBBCF1F5FEB89EF5FEB8BB2CF55
:10AE3A00E02FF0E0DE011B96EA0FFB1F2083DE0104
:10AE4A0016960E94B1090E947FDB659608952D9798
:10AE5A000E947ADB1A2F09893A89FE013996FA93F8
:10AE6A00EA93E0E0EA93A0E0B0E00E9477D4EC81B4
:10AE7A00EF7EEC83E07FE860EC83E32FF0E0E050C4
:10AE8A00FD4FED83FE831987FE013B96008335C093
:10AE9A002D970E947ADB1A2F09893A89EC81E061A1
:10AEAA00EC83E07FE860EC83F32FE0E06627772706
:10AEBA00E060F060606D7861DF01CB01E0915C04D5
:10AECA00FF2766277727EA2BFB2B682B792BED8345
:10AEDA00FE836F837887E0E0E987FE013A96008374
:10AEEA00FE013B961083FE013C96FA93EA93EFEF3C
:10AEFA00EA93A5E0B0E00E9477D4DE0114960E949E
:10AF0A00B1090E9481DB6396089562970E9478DBFB
:10AF1A00E0916304E07409F47BC4A091AC07A43007
:10AF2A0038F4E091AC07EF5FE093AC07E15003C05F
:10AF3A00E0E0E093AC07A091AC07A33008F068C446
:10AF4A00AEEAB7E0E091AC07F0E0BD01ACE0B0E0FA
:10AF5A000E942DDCE60FF71F5181AEEAB7E0E091BF
:10AF6A00AC07F0E0BD01ACE0B0E00E942DDCE60FDA
:10AF7A00F71F1281AEEAB7E0E091AC07F0E0BD013D
:10AF8A00ACE0B0E00E942DDCE60FF71F33811130F0
:10AF9A0010F0103108F03CC4E091AB07F0E0E23069
:10AFAA00A0E0FA0729F0E330A0E0FA0709F030C47C
:10AFBA00AEEAB7E0E091AC07F0E0BD01ACE0B0E08A
:10AFCA000E942DDCDB01AE0FBF1FAC91A13008F44B
:10AFDA0040C0AEEAB7E0E091AC07F0E0BD01ACE0FA
:10AFEA00B0E00E942DDCDB01AE0FBF1FEC91E150F7
:10AFFA00EC93AEEAB7E0E091AC07F0E0BD01ACE05B
:10B00A00B0E00E942DDCDB01AE0FBF1FEC91E030F7
:10B01A00F9F400E0232F0117D8F4A2EDB7E0E22FEC
:10B02A00F0E00E94F6DBAE0FBF1F1296EC91EE7FA6
:10B03A00EC93A2EDB7E0E22FF0E00E94F6DBAE0F50
:10B04A00BF1F1296EC91E260EC930F5F2F5FE3CF84
:10B05A0048C0A091AB07A23009F043C0AEEAB7E0FE
:10B06A00E091AC07F0E0BD01ACE0B0E00E942DDC5D
:10B07A00DB01AE0FBF1F1A96AC91A13088F0AEEA81
:10B08A00B7E0E091AC07F0E0BD01ACE0B0E00E94AF
:10B09A002DDCDB01AE0FBF1F1A96EC91E15020C0E8
:10B0AA00EE81E07FE260EE83EF7EEE83E0E0EF8305
:10B0BA00E887E1E0EB87E0E0EC87DE0116960E9484
:10B0CA00B109AEEAB7E0E091AC07F0E0BD01ACE04F
:10B0DA00B0E00E942DDCDB01AE0FBF1F1A96E4E13F
:10B0EA00EC93AEEAB7E0E091AC07F0E0BD01ACE06A
:10B0FA00B0E00E942DDCDB01AE0FBF1F1696AC91AB
:10B10A000E94E03DE03011F1AAE7B8E0E091AC0717
:10B11A00F0E0BD01AAE0B0E00E942DDCDB01AE0F39
:10B12A00BF1F16960E9447DD4E2FAAE7B8E0E091AE
:10B13A00AC07F0E0BD01AAE0B0E00E942DDCDB0123
:10B14A00AE0FBF1F17960E9447DD37C0AEEAB7E0C1
:10B15A00E091AC07F0E0BD01ACE0B0E00E942DDC6C
:10B16A00DB01AE0FBF1F1596AC910E94E03DE030A7
:10B17A0011F1AAE7B8E0E091AC07F0E0BD01AAE05E
:10B18A00B0E00E942DDCDB01AE0FBF1F13960E94B8
:10B19A0047DD4E2FAAE7B8E0E091AC07F0E0BD0129
:10B1AA00AAE0B0E00E942DDCDB01AE0FBF1F1496AF
:10B1BA000E9447DD02C040E0E0E0EF8BAEEAB7E074
:10B1CA00E091AC07F0E0BD01ACE0B0E00E942DDCFC
:10B1DA00DB01AE0FBF1F1796AC914A1799F4AEEA7E
:10B1EA00B7E0E091AC07F0E0BD01ACE0B0E00E944E
:10B1FA002DDCDB01AE0FBF1F1896AC91EF89EA1761
:10B20A0009F447C0AEEAB7E0E091AC07F0E0BD014F
:10B21A00ACE0B0E00E942DDCE60FF71F4783AEEAF0
:10B22A00B7E0E091AC07F0E0BD01ACE0B0E00E940D
:10B23A002DDCE60FF71F3896AF89A083A091AB07E4
:10B24A00A23011F55A93AEEAB7E0E091AC07F0E00C
:10B25A00BD01ACE0B0E00E942DDCDB01AE0FBF1FE8
:10B26A001896EC91EA93AEEAB7E0E091AC07F0E009
:10B27A00BD01ACE0B0E00E942DDCDB01AE0FBF1FC8
:10B28A001796AC91E4DD05C05A93E88DEA93A42F92
:10B29A00FFDD00E0232F011708F0E8C1A2EDB7E0B7
:10B2AA00E22FF0E00E94F6DBAE0FBF1F1296EC9180
:10B2BA00EE8BA2EDB7E0E22FF0E00E94F6DBAE0FD4
:10B2CA00BF1F1396EC91ED8BEE89E071A1F0A8E90E
:10B2DA00B8E0E22FF0E0BD01ACE0B0E00E942DDC66
:10B2EA00DB01AE0FBF1F13960E9447DDAE2F0E94EF
:10B2FA000465E03009F412C0A8E9B8E0E22FF0E0F2
:10B30A00BD01ACE0B0E00E942DDCDB01AE0FBF1F37
:10B31A000E9447DDE295E370EF5F55C0ED89E27068
:10B32A00A1F0A8E9B8E0E22FF0E0BD01ACE0B0E09E
:10B33A000E942DDCDB01AE0FBF1F12960E9447DD73
:10B34A00AE2F0E94E03DE03009F413C0A8E9B8E04E
:10B35A00E22FF0E0BD01ACE0B0E00E942DDCDB01A1
:10B36A00AE0FBF1F0E9447DDE695E695E370EF5FDB
:10B37A002AC0ED89E170A1F0A8E9B8E0E22FF0E077
:10B38A00BD01ACE0B0E00E942DDCDB01AE0FBF1FB7
:10B39A0011960E9447DDAE2F0E94E03DE03009F48D
:10B3AA0011C0A8E9B8E0E22FF0E0BD01ACE0B0E0DE
:10B3BA000E942DDCDB01AE0FBF1F0E9447DDE37048
:10B3CA00EF5F01C0E0E0EC8BEE89E072A1F0A8E942
:10B3DA00B8E0E22FF0E0BD01ACE0B0E00E942DDC65
:10B3EA00DB01AE0FBF1F17960E9447DDAE2F0E94EA
:10B3FA000465E03009F411C0A8E9B8E0E22FF0E0F2
:10B40A00BD01ACE0B0E00E942DDCDB01AE0FBF1F36
:10B41A0014960E9447DDE29551C0ED89E870A1F0CB
:10B42A00A8E9B8E0E22FF0E0BD01ACE0B0E00E948C
:10B43A002DDCDB01AE0FBF1F16960E9447DDAE2F33
:10B44A000E94E03DE03009F412C0A8E9B8E0E22F1A
:10B45A00F0E0BD01ACE0B0E00E942DDCDB01AE0FF4
:10B46A00BF1F14960E9447DDE695E69527C0ED8931
:10B47A00E470A1F0A8E9B8E0E22FF0E0BD01ACE089
:10B48A00B0E00E942DDCDB01AE0FBF1F15960E94B3
:10B49A0047DDAE2F0E94E03DE03009F416C0A8E96E
:10B4AA00B8E0E22FF0E0BD01ACE0B0E00E942DDC94
:10B4BA00DB01AE0FBF1F14960E9447DDE370EF5FFA
:10B4CA00E295E07FAC89EA2BEC8BEE89E074A1F07F
:10B4DA00A8E9B8E0E22FF0E0BD01ACE0B0E00E94DC
:10B4EA002DDCDB01AE0FBF1F1B960E9447DDAE2F7E
:10B4FA000E940465E03009F413C0A8E9B8E0E22F1D
:10B50A00F0E0BD01ACE0B0E00E942DDCDB01AE0F43
:10B51A00BF1F18960E9447DDE295E370EF5F57C0A0
:10B52A00ED89E072A1F0A8E9B8E0E22FF0E0BD01F0
:10B53A00ACE0B0E00E942DDCDB01AE0FBF1F1A9613
:10B54A000E9447DDAE2F0E94E03DE03009F414C0AE
:10B55A00A8E9B8E0E22FF0E0BD01ACE0B0E00E945B
:10B56A002DDCDB01AE0FBF1F18960E9447DDE69562
:10B57A00E695E370EF5F2BC0ED89E071A1F0A8E9D1
:10B58A00B8E0E22FF0E0BD01ACE0B0E00E942DDCB3
:10B59A00DB01AE0FBF1F19960E9447DDAE2F0E9436
:10B5AA00E03DE03009F412C0A8E9B8E0E22FF0E08B
:10B5BA00BD01ACE0B0E00E942DDCDB01AE0FBF1F85
:10B5CA0018960E9447DDE370EF5F01C0E0E0EB8B65
:10B5DA00A2EDB7E0E22FF0E00E94F6DBAE0FBF1F4C
:10B5EA00AC91EC89EA1769F4A2EDB7E0E22FF0E03A
:10B5FA000E94F6DBAE0FBF1F1196AC91EB89EA17DA
:10B60A0091F1A2EDB7E0E22FF0E00E94F6DBEA0F3B
:10B61A00FB1FAC89A083A2EDB7E0E22FF0E00E9405
:10B62A00F6DBEA0FFB1F3196AB89A083AEEAB7E0DF
:10B63A00E091AC07F0E0BD01ACE0B0E00E942DDC87
:10B64A00DB01AE0FBF1F1996E4E1EC93A091AB07A3
:10B65A00A23029F45A933A93A12F7CDB04C05A935F
:10B66A000A93A22F3BDB0F5F2F5F15CEAEEAB7E03E
:10B67A00E091AC07F0E0BD01ACE0B0E00E942DDC47
:10B68A00DB01AE0FBF1F1996AC91A13088F0AEEA6C
:10B69A00B7E0E091AC07F0E0BD01ACE0B0E00E9499
:10B6AA002DDCDB01AE0FBF1F1996EC91E150AFC044
:10B6BA00A091AB07A230B1F5AEEAB7E0E091AC07D2
:10B6CA00F0E0BD01ACE0B0E00E942DDCDB01AE0F82
:10B6DA00BF1F1996E9E0EC935A933A93A12F3ADBEC
:10B6EA005A93AEEAB7E0E091AC07F0E0BD01ACE0F6
:10B6FA00B0E00E942DDCDB01AE0FBF1F1896EC9163
:10B70A00EA93AEEAB7E0E091AC07F0E0BD01ACE045
:10B71A00B0E00E942DDCDB01AE0FBF1F1796AC9183
:10B72A0096DB76C0AEEAB7E0E091AC07F0E0BD0187
:10B73A00ACE0B0E00E942DDCDB01AE0FBF1F199612
:10B74A00EAE0EC93AEEAB7E0E091AC07F0E0BD01C5
:10B75A00ACE0B0E00E942DDCDB01AE0FBF1F1496F7
:10B76A00AC91A11790F1AEEAB7E0E091AC07F0E036
:10B77A00BD01ACE0B0E00E942DDCDB01AE0FBF1FC3
:10B78A001496E0E0EC935A93AEEAB7E0E091AC0786
:10B79A00F0E0BD01ACE0B0E00E942DDCDB01AE0FB1
:10B7AA00BF1F1896EC91EA93AEEAB7E0E091AC07B6
:10B7BA00F0E0BD01ACE0B0E00E942DDCDB01AE0F91
:10B7CA00BF1F1796AC9164DB23C0AEEAB7E0E091E5
:10B7DA00AC07F0E0BD01ACE0B0E00E942DDCE60F62
:10B7EA00F71F04815A930A93A02FA30F77DAAEEAC0
:10B7FA00B7E0E091AC07F0E0BD01ACE0B0E00E9438
:10B80A002DDCDB01AE0FBF1F1496EC91EF5FEC93BA
:10B81A000E947FDB689608950E947ADBECEAF7E0E3
:10B82A00FA93EA93E0E0EA93A9E6B0E00E9477D4BB
:10B83A00AAE7B8E00E9447DDE093AD07ABE7B8E0BE
:10B84A000E9447DDE093D50710E0123008F0A2C04D
:10B85A00ACE7B8E0E12FF0E0BD01AAE0B0E00E9459
:10B86A002DDCDB01AE0FBF1F0E9443DD9F01ADEA55
:10B87A00B7E0E12FF0E0BD01A8E2B0E00E942DDCC4
:10B88A00E60FF71F3496FF93EF93ACE7B8E0E12F8A
:10B89A00F0E0BD01AAE0B0E00E942DDCDB01AE0FB2
:10B8AA00BF1F12960E9447DDAF91BF91EC93ADEA9C
:10B8BA00B7E0E12FF0E0BD01A8E2B0E00E942DDC84
:10B8CA00E60FF71F3596FF93EF93ACE7B8E0E12F49
:10B8DA00F0E0BD01AAE0B0E00E942DDCDB01AE0F72
:10B8EA00BF1F16960E9447DDAF91BF91EC93ADEA58
:10B8FA00B7E0E12FF0E0BD01A8E2B0E00E942DDC44
:10B90A00E60FF71F2787308BADEAB7E0E12FF0E0AB
:10B91A00BD01A8E2B0E00E942DDCDB01AE0FBF1F23
:10B92A001E96EC91E07FE460EC93ADEAB7E0E12F7C
:10B93A00F0E0BD01A8E2B0E00E942DDCDB01AE0F11
:10B94A00BF1F1196F9013196ED93FC93ADEAB7E06A
:10B95A00E12FF0E0BD01A8E2B0E00E942DDCDB019E
:10B96A00AE0FBF1F5C96F9013496ED93FC93ADEAD6
:10B97A00B7E0E12FF0E0BD01A8E2B0E00E942DDCC3
:10B98A00DB01AE0FBF1F5B96EC91E07FE860EC93A2
:10B99A001F5F5BCFA0E9B8E00E9447DDE093B507DF
:10B9AA00A1E9B8E00E9447DDE093B807A2E9B8E050
:10B9BA000E9447DDE093DD07A3E9B8E00E9447DD76
:10B9CA00E093E00710E01831A0F500E0A4E9B8E040
:10B9DA00E12FF0E00E94F6DBAE0FBF1F11960E9426
:10B9EA0047DDE03009F001E0A4E9B8E0E12FF0E03A
:10B9FA000E94F6DBAE0FBF1F12960E9447DDE030B1
:10BA0A0009F00260A4E9B8E0E12FF0E00E94F6DB59
:10BA1A00AE0FBF1F13960E9447DDE03009F00460A5
:10BA2A00ADEFB7E0E12FF0E0EA0FFB1F00831F5FE5
:10BA3A00CACF0E9481DB24960895BA93AA930E94E2
:10BA4A0078DB10E0123008F0CDC0ADEAB7E0E12FA4
:10BA5A00F0E0BD01A8E2B0E00E942DDCDB01AE0FF0
:10BA6A00BF1FEC91E030B1F0ADEAB7E0E12FF0E0B2
:10BA7A00BD01A8E2B0E00E942DDCE60FF71F0180AD
:10BA8A001280AE81BF811196ED91FC911197E0155C
:10BA9A00F10509F0A5C0EE81FF810581ADEAB7E0A5
:10BAAA00E12FF0E0BD01A8E2B0E00E942DDCE60F34
:10BABA00F71F2681ADEAB7E0E12FF0E0BD01A8E269
:10BACA00B0E00E942DDCE60FF71F5085ADEAB7E023
:10BADA00E12FF0E0BD01A8E2B0E00E942DDCE60F04
:10BAEA00F71F37812523A02FA523EFEFE327EA23AA
:10BAFA002E27E52FE095E0232E2BADEAB7E0E12FC4
:10BB0A00F0E0BD01A8E2B0E00E942DDCE60FF71FCD
:10BB1A002683ADEAB7E0E12FF0E0BD01A8E2B0E08C
:10BB2A000E942DDCE60FF71F0783EE81FF81E68175
:10BB3A00EF700E2FADEAB7E0E12FF0E0BD01A8E209
:10BB4A00B0E00E942DDCE60FF71F2185ADEAB7E0D1
:10BB5A00E12FF0E0BD01A8E2B0E00E942DDCE60F83
:10BB6A00F71F5385ADEAB7E0E12FF0E0BD01A8E287
:10BB7A00B0E00E942DDCE60FF71F32852523A02FA7
:10BB8A00A523EFEFE327EA232E27E52FE095E0230D
:10BB9A002E2BADEAB7E0E12FF0E0BD01A8E2B0E05C
:10BBAA000E942DDCE60FF71F2187ADEAB7E0E12FEF
:10BBBA00F0E0BD01A8E2B0E00E942DDCE60FF71F1D
:10BBCA000287ADEAB7E0E12FF0E0BD01A8E2B0E0FC
:10BBDA000E942DDCDB01AE0FBF1F1396EAE0EC9347
:10BBEA001F5F30CF0E947FDB2896089524970E941A
:10BBFA0078DBE0916304E07409F4BCC3A091AC075C
:10BC0A00A43038F4E091AC07EF5FE093AC07E15061
:10BC1A0003C0E0E0E093AC07A091AC07A23008F0C3
:10BC2A00A9C3ADEAB7E0E091AC07F0E0BD01A8E234
:10BC3A00B0E00E942DDCDB01AE0FBF1FEC91E030BB
:10BC4A0009F498C3ADEAB7E0E091AC07F0E0BD01B2
:10BC5A00A8E2B0E00E942DDCDB01AE0FBF1F1396F5
:10BC6A00AC91A13008F463C0ADEAB7E0E091AC074B
:10BC7A00F0E0BD01A8E2B0E00E942DDCDB01AE0FCE
:10BC8A00BF1F1396EC91E150EC93ADEAB7E0E09157
:10BC9A00AC07F0E0BD01A8E2B0E00E942DDCDB01B8
:10BCAA00AE0FBF1F1396EC91E03009F040C0ADEA29
:10BCBA00B7E0E091AC07F0E0BD01A8E2B0E00E9475
:10BCCA002DDCDB01AE0FBF1F1696E0E0EC93ADEA68
:10BCDA00B7E0E091AC07F0E0BD01A8E2B0E00E9455
:10BCEA002DDCDB01AE0FBF1F1796E0E0EC93ADEA47
:10BCFA00B7E0E091AC07F0E0BD01A8E2B0E00E9435
:10BD0A002DDCDB01AE0FBF1F1996E0E0EC93ADEA24
:10BD1A00B7E0E091AC07F0E0BD01A8E2B0E00E9414
:10BD2A002DDCDB01AE0FBF1F1A96E0E0EC93E0E0DA
:10BD3A002E2F3E2FE091AC07E03011F450E001C005
:10BD4A005CE040E011E0103009F47DC0ADEFB7E0EF
:10BD5A00EE27A50FBE1F0C9102FF10C0A4E9B8E0A0
:10BD6A00E52FF0E00E94F6DBAE0FBF1F13960E948C
:10BD7A0047DDAE2F0E940465E03009F40EC0A4E945
:10BD8A00B8E0E52FF0E00E94F6DBAE0FBF1F0E947D
:10BD9A0047DDE295E370EE8343C001FF10C0A4E9DA
:10BDAA00B8E0E52FF0E00E94F6DBAE0FBF1F129657
:10BDBA000E9447DDAE2F0E94E03DE03009F40FC03B
:10BDCA00A4E9B8E0E52FF0E00E94F6DBAE0FBF1F52
:10BDDA000E9447DDE695E695E370EE8321C000FFF9
:10BDEA0010C0A4E9B8E0E52FF0E00E94F6DBAE0F40
:10BDFA00BF1F11960E9447DDAE2F0E94E03DE03042
:10BE0A0009F40DC0A4E9B8E0E52FF0E00E94F6DBE2
:10BE1A00AE0FBF1F0E9447DDE370EE8301C010C062
:10BE2A00EE81F0E0309711F4312B0AC0E130A0E046
:10BE3A00FA0729F0E230A0E0FA0711F4312B212B9E
:10BE4A005F5F110F80CFADEAB7E0E091AC07F0E099
:10BE5A00BD01A8E2B0E00E942DDCE60FF71FA0A109
:10BE6A003A1771F0ADEAB7E0E091AC07F0E0BD0136
:10BE7A00A8E2B0E00E942DDCE60FF71F30A341E0F4
:10BE8A00ADEAB7E0E091AC07F0E0BD01A8E2B0E0AE
:10BE9A000E942DDCE60FF71FA2A12A1771F0ADEA66
:10BEAA00B7E0E091AC07F0E0BD01A8E2B0E00E9483
:10BEBA002DDCE60FF71F22A341E0E0E02E2F3E2FF4
:10BECA0011E0103109F47DC0ADEFB7E0EE27A50F00
:10BEDA00BE1F0C9102FF10C0A4E9B8E0E52FF0E004
:10BEEA000E94F6DBAE0FBF1F13960E9447DDAE2FEE
:10BEFA000E940465E03009F40EC0A4E9B8E0E52F19
:10BF0A00F0E00E94F6DBAE0FBF1F0E9447DDE2950C
:10BF1A00E370EE8343C001FF10C0A4E9B8E0E52F47
:10BF2A00F0E00E94F6DBAE0FBF1F12960E9447DDBB
:10BF3A00AE2F0E94E03DE03009F40FC0A4E9B8E05A
:10BF4A00E52FF0E00E94F6DBAE0FBF1F0E9447DD2F
:10BF5A00E695E695E370EE8321C000FF10C0A4E9E0
:10BF6A00B8E0E52FF0E00E94F6DBAE0FBF1F119696
:10BF7A000E9447DDAE2F0E94E03DE03009F40DC07B
:10BF8A00A4E9B8E0E52FF0E00E94F6DBAE0FBF1F90
:10BF9A000E9447DDE370EE8301C010C0EE81F0E03D
:10BFAA00309711F4312B0AC0E130A0E0FA0729F0EA
:10BFBA00E230A0E0FA0711F4312B212B5F5F110F59
:10BFCA0080CFADEAB7E0E091AC07F0E0BD01A8E2AE
:10BFDA00B0E00E942DDCE60FF71FA1A13A1771F01D
:10BFEA00ADEAB7E0E091AC07F0E0BD01A8E2B0E04D
:10BFFA000E942DDCE60FF71F31A341E0ADEAB7E05E
:10C00A00E091AC07F0E0BD01A8E2B0E00E942DDCAF
:10C01A00E60FF71FA3A12A1771F0ADEAB7E0E09186
:10C02A00AC07F0E0BD01A8E2B0E00E942DDCE60F0B
:10C03A00F71F23A341E0403089F4ADEAB7E0E0916D
:10C04A00AC07F0E0BD01A8E2B0E00E942DDCDB0104
:10C05A00AE0FBF1F1D96AC91A13008F412C0ADEA15
:10C06A00B7E0E091AC07F0E0BD01A8E2B0E00E94C1
:10C07A002DDCDB01AE0FBF1F1D96EC91E150EC9356
:10C08A0020C0ADEAB7E0E091AC07F0E0BD01A8E25C
:10C09A00B0E00E942DDCDB01AE0FBF1F1D96E0E170
:10C0AA00EC93ADEAB7E0E091AC07F0E0BD01A8E29D
:10C0BA00B0E00E942DDCDB01AE0FBF1F5B960E9431
:10C0CA00B109ADEAB7E0E091AC07F0E0BD01A8E242
:10C0DA00B0E00E942DDCDB01AE0FBF1F1496AC91BD
:10C0EA00A03091F4ADEAB7E0E091AC07F0E0BD0111
:10C0FA00A8E2B0E00E942DDCDB01AE0FBF1F15964F
:10C10A00AC91A03009F436C140E0E1E0E987EFE004
:10C11A00E887EF83ADEAB7E0E091AC07F0E0BD0154
:10C12A00A8E2B0E00E942DDCDB01AE0FBF1F15961E
:10C13A00AC910E94E03DE03089F1ACE7B8E0E091D3
:10C14A00AC07F0E0BD01AAE0B0E00E942DDCDB0103
:10C15A00AE0FBF1F17960E9447DDE987ACE7B8E02C
:10C16A00E091AC07F0E0BD01AAE0B0E00E942DDC4E
:10C17A00DB01AE0FBF1F18960E9447DDE887ACE7C8
:10C18A00B8E0E091AC07F0E0BD01AAE0B0E00E949F
:10C19A002DDCDB01AE0FBF1F199643C0ADEAB7E035
:10C1AA00E091AC07F0E0BD01A8E2B0E00E942DDC0E
:10C1BA00DB01AE0FBF1F1496AC910E94E03DE03048
:10C1CA0099F1ACE7B8E0E091AC07F0E0BD01AAE074
:10C1DA00B0E00E942DDCDB01AE0FBF1F13960E9458
:10C1EA0047DDE987ACE7B8E0E091AC07F0E0BD01D4
:10C1FA00AAE0B0E00E942DDCDB01AE0FBF1F14964F
:10C20A000E9447DDE887ACE7B8E0E091AC07F0E0D0
:10C21A00BD01AAE0B0E00E942DDCDB01AE0FBF1F1A
:10C22A0015960E9447DDEF83ADEAB7E0E091AC07CF
:10C23A00F0E0BD01A8E2B0E00E942DDCE60FF71F96
:10C24A00A489E985EA1781F0ADEAB7E0E091AC0785
:10C25A00F0E0BD01A8E2B0E00E942DDCE60FF71F76
:10C26A007496A985A08341E0ADEAB7E0E091AC07F6
:10C27A00F0E0BD01A8E2B0E00E942DDCE60FF71F56
:10C28A00A589E885EA1781F0ADEAB7E0E091AC0745
:10C29A00F0E0BD01A8E2B0E00E942DDCE60FF71F36
:10C2AA007596A885A08341E0ADEAB7E0E091AC07B6
:10C2BA00F0E0BD01A8E2B0E00E942DDCE60FF71F16
:10C2CA00A689EF81EA1781F0ADEAB7E0E091AC0701
:10C2DA00F0E0BD01A8E2B0E00E942DDCE60FF71FF6
:10C2EA007696AF81A08341E0403089F4ADEAB7E0A9
:10C2FA00E091AC07F0E0BD01A8E2B0E00E942DDCBD
:10C30A00DB01AE0FBF1F1C96AC91A13008F412C01E
:10C31A00ADEAB7E0E091AC07F0E0BD01A8E2B0E019
:10C32A000E942DDCDB01AE0FBF1F1C96EC91E15081
:10C33A00EC9320C0ADEAB7E0E091AC07F0E0BD01B4
:10C34A00A8E2B0E00E942DDCDB01AE0FBF1F1C96F5
:10C35A00E0E1EC93ADEAB7E0E091AC07F0E0BD01B3
:10C36A00A8E2B0E00E942DDCDB01AE0FBF1F1E96D3
:10C37A000E94B1090E947FDB2A96089508951A93B4
:10C38A001A2FA9E01A9FF001E15EF64FA081A73BA0
:10C39A0021F4A12F0E94279030C31730D0F4103017
:10C3AA0011F4139815C0113011F4769811C0123097
:10C3BA0011F42C980DC0133011F4109809C01430E0
:10C3CA0011F4179805C0153011F4A39801C02F98DD
:10C3DA003DC01D30B0F4173011F4169811C0183052
:10C3EA0011F411980DC0193011F48E9809C01A3041
:10C3FA0011F48C9805C01B3011F42D9801C02E98A9
:10C40A0025C0123190F41D3011F474980DC01E30FD
:10C41A0011F4759809C01F3011F4A49805C01031A1
:10C42A0011F4729801C0739811C0163170F4123168
:10C43A0011F4149809C0133111F45F9805C014312E
:10C44A0011F48D9801C0129801C01598D6C21A939A
:10C45A001A2F1730D0F4103011F4139A15C0113076
:10C46A0011F4769A11C0123011F42C9A0DC01330BF
:10C47A0011F4109A09C0143011F4179A05C0153036
:10C48A0011F4A39A01C02F9AA7C01D30B0F4173037
:10C49A0011F4169A11C0183011F4119A0DC01930FE
:10C4AA0011F48E9A09C01A3011F48C9A05C01B3007
:10C4BA0011F42D9A01C02E9A8FC0123190F41D30BA
:10C4CA0011F4749A0DC01E3011F4759A09C01F3008
:10C4DA0011F4A49A05C0103111F4729A01C0739A2A
:10C4EA007BC0173190F4123111F4149A0DC0133134
:10C4FA0011F45F9A09C0143111F48D9A05C01531EF
:10C50A0011F4129A01C0159A67C01F3198F51731B4
:10C51A0021F4E0910E09E16027C0183121F4E0917D
:10C52A000E09E26021C0193121F4E0910E09E4609C
:10C53A001BC01A3121F4E0910E09E86015C01B31C5
:10C54A0021F4E0910E09E0680FC01C3121F4E0915A
:10C55A000E09E06409C01D3121F4E0910E09E06280
:10C56A0003C0E0910E09E061E0930E09E8E0E09370
:10C57A00080932C01F3121F4E0910D09E06827C093
:10C58A00103221F4E0910D09E06421C0113221F446
:10C59A00E0910D09E0621BC0123221F4E0910D090D
:10C5AA00E06115C0133221F4E0910D09E1600FC07A
:10C5BA00143221F4E0910D09E26009C0153221F428
:10C5CA00E0910D09E46003C0E0910D09E860E09391
:10C5DA000D09E8E0E093070910C21A931A2F1730E1
:10C5EA00D0F4103011F4139815C0113011F4769864
:10C5FA0011C0123011F42C980DC0133011F4109898
:10C60A0009C0143011F4179805C0153011F4A39815
:10C61A0001C02F98A7C01D30B0F4173011F4169836
:10C62A0011C0183011F411980DC0193011F48E98F8
:10C63A0009C01A3011F48C9805C01B3011F42D98DA
:10C64A0001C02E988FC0123190F41D3011F47498E5
:10C65A000DC01E3011F4759809C01F3011F4A4984A
:10C66A0005C0103111F4729801C073987BC017315C
:10C67A0090F4123111F414980DC0133111F45F982B
:10C68A0009C0143111F48D9805C0153111F41298AE
:10C69A0001C0159867C01F3198F5173121F4E09150
:10C6AA000E09EE7F27C0183121F4E0910E09ED7FC3
:10C6BA0021C0193121F4E0910E09EB7F1BC01A3118
:10C6CA0021F4E0910E09E77F15C01B3121F4E091B6
:10C6DA000E09EF770FC01C3121F4E0910E09EF7BB0
:10C6EA0009C01D3121F4E0910E09EF7D03C0E091EC
:10C6FA000E09EF7EE0930E09E8E0E093080932C0E4
:10C70A001F3121F4E0910D09EF7727C0103221F48F
:10C71A00E0910D09EF7B21C0113221F4E0910D095E
:10C72A00EF7D1BC0123221F4E0910D09EF7E15C096
:10C73A00133221F4E0910D09EE7F0FC0143221F477
:10C74A00E0910D09ED7F09C0153221F4E0910D0940
:10C75A00EB7F03C0E0910D09E77FE0930D09E8E064
:10C76A00E09307094AC11A931A2FEEE7F5E060E051
:10C77A0070E00E9405DDE12FFF27662777270E94D8
:10C78A0005DD84E00E94FFDA2896E12FF0E0E2302E
:10C79A00A0E0FA0749F4E0911209E061E093120976
:10C7AA00E0911109EF7E9AC0E330A0E0FA0749F45C
:10C7BA00E0911209E460E0931209E0911109EB7F1C
:10C7CA008DC0E430A0E0FA0749F4E0911209E06272
:10C7DA00E0931209E0911109EF7D80C0E530A0E0F5
:10C7EA00FA0749F4E0911209E068E0931209E0912E
:10C7FA001109EF7773C0EB30A0E0FA0771F4E0910A
:10C80A001009E160E0931009E0910F09EE7FE093CF
:10C81A000F09E0E0E093090966C0EC30A0E0FA07EE
:10C82A0049F4E0911209E860E0931209E0911109D4
:10C83A00E77F54C0ED30A0E0FA0771F4E0911009E7
:10C84A00E460E0931009E0910F09EB7FE0930F0990
:10C85A00E0E0E093090947C0EE30A0E0FA0771F47E
:10C86A00E0911009E260E0931009E0910F09ED7F71
:10C87A00E0930F09E0E0E093090935C0E031A0E058
:10C88A00FA0771F4E0911009E061E0931009E09170
:10C89A000F09EF7EE0930F09E0E0E093090923C056
:10C8AA00E131A0E0FA0771F4E0911009E860E09341
:10C8BA001009E0910F09E77FE0930F09E0E0E093A8
:10C8CA00090911C0E631A0E0FA0769F4E0911209FA
:10C8DA00E064E0931209E0911109EF7BE0931109FA
:10C8EA00E0E0E0930A0989C01A931A2FEFE8F5E00D
:10C8FA0060E070E00E9405DDE12FFF2766277727B9
:10C90A000E9405DD84E00E94FFDA2896E12FF0E01C
:10C91A00E230A0E0FA0721F4E0911109E06168C071
:10C92A00E330A0E0FA0721F4E0911109E46060C065
:10C93A00E430A0E0FA0721F4E0911109E06258C05E
:10C94A00E530A0E0FA0721F4E0911109E06850C04F
:10C95A00EB30A0E0FA0749F4E0910F09E160E093B7
:10C96A000F09E0E0E093090948C0EC30A0E0FA07BB
:10C97A0021F4E0911109E8603BC0ED30A0E0FA072C
:10C98A0049F4E0910F09E460E0930F09E0E0E093D5
:10C99A00090933C0EE30A0E0FA0749F4E0910F0923
:10C9AA00E260E0930F09E0E0E093090926C0E03174
:10C9BA00A0E0FA0749F4E0910F09E061E0930F095A
:10C9CA00E0E0E093090919C0E131A0E0FA0749F46F
:10C9DA00E0910F09E860E0930F09E0E0E0930909AC
:10C9EA000CC0E631A0E0FA0741F4E0911109E064D5
:10C9FA00E0931109E0E0E0930A09199108950E9471
:10CA0A007ADB3A2F3F3010F0363208F01FC0E32F9E
:10CA1A00EF501E2FA9E01A9FF001E45EF64FE08165
:10CA2A00E47011F0E1E054C3A9E01A9FF001E45E5A
:10CA3A00F64FE081E295E7700E2F013021F00430C5
:10CA4A0011F0053011F4E1E043C319C0363210F099
:10CA5A00363308F014C0E32FE6521E2FA3E01A9FC4
:10CA6A00F001E551F64FE081E295E7700E2F0130B3
:10CA7A0021F0043011F0053011F4E1E029C3A32FAD
:10CA8A000E94798825C30E947ADBE0911409EF7E1F
:10CA9A00E0931409EF7DE0931409E4E1E0931809A7
:10CAAA00E0911409EF7BE0931409E0911509EE7FF8
:10CABA00E0931509ED7FE0931509ECE1F9E0FA93AB
:10CACA00EA93E0E0EA93AFECB0E00E9477D46E9A82
:10CADA00089A6A9A6B9A0C9A579A0D9A10E017312B
:10CAEA0008F018C1A9E01A9FF001E15EF64FFF9322
:10CAFA00EF93A5E4B1E0E12FF0E0BD01A7E0B0E0DB
:10CB0A000E942DDCDB01AE0FBF1F0E9447DDAF91F3
:10CB1A00BF91EC93A9E01A9FF001E45EF64FFF93F0
:10CB2A00EF93A5E4B1E0E12FF0E0BD01A7E0B0E0AA
:10CB3A000E942DDCDB01AE0FBF1F12960E9447DD5B
:10CB4A00E07121F5A5E4B1E0E12FF0E0BD01A7E035
:10CB5A00B0E00E942DDCDB01AE0FBF1F12960E94CF
:10CB6A0047DDE07299F4A5E4B1E0E12FF0E0BD0100
:10CB7A00A7E0B0E00E942DDCDB01AE0FBF1F1296CA
:10CB8A000E9447DDE07411F4E0E001C0E1E0AF91FA
:10CB9A00BF91E170EE0F0E2EEC91ED7FE029EC9340
:10CBAA00A5E4B1E0E12FF0E0BD01A7E0B0E00E940A
:10CBBA002DDCDB01AE0FBF1F15960E9447DDE07228
:10CBCA0049F0A9E01A9FF001E35EF64FDF01EC910C
:10CBDA00E061EC93A5E4B1E0E12FF0E0BD01A7E04C
:10CBEA00B0E00E942DDCDB01AE0FBF1F15960E943C
:10CBFA0047DDE07449F0A9E01A9FF001E35EF64FC1
:10CC0A00DF01EC91E062EC93A5E4B1E0E12FF0E002
:10CC1A00BD01A7E0B0E00E942DDCDB01AE0FBF1F13
:10CC2A0012960E9447DDE07829F0E0911409E0614C
:10CC3A00E0931409A8EBB9E0E12FF0E0F595E79548
:10CC4A00AE0FBF1F0E9447DD0E2F10FF0DC0E02F51
:10CC5A00E07F49F0A9E01A9FF001E45EF64FDF0198
:10CC6A00EC91E068EC930CC0E02FEF7049F0A9E07A
:10CC7A001A9FF001E45EF64FDF01EC91E068EC9355
:10CC8A00A9E01A9FF001E15EF64FA081A63309F0F0
:10CC9A003FC0E12FFF2766277727EC52FF4F6F4FE0
:10CCAA006BBF36913731A0F5A9E03A9FF001E35EF8
:10CCBA00F64FDF01EC91E064EC93E12FF0E0E13014
:10CCCA00A0E0FA0711F46E9823C0E330A0E0FA0757
:10CCDA0011F408981DC0E031A0E0FA0711F46A982F
:10CCEA0017C0E131A0E0FA0711F46B9811C0E231E4
:10CCFA00A0E0FA0711F40C980BC0E331A0E0FA07A0
:10CD0A0011F4579805C0E631A0E0FA0709F40D9826
:10CD1A001F5FE5CEEBEEF9E0FA93EA93E0E0EA93DF
:10CD2A00A0E3B0E00E9477D410E0103108F08CC084
:10CD3A00A3E01A9FF001E351F64F0F01A6EEB1E00E
:10CD4A00E12FF0E0EE0FFF1FAE0FBF1F0E9447DD7D
:10CD5A00D001EC93A3E01A9FF001E551F64F0F01C1
:10CD6A00A6EEB1E0E12FF0E0EE0FFF1FAE0FBF1FFE
:10CD7A0011960E9447DDE170E1F4A6EEB1E0E12FE1
:10CD8A00F0E0EE0FFF1FAE0FBF1F11960E9447DDA6
:10CD9A00E27079F4A6EEB1E0E12FF0E0EE0FFF1FAA
:10CDAA00AE0FBF1F11960E9447DDE47011F4E0E058
:10CDBA0001C0E1E0D001E170EE0F0E2EEC91ED7FA3
:10CDCA00E029EC93A6EEB1E0E12FF0E0EE0FFF1FB1
:10CDDA00AE0FBF1F11960E9447DDE87069F0A0915F
:10CDEA00220EA33420F0E0911409E06203C0E0911E
:10CDFA001409E061E0931409A4ECB9E0E12FF0E032
:10CE0A00F595E795AE0FBF1F0E9447DD0E2F10FF65
:10CE1A000DC0E02FE07F49F0A3E01A9FF001E55131
:10CE2A00F64FDF01EC91E068EC930CC0E02FEF7055
:10CE3A0049F0A3E01A9FF001E551F64FDF01EC91AA
:10CE4A00E068EC931F5F71CFA2E1B9E0E0911409A9
:10CE5A00E295E1700E2EEC91EE7FE029EC93ABE0C7
:10CE6A00B9E0E0911409E295EF70E695E170E29578
:10CE7A00E07FEE0FEE0F0E2EEC91EF7BE029EC93A4
:10CE8A00E0911009E07EE0931009E0919209E074C4
:10CE9A0081F0A4EAB1E00E9443DDDF01EEE00E94E6
:10CEAA00B3DBE17029F0E0911009E061E093100929
:10CEBA000FC0A9EBB1E00E9443DDDF01EEE00E9462
:10CECA00B3DBE17029F0E0911009E061E093100909
:10CEDA00E0918009E07481F0A6E9B1E00E9443DDA7
:10CEEA00DF01EEE00E94B3DBE17029F0E091100966
:10CEFA00E860E09310090FC0A0ECB1E00E9443DDA6
:10CF0A00DF01EEE00E94B3DBE17029F0E091100945
:10CF1A00E860E0931009A4EAB1E00E9443DDDF0172
:10CF2A00EEE00E94B3DBE17029F0E0911009E460C1
:10CF3A00E0931009E0913809E07481F0AEE5B1E0C0
:10CF4A000E9443DDDF01EEE00E94B3DBE17029F0CD
:10CF5A00E0911009E260E09310090FC0ABEAB1E07A
:10CF6A000E9443DDDF01EEE00E94B3DBE17029F0AD
:10CF7A00E0911009E260E0931009A6E9B1E00E948D
:10CF8A0043DDDF01EEE00E94B3DBE17029F0E091BE
:10CF9A001009E160E0931009E0910F09E07EE09347
:10CFAA000F09A0910F09E0911009E095EF71EA2BA2
:10CFBA00E0930F09E0E0E0930909E0911209E370B8
:10CFCA00E0931209ACE6B1E00E9443DDDF01EEE036
:10CFDA000E94B3DBE17029F0E0911209E068E09366
:10CFEA001209E0918909E07481F0ADE9B1E00E948B
:10CFFA0043DDDF01EEE00E94B3DBE17029F0E0914E
:10D00A001209E064E09312090FC0A3EEB1E00E9496
:10D01A0043DDDF01EEE00E94B3DBE17029F0E0912D
:10D02A001209E064E0931209A5E6B1E00E9443DD2B
:10D03A00DF01EEE00E94B3DBE17029F0E091120912
:10D04A00E062E0931209E0912609E07451F4A7E541
:10D05A00B1E00E9443DDDF01EEE00E94B3DBE17044
:10D06A0009F405C0E0911209E061E0931209ADE903
:10D07A00B1E00E9443DDDF01EEE00E94B3DBE17024
:10D08A0029F0E0911209E860E0931209AEE5B1E0F7
:10D09A000E9443DDDF01EEE00E94B3DBE17029F07C
:10D0AA00E0911209E460E0931209E0911109E3703A
:10D0BA00E0931109A0911109E0911209E095EC7F22
:10D0CA00EA2BE0931109E0E0E0930609E0930A09EC
:10D0DA000E9481DB2496089527970E9478DBE091CD
:10D0EA001609EF73E73160F1E0911209EE7FE093E0
:10D0FA001209E0910B09EF7BE0930B09E0E0E09362
:10D10A000609E0930A09E0911609E07CE093160902
:10D11A00E0911309E770E063E0931309E0E0E2B9F4
:10D12A00E5B1EF70E5B95F98EEB1E378EEB9E1B336
:10D13A00EF78E1BBE4B3E77EE4BBA0E088D9C9C2DB
:10D14A00E0911309E87FE83008F4C3C2A3E1B9E02B
:10D15A0083E0EFE10E9439DDE0911309E87FE830CE
:10D16A00D1F4A1E4B8E0E0911609EF73FF2766272E
:10D17A007727EC5FFE4F6F4F6BBFE691F0E0EE0F43
:10D18A00FF1FAE0FBF1FED91FC911197E0931A0993
:10D19A00F0931B099EC2E0911309E87F09F099C236
:10D1AA00A1E4B8E0E0911609EF73FF276627772715
:10D1BA00EC5FFE4F6F4F6BBFE691F0E0EE0FFF1F83
:10D1CA00AE0FBF1FED91FD91A0911A09B0911B09F5
:10D1DA00EA0FFB1FE0931A09F0931B09A0911A09A1
:10D1EA00B0911B09E0911B09F070EA0FFB1FE09355
:10D1FA001A09F0931B090E9408DCE0931A09F093BC
:10D20A001B09E0911309F0E0E770F070E230A0E04A
:10D21A00FA07E1F5A2E3B0E0E0911609EF73F0E056
:10D22A00BD01AAE0B0E00E942DDCDB01AE0FBF1FFA
:10D23A00E0911A09F0911B090E945BDDE091160941
:10D24A00EF73FF2766277727E45EFE4F6F4F6BBFAA
:10D25A00E691E03061F4EAEAF1E060E070E00E9411
:10D26A00F0DC9F01E8EDF1E060E070E00BC0E6E081
:10D27A00F2E060E070E00E94F0DC9F01E4E3F2E09B
:10D28A0060E070E00E94F0DCAF0103C1E330A0E08F
:10D29A00FA07E9F5A2E3B0E0E0911609EF73F0E0CE
:10D2AA00BD01AAE0B0E00E942DDCDB01AE0FBF1F7A
:10D2BA001296E0911A09F0911B090E945BDDE09138
:10D2CA001609EF73FF2766277727E45EFE4F6F4F35
:10D2DA006BBFE691E03061F4ECEAF1E060E070E007
:10D2EA000E94F0DC9F01EAEDF1E060E070E00BC023
:10D2FA00E8E0F2E060E070E00E94F0DC9F01E6E323
:10D30A00F2E060E070E00E94F0DCAF01C2C0E430FD
:10D31A00A0E0FA07E9F5A2E3B0E0E0911609EF739D
:10D32A00F0E0BD01AAE0B0E00E942DDCDB01AE0F07
:10D33A00BF1F1496E0911A09F0911B090E945BDD48
:10D34A00E0911609EF73FF2766277727E45EFE4F01
:10D35A006F4F6BBFE691E03061F4EEEAF1E060E016
:10D36A0070E00E94F0DC9F01ECEDF1E060E070E01B
:10D37A000BC0EAE0F2E060E070E00E94F0DC9F019E
:10D38A00E8E3F2E060E070E00E94F0DCAF0181C007
:10D39A00E530A0E0FA07E9F5A2E3B0E0E09116096A
:10D3AA00EF73F0E0BD01AAE0B0E00E942DDCDB01E2
:10D3BA00AE0FBF1F1696E0911A09F0911B090E9441
:10D3CA005BDDE0911609EF73FF2766277727E45E96
:10D3DA00FE4F6F4F6BBFE691E03061F4E0EBF1E096
:10D3EA0060E070E00E94F0DC9F01EEEDF1E060E0A9
:10D3FA0070E00BC0ECE0F2E060E070E00E94F0DC6C
:10D40A009F01EAE3F2E060E070E00E94F0DCAF0125
:10D41A0040C0E630A0E0FA07E1F5A2E3B0E0E0910F
:10D42A001609EF73F0E0BD01AAE0B0E00E942DDC1E
:10D43A00DB01AE0FBF1F1896E0911A09F0911B0984
:10D44A000E945BDDE0911609EF73FF2766277727B5
:10D45A00E45EFE4F6F4F6BBFE691E03061F4E2EBA2
:10D46A00F1E060E070E00E94F0DC9F01E0EEF1E0A4
:10D47A0060E070E00BC0EEE0F2E060E070E00E9475
:10D48A00F0DC9F01ECE3F2E060E070E00E94F0DC87
:10D49A00AF01E4EAF5E060E070E00E9405DDE091AA
:10D4AA001609EF73F0E031966F2F660F660B762F31
:10D4BA000E9405DDE0911A09F0911B09662777277A
:10D4CA000E9405DD88E00E94FFDA2C96A0911A09D5
:10D4DA00B0911B09A217B30718F04A175B0708F4A3
:10D4EA0002C011E013C010E0E0911709EC7771F463
:10D4FA00A7E1B9E0E0911609EF73EF5FEF71EE0F64
:10D50A00EE0F0E2EEC91E378E029EC93A12F0E9406
:10D51A00F7CBE7E0EF83E9EFE887E985E160E987A0
:10D52A00E12FE170EE0F0E2EE985ED7FE029E98704
:10D53A00E0911609EF73EF5FEF73EE0FEE0F0E2E09
:10D54A00E985E370E029E987E0911A09F0911B095E
:10D55A00EB87FC87E0911309F0E0E770F070E230A6
:10D56A00A0E0FA0711F4E1E019C0E330A0E0FA07FD
:10D57A0011F4E2E013C0E430A0E0FA0711F4E3E0AA
:10D58A000DC0E530A0E0FA0711F4E4E007C0E63088
:10D59A00A0E0FA0711F4E5E001C0E0E0EA87E0E084
:10D5AA00E2B9E5B1EF70E5B95F98EEB1E378EEB9AB
:10D5BA00E1B3EF78E1BBE4B3E77EE4BBDE011696A4
:10D5CA000E94CA9FE0911609EF73E63198F4A6E12A
:10D5DA00B9E080E0EFE30E9435DDE0911309E770DE
:10D5EA00E062E0931309E0911609EF73AE2F0E94EF
:10D5FA002C626FC0A2E2B0E00E9447DD1E2EE091CD
:10D60A001309E770E250A1E00E949ADBE129A2E245
:10D61A00B0E00E9463DDEFEAF5E060E070E00E94AE
:10D62A0005DD80E00E94FFDA2496E0911709EC7785
:10D63A0091F4EAEBF5E060E070E00E9405DD80E03D
:10D64A000E94FFDA2496E0911309E770E23011F4A0
:10D65A000E942A3914C0EEEBF5E060E070E00E9407
:10D66A0005DDE0911709E695E695EF71FF27662734
:10D67A0077270E9405DD84E00E94FFDA2896A2E15E
:10D68A00B9E0E0911409E295E1700E2EEC91EE7F7B
:10D69A00E029EC93ABE0B9E0E0911409E295EF7070
:10D6AA00E695E170E295E07FEE0FEE0F0E2EEC911B
:10D6BA00EF7BE029EC93E0E0E0930609E0930A09A6
:10D6CA00E0911309E87FE160E0931309E6E0E09353
:10D6DA00270E0E947FDB2D9608952F970E9478DBF4
:10D6EA00E0911609EF73E73260F1E0911609E07CE8
:10D6FA00E0931609E0911309E770E062E0931309D9
:10D70A00E0911209EE7FE0931209E0910B09EF7B99
:10D71A00E0930B09E0E0E0930609E0930A09E2B915
:10D72A00E5B1EF70E5B95F98EEB1E378EEB9E1B330
:10D73A00EF78E1BBE4B3E77EE4BBA0E00E942C6291
:10D74A00D0C2E0911309E87FE83008F4CAC2E09138
:10D75A001609EF730E2FA3E1B9E083E0EFE10E940F
:10D76A0039DDE0911309E87FE830D1F40731B8F4E4
:10D77A00A1E4B8E0E02FFF2766277727EC5FFE4F8A
:10D78A006F4F6BBFE691F0E0EE0FFF1FAE0FBF1FAA
:10D79A00ED91FC911197E0931A09F0931B09A1C22C
:10D7AA00E0911309E87F09F09CC2E7E0EF83E9EF13
:10D7BA00E887E6E0EA87E985E160E987E260E987E8
:10D7CA00E0911609EF73EF5FEF73EE0FEE0F0E2E77
:10D7DA00E985E370E029E987E0E0EB87EC87073128
:10D7EA0008F0ABC1A1E4B8E0E02FFF27662777274E
:10D7FA00EC5FFE4F6F4F6BBFE691F0E0EE0FFF1F3D
:10D80A00AE0FBF1FED91FD91A0911A09B0911B09AE
:10D81A00AE0FBF1FFD010E9408DC9F01A2E3B0E02A
:10D82A00E02FF0E0BD01AAE0B0E00E942DDCDB01B0
:10D83A00AE0FBF1F0E9443DDAF014217530718F016
:10D84A0020E030E0E1C0A2E3B0E0E02FF0E0BD016B
:10D85A00AAE0B0E00E942DDCDB01AE0FBF1F1296DA
:10D86A000E9443DDEB8BFC8BE217F30708F1241BC4
:10D87A00350BF901662777276E2F7F2FE0E0F0E05E
:10D88A007F936F93FF93EF93EB89FC89E41BF50B6E
:10D89A0066277727AFE8B2E080E090E00E9435DCA7
:10D8AA00AF91BF918F919F910E948BDC9F01ACC079
:10D8BA00A2E3B0E0E02FF0E0BD01AAE0B0E00E94F0
:10D8CA002DDCDB01AE0FBF1F14960E9443DDE98BEE
:10D8DA00FA8BE217F30730F1AB89BC892A1B3B0BA1
:10D8EA00D90188279927E1E10E94C4DB7F936F93CE
:10D8FA00FF93EF93AB89BC89E989FA89EA1BFB0B91
:10D90A0066277727AFE8B2E080E090E00E9435DC36
:10D91A00AF91BF918F919F910E948BDC9F012C59EF
:10D92A003F4F72C0A2E3B0E0E02FF0E0BD01AAE0F1
:10D93A00B0E00E942DDCDB01AE0FBF1F16960E94DD
:10D94A0043DDEF87F88BE217F30730F1A989BA892B
:10D95A002A1B3B0BD90188279927E1E10E94C4DBE6
:10D96A007F936F93FF93EF93A989BA89EF85F8891B
:10D97A00EA1BFB0B66277727A4EBB1E080E090E077
:10D98A000E9435DCAF91BF918F919F910E948BDCF1
:10D99A009F01245D3E4F38C0A2E3B0E0E02FF0E0E3
:10D9AA00BD01AAE0B0E00E942DDCDB01AE0FBF1F73
:10D9BA0018960E9443DDED87FE87AF85B8892A1B3A
:10D9CA003B0BD90188279927E3E10E94C4DB7F93A7
:10D9DA006F93FF93EF93AF85B889ED85FE85EA1BB8
:10D9EA00FB0BF695E79566277727ACEEB2E080E069
:10D9FA0090E00E9435DCAF91BF918F919F910E9478
:10DA0A008BDC9F01285A3D4FE3EDF5E060E070E0C2
:10DA1A000E9405DDE02FF0E031966F2F660F660B4E
:10DA2A00762F0E9405DDF901662777270E94E0DD3F
:10DA3A00DF01CB01E0E0F0E068EC72E40E94B7DEBF
:10DA4A000E9405DD88E00E94FFDA2C96F6982B8763
:10DA5A003C8710E0173108F06FC00117B1F5A5EA4D
:10DA6A00B8E0E12FFF2766277727E451FF4F6F4F72
:10DA7A006BBFE691F0E0AE0FBF1FEC91E07421F5A9
:10DA8A00E2EEF5E060E070E00E9405DDE02FF0E0F4
:10DA9A0031966F2F660F660B762F0E9405DDE12FF8
:10DAAA00F0E031966F2F660F660B762F0E9405DD28
:10DABA0088E00E94FFDA2C96E0911709E260E09371
:10DACA001709E985ED7FE98735C0A5EAB8E0E12FB6
:10DADA00FF2766277727E451FF4F6F4F6BBFE69109
:10DAEA00F0E0AE0FBF1FEC91E07421F1ECEFF5E02E
:10DAFA0060E070E00E9405DDE02FF0E031966F2FC4
:10DB0A00660F660B762F0E9405DDE12FF0E0319655
:10DB1A006F2F660F660B762F0E9405DD88E00E9444
:10DB2A00FFDA2C96E0911709E260E0931709E9857C
:10DB3A00ED7FE9871F5F8ECF78C0075110E0103163
:10DB4A0008F073C00117C1F5A5EAB8E0E12FFF2775
:10DB5A0066277727EE56FD4F6F4F6BBFE691F0E0D1
:10DB6A00AE0FBF1FEC91E07831F5E2EEF5E060E030
:10DB7A0070E00E9405DDE0911609EF73F0E031963E
:10DB8A006F2F660F660B762F0E9405DDE12FF0E0FE
:10DB9A0077966F2F660F660B762F0E9405DD88E059
:10DBAA000E94FFDA2C96E0911709E260E0931709C8
:10DBBA00E985ED7FE98737C0A5EAB8E0E12FFF27BD
:10DBCA0066277727EE56FD4F6F4F6BBFE691F0E061
:10DBDA00AE0FBF1FEC91E07831F1ECEFF5E060E0B9
:10DBEA0070E00E9405DDE0911609EF73F0E03196CE
:10DBFA006F2F660F660B762F0E9405DDE12FF0E08E
:10DC0A0077966F2F660F660B762F0E9405DD88E0E8
:10DC1A000E94FFDA2C96E0911709E260E093170957
:10DC2A00E985ED7FE9871F5F8ACFE0911609EF73D7
:10DC3A000E2FA02F0E94F262DE0116960E94CA9F42
:10DC4A00063298F4A6E1B9E080E0EFE30E9435DD00
:10DC5A00E0911609EF73AE2F0E942C62E09113092E
:10DC6A00E770E062E09313093CC0E9E1F6E060E0A6
:10DC7A0070E00E9405DD80E00E94FFDA2496E091C0
:10DC8A001709E695E170A0E0EA17E1E009F0EE274E
:10DC9A00AE2F0E94F7CBE0911309E87FE0931309B6
:10DCAA00A2E1B9E0E0911409E295E1700E2EEC913F
:10DCBA00EE7FE029EC93ABE0B9E0E0911409E2953C
:10DCCA00EF70E695E170E295E07FEE0FEE0F0E2E13
:10DCDA00EC91EF7BE029EC93E0E0E0930609E09316
:10DCEA000A090E947FDB6596089526970E9478DBD1
:10DCFA00E5E2F6E060E070E00E9405DDABE1B0E04D
:10DD0A000E9443DD662777270E9405DD84E00E9492
:10DD1A00FFDA2896ABE1B0E00E9443DDE03CA3E3E2
:10DD2A00FA0740F0ABE1B0E00E9443DDE134AFE333
:10DD3A00FA0708F002C021E001C020E0A22F0E94E9
:10DD4A00F7CBE6E3F6E060E070E00E9405DDADE1C6
:10DD5A00B0E00E9443DD662777270E9405DDAFE128
:10DD6A00B0E00E9443DD662777270E9405DD88E040
:10DD7A000E94FFDA2C96ADE1B0E00E9443DDE53A5D
:10DD8A00A7E1FA07C0F0ADE1B0E00E9443DDE73E4B
:10DD9A00ACE1FA0780F4AFE1B0E00E9443DDE53A76
:10DDAA00A7E1FA0740F0AFE1B0E00E9443DDE73EA9
:10DDBA00ACE1FA0708F002C051E001C050E0A52F1B
:10DDCA000E94F7CBEFE4F6E060E070E00E9405DD28
:10DDDA00A2E2B0E00E9447DDFF27662777270E946C
:10DDEA0005DD84E00E94FFDA2896E0E01E2F3E2F30
:10DDFA00173108F03FC1E4E6F6E060E070E00E9407
:10DE0A0005DDE12FF0E031966F2F660F660B762F56
:10DE1A000E9405DDA2E3B0E0E12FF0E0BD01AAE037
:10DE2A00B0E00E942DDCDB01AE0FBF1F0E9443DD74
:10DE3A00662777270E9405DDA2E3B0E0E12FF0E034
:10DE4A00BD01AAE0B0E00E942DDCDB01AE0FBF1FCE
:10DE5A0012960E9443DD662777270E9405DDA2E31A
:10DE6A00B0E0E12FF0E0BD01AAE0B0E00E942DDCB5
:10DE7A00DB01AE0FBF1F14960E9443DD662777278A
:10DE8A000E9405DDA2E3B0E0E12FF0E0BD01AAE0C7
:10DE9A00B0E00E942DDCDB01AE0FBF1F16960E9478
:10DEAA0043DD662777270E9405DDA2E3B0E0E12F74
:10DEBA00F0E0BD01AAE0B0E00E942DDCDB01AE0F6C
:10DECA00BF1F18960E9443DD662777270E9405DD4B
:10DEDA0088E10E94FFDA6C9600E000E0053008F065
:10DEEA00B6C0E02FF0E0309769F4A2E3B0E0E12F8A
:10DEFA00F0E0BD01AAE0B0E00E942DDCDB01AE0F2C
:10DF0A00BF1F47C0E130A0E0FA0771F4A2E3B0E016
:10DF1A00E12FF0E0BD01AAE0B0E00E942DDCDB01B8
:10DF2A00AE0FBF1F129635C0E230A0E0FA0771F4B7
:10DF3A00A2E3B0E0E12FF0E0BD01AAE0B0E00E9468
:10DF4A002DDCDB01AE0FBF1F149623C0E330A0E027
:10DF5A00FA0771F4A2E3B0E0E12FF0E0BD01AAE014
:10DF6A00B0E00E942DDCDB01AE0FBF1F169611C078
:10DF7A00E430A0E0FA0789F4A2E3B0E0E12FF0E090
:10DF8A00BD01AAE0B0E00E942DDCDB01AE0FBF1F8D
:10DF9A0018960E9443DDEE83FF83E12FFF27662751
:10DFAA007727E45EFE4F6F4F6BBFE691E030C1F416
:10DFBA00E02FAAEAB1E080E0FF2766277727EE0F75
:10DFCA00FF1F661F771FEA0FFB1F681F791F0E943A
:10DFDA00F0DCEA87FB87E02FA8EDB1E080E017C00C
:10DFEA00E02FA6E0B2E080E0FF2766277727EE0F52
:10DFFA00FF1F661F771FEA0FFB1F681F791F0E940A
:10E00A00F0DCEA87FB87E02FA4E3B2E080E0FF2799
:10E01A0066277727EE0FFF1F661F771FEA0FFB1F82
:10E02A00681F791F0E94F0DCE887F987EE81FF817B
:10E03A00AA85BB85EA17FB0738F0E885F985AE8122
:10E04A00BF81EA17FB0708F402C00F5F47CFA02F72
:10E05A00E5E0EA17E1E009F0EE27AE2F0E94F7CBE0
:10E06A00053010F4303009F003C0E12FEF5F3E2F86
:10E07A001F5FBECEEFEAF5E060E070E00E9405DDCA
:10E08A0080E00E94FFDA2496A2E2B0E00E9447DD17
:10E09A00EF3181F5203029F4E3E8F6E060E070E042
:10E0AA0022C0503029F4E6E9F6E060E070E01BC0D7
:10E0BA003130A8F0EEEBF5E060E070E00E9405DD9B
:10E0CA00E0911709E695E695EF71FF27662777270E
:10E0DA000E9405DD84E00E94FFDA28960AC0EAEB76
:10E0EA00F5E060E070E00E9405DD80E00E94FFDA62
:10E0FA0024960AC0E8EAF6E060E070E00E9405DDD6
:10E10A0080E00E94FFDA24960E947FDB2C96089515
:10E11A000E947ADB0A2F3C81373108F086C0A9E0D9
:10E12A003A9FF001E45EF64FDF01EC91E068EC9370
:10E13A0030FF1CC03695A8EBB9E0EE27A30FBE1F2F
:10E14A000E9447DD1E2F023019F4E07FE03169F0AA
:10E15A001F70E02FE295E07F1E2BA8EBB9E0EE27B7
:10E16A00A30FBE1FE12F0E9463DD18C03695A8EBEE
:10E17A00B9E0EE27A30FBE1F0E9447DD1E2F023013
:10E18A0019F4EF70E13051F0107F102BA8EBB9E0D1
:10E19A00EE27A30FBE1FE12F0E9463DD46C00E9437
:10E1AA007ADB0A2F3C81373108F03FC0A3E03A9F5F
:10E1BA00F001E551F64FDF01EC91E068EC9330FF96
:10E1CA001CC03695A4ECB9E0EE27A30FBE1F0E942F
:10E1DA0047DD1E2F023019F4E07FE03169F01F702D
:10E1EA00E02FE295E07F1E2BA4ECB9E0EE27A30F07
:10E1FA00BE1FE12F0E9463DD18C03695A4ECB9E07A
:10E20A00EE27A30FBE1F0E9447DD1E2F023019F40E
:10E21A00EF70E13051F0107F102BA4ECB9E0EE273B
:10E22A00A30FBE1FE12F0E9463DD0E9481DB2596AA
:10E23A0008951A930A930A2FEBEBF6E060E070E078
:10E24A000E9405DDE02FFF27662777270E9405DD5C
:10E25A0084E00E94FFDA2896073108F047C0A9E057
:10E26A000A9FF001E45EF64FDF01EC91EF77EC9341
:10E27A00A9E00A9FF001E25EF64FDF01EC91E07F30
:10E28A00EC9300FF02C01FE001C010EFA8EBB9E059
:10E29A00E02FF0E0F595E795AE0FBF1F0E9447DD2E
:10E2AA00E1230E9463DDA9E00A9FF001E45EF64FD4
:10E2BA00E081E17089F00A9FF001E45EF64FE081A7
:10E2CA00E077E03440F00A9FF001E45EF64FDF01A8
:10E2DA00EC91EF78EC9309C0A9E00A9FF001E45EA3
:10E2EA00F64FDF01EC91EF78EC934AC00751003109
:10E2FA0008F046C0A3E00A9FF001E551F64FDF019E
:10E30A00EC91EF77EC93A3E00A9FF001E451F64F0A
:10E31A00DF01EC91EF70EC9300FF02C01FE001C037
:10E32A0010EFA4ECB9E0E02FF0E0F595E795AE0F19
:10E33A00BF1F0E9447DDE1230E9463DDA3E00A9F1D
:10E34A00F001E551F64FE081E17089F00A9FF00192
:10E35A00E551F64FE081E077E03440F00A9FF001A2
:10E36A00E551F64FDF01EC91EF78EC9309C0A9E093
:10E37A000A9FF001E45EF64FDF01EC91EF78EC932F
:10E38A000991199108950E9478DBE0911309E770C9
:10E39A00E23008F0A1C3A7E2B1E00E9447DDE03015
:10E3AA0079F0A7E2B1E00E9447DDAE2F0E94E03D7E
:10E3BA00A5E1B9E0E1700E2EEC91EE7FE029EC9335
:10E3CA00A8E2B1E00E9447DDE03081F0A8E2B1E0C6
:10E3DA000E9447DDAE2F0E94E03DA5E1B9E0E17061
:10E3EA00EE0F0E2EEC91ED7FE029EC9316E117313A
:10E3FA0008F0C7C1A9E01A9FF001E15EF64F20813B
:10E40A00263309F4BCC1A9E01A9FF001E45EF64F75
:10E41A00E081E295E7705E2F40E0E0911309E77032
:10E42A00E13041F41A9FF001E45EF64FE081E170B9
:10E43A003E2F73C0273B09F4A2C1A9E01A9FF0013D
:10E44A00E45EF64FE081E27009F441C0A5E4B1E070
:10E45A00E12FF0E0BD01A7E0B0E00E942DDCDB0176
:10E46A00AE0FBF1F12960E9447DDE07121F0E091C6
:10E47A001509E17059F5A5E4B1E0E12FF0E0BD011D
:10E48A00A7E0B0E00E942DDCDB01AE0FBF1F1296A1
:10E49A000E9447DDE07221F0E0911509E270B1F4C3
:10E4AA00A5E4B1E0E12FF0E0BD01A7E0B0E00E94F1
:10E4BA002DDCDB01AE0FBF1F12960E9447DDE07410
:10E4CA0021F0E0911409E07809F401C001C002C00A
:10E4DA0030E016C0A22F0E94E03D3E2FA9E01A9F0D
:10E4EA00F001E35EF64FE081E07121F0E091240E45
:10E4FA00E17009F405C0303011F030E001C031E0BC
:10E50A00A9E01A9FF001E45EF64FDF01E32FE17004
:10E51A000E2EEC91EE7FE029EC93303069F1E52F75
:10E52A00F0E0309721F0E130A0E0FA07D9F4E09169
:10E53A001409E770E23098F0EAECF6E060E070E087
:10E54A000E9405DDE12FF0E031966F2F660F660B12
:10E55A00762F0E9405DD84E00E94FFDA289641E0CA
:10E56A0052E009C0E430A0E0FA0721F0E530A0E06B
:10E57A00FA0709F442E029C0503011F0513009F489
:10E58A0024C042E050E0A9E01A9FF001E45EF64F91
:10E59A00DF01EC91EB7FEC93A9E01A9FF001ED5DAE
:10E5AA00F64FA0E0B0E0A083B183A9E01A9FF00182
:10E5BA00E05EF64FA0E0A083A9E01A9FF001E25EB8
:10E5CA00F64FDF01EC91E07FEC93E42FF0E0309717
:10E5DA0009F484C0E130A0E0FA0709F05CC0A12F79
:10E5EA000E942C62A9E01A9FF001E35EF64FDF0158
:10E5FA00EC91E068EC93A9E01A9FF001E05EF64F17
:10E60A00A0E0A083A9E01A9FF001E25EF64FDF01C5
:10E61A00EC91E07FEC93A9E01A9FF001E35EF64FDC
:10E62A00E081E074B9F1E12FFF2766277727EC52E2
:10E63A00FF4F6F4F6BBF06910A9FF001E45EF64FE2
:10E64A00DF01EC91E160EC93A9E00A9FF001E45E3E
:10E65A00F64FDF01EC91EF78E062EC93A9E00A9FB4
:10E66A00F001E35EF64FDF01EC91E068EC93A9E07C
:10E67A000A9FF001E05EF64FA0E0A083A9E00A9F9E
:10E68A00F001E25EF64FDF01EC91E07FEC93A02F00
:10E69A000E942C6223C0E230A0E0FA07F9F4A12F0D
:10E6AA000E94C461A9E01A9FF001E35EF64FE0817F
:10E6BA00E074A1F0E12FFF2766277727EC52FF4F7E
:10E6CA006F4F6BBF06910A9FF001E45EF64FDF01C0
:10E6DA00EC91EE7FEC93A02F0E94C461E0911409A3
:10E6EA00E770E23050F0A9E01A9FF001E45EF64FBD
:10E6FA00E081E295E7705E1709F432C0E6EDF6E0D4
:10E70A0060E070E00E9405DDE12FF0E031966F2FA6
:10E71A00660F660B762F0E9405DDA9E01A9FF001AD
:10E72A00E45EF64FE081E295E770FF2766277727D8
:10E73A000E9405DDE52FFF27662777270E9405DD62
:10E74A00E32FFF27662777270E9405DDE42FFF279F
:10E75A00662777270E9405DD84E10E94FFDA689622
:10E76A00A9E01A9FF001E45EF64FDF01E52FE7709A
:10E77A00E295E07F0E2EEC91EF78E029EC931150B0
:10E78A0036CE10E0103108F0A7C1A3E01A9FF001BD
:10E79A00E351F64F20811A9FF001E551F64FE081CF
:10E7AA00E295E7705E2F40E0E0911309E770E130EF
:10E7BA0041F41A9FF001E551F64FE081E1703E2FD6
:10E7CA005DC0A22F0E94E03D3E2FA3E01A9FF001F8
:10E7DA00E551F64FE081E27009F443C01A9FF00157
:10E7EA00E551F64FE081E270A9F1A6EEB1E0E12F22
:10E7FA00F0E0EE0FFF1FAE0FBF1F11960E9447DD1C
:10E80A00E17021F0E0911509E17019F5A6EEB1E089
:10E81A00E12FF0E0EE0FFF1FAE0FBF1F11960E940F
:10E82A0047DDE27021F0E0911509E27091F4A6EE5D
:10E83A00B1E0E12FF0E0EE0FFF1FAE0FBF1F119600
:10E84A000E9447DDE47021F0E0911409E07809F4B0
:10E85A0001C001C002C030E004C0A22F0E94E03D06
:10E86A003E2FA3E01A9FF001E551F64FDF01E32F97
:10E87A00E1700E2EEC91EE7FE029EC933030A9F195
:10E88A00E52FF0E0309721F0E130A0E0FA0761F5DA
:10E89A00E0911409E770E23098F0EAECF6E060E003
:10E8AA0070E00E9405DDE12FF0E031966F2F660FD0
:10E8BA00660B762F0E9405DD84E00E94FFDA289617
:10E8CA0041E052E0A3E01A9FF001E551F64FDF0163
:10E8DA00EC91E37FEC93A3E01A9FF001E451F64F29
:10E8EA00DF01EC91EF70EC9310C0503011F0513011
:10E8FA0009F40BC042E050E0A3E01A9FF001E45192
:10E90A00F64FDF01EC91EF70EC93E42FF0E03097D3
:10E91A0009F48FC0E130A0E0FA0709F043C0E12F03
:10E92A00FF2766277727A3E0B0E00E942DDCEE5987
:10E93A00FD4F6F4F6BBFE691E030D1F0E12FFF271B
:10E94A0066277727A3E0B0E00E942DDCEE59FD4F41
:10E95A006F4FEF5FFF4F6F4F7F4F6BBFE691A091F5
:10E96A000E09EA2BE0930E09E0E0E093080919C0CA
:10E97A00E12FFF2766277727A3E0B0E00E942DDC6E
:10E98A00EE59FD4F6F4FEF5FFF4F6F4F7F4F6BBFDA
:10E99A00E691A0910D09EA2BE0930D09E0E0E093DE
:10E9AA00070947C0E230A0E0FA0709F042C0E12FA8
:10E9BA00FF2766277727A3E0B0E00E942DDCEE59F7
:10E9CA00FD4F6F4F6BBFE691E030D1F0E12FFF278B
:10E9DA0066277727A3E0B0E00E942DDCEE59FD4FB1
:10E9EA006F4FEE5FFF4F6F4F7F4F6BBFE691A09166
:10E9FA000E09EA23E0930E09E0E0E093080919C042
:10EA0A00E12FFF2766277727A3E0B0E00E942DDCDD
:10EA1A00EE59FD4F6F4FEE5FFF4F6F4F7F4F6BBF4A
:10EA2A00E691A0910D09EA23E0930D09E0E0E09355
:10EA3A000709E0911409E770E23050F0A3E01A9F49
:10EA4A00F001E551F64FE081E295E7705E1709F4AF
:10EA5A0032C0E6EDF6E060E070E00E9405DDE12FED
:10EA6A00F0E078966F2F660F660B762F0E9405DD11
:10EA7A00A3E01A9FF001E551F64FE081E295E770B5
:10EA8A00FF27662777270E9405DDE52FFF276627E0
:10EA9A0077270E9405DDE32FFF27662777270E9445
:10EAAA0005DDE42FFF27662777270E9405DD84E12D
:10EABA000E94FFDA6896A3E01A9FF001E551F64F2B
:10EACA00DF01E52FE770E295E07F0E2EEC91EF78FB
:10EADA00E029EC931F5F56CE0E947FDB26960895AD
:10EAEA0027970E947ADB8D013B852C85E7E0ED8331
:10EAFA00E9EFEE83EF81E160EF83E32FE170EE0F40
:10EB0A000E2EEF81ED7FE029EF83203011F4E7E04C
:10EB1A0001C0E8E0E887E22FEF73EE0FEE0F0E2E4A
:10EB2A00EF81E370E029EF8309871A87DE011496E3
:10EB3A000E94CA9FA32F0E94F7CB0E9481DB2D96C9
:10EB4A00089563970E9478DBE0911309E770E23039
:10EB5A0088F0E0911309E770E73019F40E94726BAC
:10EB6A0002C00E947168E4E1E09318090E947FDB09
:10EB7A0069960895E0E0F0E0E0931A09F0931B0922
:10EB8A00E0911709E170C9F1E0911709EE7FE0936E
:10EB9A001709E6EFF6E060E070E00E9405DD80E02C
:10EBAA000E94FFDA2496E0E0EC8BAC89A03210F5E3
:10EBBA00EBEFF6E060E070E00E9405DDE88DFF27EC
:10EBCA00662777270E9405DDA1E4B8E0EC8DF0E026
:10EBDA00EE0FFF1FAE0FBF1FED91FD91662777273E
:10EBEA000E9405DD88E00E94FFDA2C96EC89EF5F2F
:10EBFA00EC8BDBCFAAE00E94089FABE1B0E00E9459
:10EC0A0043DDEE87FF87A0912A0EB0912B0EE0918B
:10EC1A006D08F0916E080E9408DCEA0FFB1FE09372
:10EC2A002A0EF0932B0EE091290EEF70E93038F49A
:10EC3A00A9E2BEE080E0EFE00E9435DD6BC0E09122
:10EC4A00290EE071D1F1E091290EEF7EE093290EB1
:10EC5A00ABE1B0E0E0912A0EF0912B0E0E945BDD51
:10EC6A00E6E0E093270EE2E0F7E060E070E00E9461
:10EC7A0005DDE0912A0EF0912B0E662777270E9478
:10EC8A0005DD84E00E94FFDA2896E0E0EA93A0918D
:10EC9A002A0EB0912B0EA03CE3E3BE0730F0A1345C
:10ECAA00EFE3BE0710F4E1E001C0E0E0EA93A091CF
:10ECBA002A0EB0912B0E14DF22C0E0912A0EF09199
:10ECCA002B0E66277727EA87FB876C877D87A0EE5E
:10ECDA00BEE280E090E00E9435DCEA87FB876C8721
:10ECEA007D87EE85FF85AA85BB858C859D856627F0
:10ECFA0077270E948BDCE0932C0EF0932D0EE09187
:10ED0A00290EE07FE093290EE0E0F0E0E0932A0E7E
:10ED1A00F0932B0EE0916D08F0916E086627772725
:10ED2A00EA87FB876C877D87ACE2B1E080E090E000
:10ED3A000E9435DCEA87FB876C877D87EE85FF8535
:10ED4A00F695E795AA85BB858C859D8566277727E5
:10ED5A00EA0FFB1F681F791FEA87FB876C877D878D
:10ED6A00EE85FF85AA85BB858C859D8566277727D5
:10ED7A000E948BDCE0932E0EAAE2B1E00E9447DDEE
:10ED8A00E13008F4A1C0E0911409E07809F443C025
:10ED9A00A0912C0EB0912D0EE4E6F0E00E9473DCF7
:10EDAA000F01ACE2B1E00E9447DDD001F0E0AE17FE
:10EDBA00BF0768F1ADE2B1E00E9447DDA0911909F1
:10EDCA00AE1738F4E0911909EF5FE0931909E150A1
:10EDDA001DC0ECE0F7E060E070E00E9405DDE09124
:10EDEA002C0EF0912D0E662777270E9405DD84E010
:10EDFA000E94FFDA2896A9E00E94E82AE091140905
:10EE0A00EF77E0931409E0E0E093190903C0E0E02A
:10EE1A00E093190959C0E0E0EB8BABE2B1E00E9444
:10EE2A0047DDEA3058F4AAE2B1E00E9447DDA0913A
:10EE3A002E0EAE1710F4E1E0EB8B14C0A0912C0E4D
:10EE4A00B0912D0EE4E6F0E00E9473DC0F01AAE215
:10EE5A00B1E00E9447DDD001F0E0AE17BF0710F421
:10EE6A00E1E0EB8BEB89E03061F1ABE2B1E00E94CB
:10EE7A0047DDA0911909AE1738F4E0911909EF5F3F
:10EE8A00E0931909E1501CC0ECE1F7E060E070E0A2
:10EE9A000E9405DDE0912E0EFF27662777270E9444
:10EEAA0005DD84E00E94FFDA2896A8E00E94E82A9D
:10EEBA00E0911409E068E0931409E0E0E09319098D
:10EECA0003C0E0E0E0931909A091220EA53420F4D2
:10EEDA00A0912E0EAB3520F0A0912E0EAD3330F559
:10EEEA00E0911809E030E9F4EDE2F7E060E070E063
:10EEFA000E9405DDE0912E0EF0E06F2F660F660B83
:10EF0A00762F0E94E0DDDF01CB01E0E0F0E060E275
:10EF1A0071E40E94B7DE0E9405DD84E00E94FFDAF8
:10EF2A002896EAE0E0931809F19A35C0A0911809E9
:10EF3A00A13088F1E0911809E150E0931809EF5FD8
:10EF4A00E0911809E03039F5E0911409E07411F103
:10EF5A00E0911409EF7BE0931409E5E4F7E060E03F
:10EF6A0070E00E9405DDE0912E0EF0E06F2F660F33
:10EF7A00660B762F0E94E0DDDF01CB01E0E0F0E0D6
:10EF8A0060E271E40E94B7DE0E9405DD84E00E941F
:10EF9A00FFDA2896F198A0911809E0E0EA17E1E073
:10EFAA0008F0EE27E98BA091310EB091320EE09174
:10EFBA007508F0917608F695E795EA0FFB1FE0933E
:10EFCA00310EF093320EE0912F0EEF70E73038F4E5
:10EFDA00AFE2BEE080E0EFE00E9435DD05C1A0911E
:10EFEA00310EB091320EE0EAF0E060E070E00E948B
:10EFFA00F0DCAE17BF0720F0E0E0E093300EE9C086
:10F00A00A091310EB091320EE2EDF0E060E070E0D6
:10F01A000E94F0DCAE17BF0720F4EAEFE093300E4F
:10F02A00D8C0E1E0EC8BEC89A0EAB0E080E0FF27F1
:10F03A0066277727EE0FFF1F661F771FEA0FFB1F52
:10F04A00681F791F0E94FBDCE091310EF091320EAD
:10F05A00EA17FB0720F4EC89EF5FEC8BE4CFEC892D
:10F06A00E150EC8BAAE0EA02F001E093300EEC8961
:10F07A00A0EAB0E080E0FF2766277727EE0FFF1FA0
:10F08A00661F771FEA0FFB1F681F791F0E94F0DCBB
:10F09A00A091310EB091320EEA1BFB0BEE87FF876F
:10F0AA00AE85BF85EAE00E9455DCEE87FF87EC89D2
:10F0BA00A0EAB0E080E0FF2766277727EE0FFF1F60
:10F0CA00661F771FEA0FFB1F681F791F0E94FBDC70
:10F0DA00EC89F0E066277727EE0FFF1F661F771F80
:10F0EA00EE55FF4F6F4F0E94F0DC0E9415DDEA1BC0
:10F0FA00FB0BAE85BF850E9473DCEE87FF87E0912C
:10F10A00300EAE85EA0FE093300EA6E3B1E00E941E
:10F11A0047DDEE83AE81A03054F1E0912F0EE0720C
:10F12A00A1F0E091300EF0E0F595E795DF01EE8170
:10F13A00F0E0E7FDFFEF3197AE17BF072CF4E0913F
:10F14A002F0EEF7DE0932F0E12C0E091300EF0E00B
:10F15A00F595E795DF01EE81F0E0E7FDFFEFAE17E9
:10F16A00BF072CF0E0912F0EE062E0932F0EA7E389
:10F17A00B1E00E9447DDEE83AE81A03054F1E09108
:10F18A002F0EE074A1F0E091300EF0E0F595E795CE
:10F19A00DF01EE81F0E0E7FDFFEF3197AE17BF0721
:10F1AA002CF4E0912F0EEF7BE0932F0E12C0E0912A
:10F1BA00300EF0E0F595E795DF01EE81F0E0E7FD2E
:10F1CA00FFEFAE17BF072CF0E0912F0EE064E0933B
:10F1DA002F0EE0912F0EE07FE0932F0EE0E0F0E09B
:10F1EA00E093310EF093320EA0913F08A13008F45B
:10F1FA0097C0E0913F08F0E0E130A0E0FA07C1F5DE
:10F20A00E0917F08F091800866277727A8EEB3E09F
:10F21A0080E090E00E9435DC7F936F93FF93EF9339
:10F22A00ADE1B0E00E9443DDAF91BF918F919F9114
:10F23A00662777270E948BDCE0938108F093820887
:10F24A00A0918108B0918208139718F4E0E0F0E0E9
:10F25A000AC0A0918108B0918208A93FE7E0BE07E1
:10F26A0030F0E8EFF7E0E0938108F093820858C0A5
:10F27A00E230A0E0FA0721F4E3E0E0933F0850C04F
:10F28A00E330A0E0FA0709F04BC0E1E0E0933F0861
:10F29A00E0917F08F0918008F695E795EE87FF8761
:10F2AA00ADE1B0E00E945BDDECE5F7E060E070E024
:10F2BA000E9405DDEA89FB89662777270E9405DD1A
:10F2CA0084E00E94FFDA2896E3E0EA93EF85F88962
:10F2DA00E53AA7E1FA0740F0AF85B889A73EECE125
:10F2EA00BE0710F4E1E001C0E0E0EA93A889B98919
:10F2FA00F7DBE1E0E0933F08E6E0E093270EA09118
:10F30A004008A23020F4F49B02C0F59B01C008C05B
:10F31A00E0910B09E068E0930B09E0E0E09306094D
:10F32A00A0914008A13008F497C0E0914008F0E0AD
:10F33A00E130A0E0FA07C1F5A0914108B091420876
:10F34A0088279927E8EEF3E060E070E00E9435DC58
:10F35A007F936F93FF93EF93AFE1B0E00E9443DD99
:10F36A00AF91BF918F919F91662777270E948BDC7F
:10F37A00E0938308F0938408A0918308B0918408ED
:10F38A00139718F4E0E0F0E00AC0A0918308B09166
:10F39A008408A93FE7E0BE0730F0E8EFF7E0E09322
:10F3AA008308F093840858C0E230A0E0FA0721F4F9
:10F3BA00E3E0E093400850C0E330A0E0FA0709F028
:10F3CA004BC0E1E0E0934008E0914108F091420827
:10F3DA00F695E795EE87FF87AFE1B0E00E945BDD27
:10F3EA00E6E0E093270EE8E6F7E060E070E00E94CE
:10F3FA0005DDEA89FB89662777270E9405DD84E017
:10F40A000E94FFDA2896E4E0EA93EF85F889E53A64
:10F41A00A7E1FA0740F0AF85B889A73EECE1BE073D
:10F42A0010F4E1E001C0E0E0EA93A889B98958DB69
:10F43A00E1E0E0934008A0913F08A23020F4F49B59
:10F44A0002C0F59B01C008C0E0910B09E068E09397
:10F45A000B09E0E0E0930609E6E1EC8BAC89A73101
:10F46A0008F0AEC6EC89A9E0EA9FF001E35EF64F28
:10F47A00E081E07849F0EC89EA9FF001E35EF64F1B
:10F48A00DF01EC91EF7797C6EC89A9E0EA9FF001DA
:10F49A00E15EF64FE081E987E0E0EF83E88BA9853A
:10F4AA00A633D9F4EC89FF2766277727EC52FF4F5A
:10F4BA006F4F6BBFE691A9E0EA9FF001E45EF64F59
:10F4CA00E081E170EA8BEC89FF2766277727EC5207
:10F4DA00FF4F6F4F6BBFE6910AC0EC89A9E0EA9F24
:10F4EA00F001E45EF64FE081E170EA8BEC89A9E075
:10F4FA00EA9FF001E45EF64FE081E295E770E88763
:10F50A00EA89E03009F4F5C4A1E4B8E0EC89FF2700
:10F51A0066277727EC5FFE4F6F4F6BBFE691F0E0EF
:10F52A00EE0FFF1FAE0FBF1FED91FD91F695E79508
:10F53A00EE87FF87A2E3B0E0EC89F0E0BD01AAE024
:10F54A00B0E00E942DDCDB01AE0FBF1F0E9443DD3D
:10F55A008F01AE85BF850A171B0720F0E0E0EE8712
:10F56A00EF87F1C0A2E3B0E0EC89F0E0BD01AAE0C8
:10F57A00B0E00E942DDCDB01AE0FBF1F12960E9485
:10F58A0043DD9F01AE85BF852A173B0710F1EE8543
:10F59A00FF85E01BF10BEE87FF87662777276E2F23
:10F5AA007F2FE0E0F0E07F936F93FF93EF93F901F1
:10F5BA00E01BF10B66277727AFE8B2E080E090E026
:10F5CA000E9435DCAF91BF918F919F910E948BDC95
:10F5DA00B8C0A2E3B0E0EC89F0E0BD01AAE0B0E077
:10F5EA000E942DDCDB01AE0FBF1F14960E9443DD83
:10F5FA00AF01AE85BF854A175B0738F1EE85FF85F7
:10F60A00E21BF30BEE87FF87AE85BF858827992714
:10F61A00E1E10E94C4DB7F936F93FF93EF93FA01BA
:10F62A00E21BF30B66277727AFE8B2E080E090E0B1
:10F63A000E9435DCAF91BF918F919F910E948BDC24
:10F64A00EE87FF87EC59FF4F7CC0A2E3B0E0EC895C
:10F65A00F0E0BD01AAE0B0E00E942DDCDB01AE0FB4
:10F66A00BF1F16960E9443DDEF8BF88FAE85BF85CC
:10F67A00EA17FB0740F1EE85FF85E41BF50BEE87E1
:10F68A00FF87AE85BF8588279927E1E10E94C4DB01
:10F69A007F936F93FF93EF93EF89F88DE41BF50B3C
:10F6AA0066277727A4EBB1E080E090E00E9435DC82
:10F6BA00AF91BF918F919F910E948BDCEE87FF875C
:10F6CA00E45DFE4F3EC0A2E3B0E0EC89F0E0BD018C
:10F6DA00AAE0B0E00E942DDCDB01AE0FBF1F189636
:10F6EA000E9443DDED8BFE8BAF89B88DEE85FF85D9
:10F6FA00EA1BFB0BEE87FF87AE85BF858827992714
:10F70A00E3E10E94C4DB7F936F93FF93EF93AF898A
:10F71A00B88DED89FE89EA1BFB0BF695E7956627FE
:10F72A007727ACEEB2E080E090E00E9435DCAF9142
:10F73A00BF918F919F910E948BDCEE87FF87E85AD9
:10F74A00FD4FEE87FF87A985A73BA1F0A63389F471
:10F75A00EC89FF2766277727EC52FF4F6F4F6BBF65
:10F76A00E691A9E0EA9FF001E15EF64FA081A73B8E
:10F77A0009F06EC0A985A73B19F4EC89EB8B0AC086
:10F78A00EC89FF2766277727EC52FF4F6F4F6BBF35
:10F79A0006900B8AA6E2BAE0EB89FF27662777274D
:10F7AA00EC5CFE4F6F4F6BBFE691F0E00E94F4DB1A
:10F7BA00AE0FBF1F1196AC91A83C11F4E0E001C056
:10F7CA00E1E0E88BAE85BF85A130E0E4BE0720F01A
:10F7DA00E0E0F0E4EE87FF87EC89A9E0EA9FF00118
:10F7EA00EF5DF64FCF0160817181EC89A9E0EA9F54
:10F7FA00F001EF5DF64FDF01ED91FD910E9404DC0F
:10F80A00DF01FB01EA1BFB0BDC01ED93FC93EC89A6
:10F81A00A9E0EA9FF001EF5DF64F0F01DF01ED91DC
:10F82A00FD91DF01EE85FF850E9408DCEA0FFB1FD0
:10F83A00D001ED93FC93EC89A9E0EA9FF001EF5D1A
:10F84A00F64FDF01ED91FD910E9408DCEE87FF87FC
:10F85A00E0911A09F0911B09AE85BF85EA0FFB1FDB
:10F86A00E0931A09F0931B09EC89A9E0EA9FF001D9
:10F87A00E35EF64FE081E074B1F0EC89FF2766277A
:10F88A007727EC52FF4F6F4F6BBFE691EA9FF0016B
:10F89A00ED5DF64FDF01ED91FD91AE85BF85EA0F73
:10F8AA00FB1FEE87FF87AE85BF85A73FE7E2BE074E
:10F8BA0020F0E6EFF7E2EE87FF87EC89A9E0EA9FFE
:10F8CA00F001ED5DF64FAE85BF85A083B183E0916F
:10F8DA001409E870C9F0E4E7F7E060E070E00E941C
:10F8EA0005DDE88DF0E031966F2F660F660B762FF7
:10F8FA000E9405DDEE89FF89662777270E9405DDCC
:10F90A0088E00E94FFDA2C96E885F0E0E230A0E079
:10F91A00FA0709F0A3C0A989A03039F5A5EEB8E025
:10F92A00EC89FF2766277727EC5FFE4F6F4F6BBF87
:10F93A00E691F0E0AE0FBF1FAC91A230A8F4A889FF
:10F94A00A03089F4A5E8B8E0EC89FF276627772775
:10F95A00E451FF4F6F4F6BBFE691F0E0AE0FBF1F50
:10F96A00EC91E07409F401C001C04FC0EC89A9E030
:10F97A00EA9FF001E25EF64FE081EF70E43058F45E
:10F98A00EC89EA9FF001E25EF64FDF0180E0EFE0EA
:10F99A000E9435DD3AC0E5E0E887E2E0EF83EC89D2
:10F9AA00EA93A3E00E948D70EC89A9E0EA9FF00136
:10F9BA00E35EF64FE081EF70EA3098F4EC89EA9F53
:10F9CA00F001E35EF64FDF0180E0EFE00E9435DDF3
:10F9DA00E6E6EA93ED89E15FEA93A0E0B0E00E94EF
:10F9EA00F12AE0E8F7E060E070E00E9405DDE88DCA
:10F9FA00F0E031966F2F660F660B762F0E9405DDB9
:10FA0A0084E00E94FFDA289673C2EC89A9E0EA9F93
:10FA1A00F001E05EF64FA081A53058F4EC89A9E028
:10FA2A00EA9FF001E05EF64FDF01EC91EF5FEC93A5
:10FA3A0014C0EC89A9E0EA9FF001E05EF64FA0E06D
:10FA4A00A083EC89A9E0EA9FF001E25EF64FDF01AC
:10FA5A00EC91E07FEC93E3E0E8874AC2E330A0E070
:10FA6A00FA0709F045C2A989A03039F5A5EEB8E030
:10FA7A00EC89FF2766277727EC5FFE4F6F4F6BBF36
:10FA8A00E691F0E0AE0FBF1FAC91A230A8F4A889AE
:10FA9A00A03089F4A5E8B8E0EC89FF276627772724
:10FAAA00E451FF4F6F4F6BBFE691F0E0AE0FBF1FFF
:10FABA00EC91E07409F401C001C050C0EC89A9E0DE
:10FACA00EA9FF001E25EF64FE081EF70E33058F40E
:10FADA00EC89EA9FF001E25EF64FDF0180E0EFE099
:10FAEA000E9435DD3AC0E5E0E887E2E0EF83EC8981
:10FAFA00EA93A3E00E948D70EC89A9E0EA9FF001E5
:10FB0A00E35EF64FE081EF70EA3098F4EC89EA9F01
:10FB1A00F001E35EF64FDF0180E0EFE00E9435DDA1
:10FB2A00E6E6EA93ED89E15FEA93A0E0B0E00E949D
:10FB3A00F12AEFE8F7E060E070E00E9405DDE88D69
:10FB4A00F0E031966F2F660F660B762F0E9405DD67
:10FB5A0084E00E94FFDA2896CBC114C0EC89A9E0A0
:10FB6A00EA9FF001E25EF64FE081EF70E13050F07B
:10FB7A00EC89EA9FF001E25EF64FDF0180E0EFE0F8
:10FB8A000E9439DDA985A63309F4B2C1A5E4B1E022
:10FB9A00EC89F0E0BD01A7E0B0E00E942DDCDB01BA
:10FBAA00AE0FBF1F14960E9443DDFF71EE87FF87D9
:10FBBA00EC89A9E0EA9FF001E15EF64FA081A73B3C
:10FBCA0079F4E0911309E770E13049F4EC89A9E08E
:10FBDA00EA9FF001E45EF64FE081E17009F401C0AA
:10FBEA0035C0A6E2BAE0EC89FF2766277727EC5CE6
:10FBFA00FE4F6F4F6BBFE691F0E00E94F4DBAE0F51
:10FC0A00BF1F1196EC91EB8BE03029F4EE85FF854E
:10FC1A000E9406DC19C0EB89EC5EEB8BAB89A83C31
:10FC2A00A8F4AE85BF8588279927F0E06F2F660F65
:10FC3A00660B762F0E9435DCDF01CB01E8ECF0E0A1
:10FC4A0060E070E00E948BDCEE87FF87EC89A9E018
:10FC5A00EA9FF001ED5DF64FDF01ED91FD91DF01C5
:10FC6A00EE85FF85AE17BF0708F48CC0EC89A9E0C2
:10FC7A00EA9FF001E45EF64FDF01EC91EB7FEC9333
:10FC8A00EC89A9E0EA9FF001E45EF64FE081E870B2
:10FC9A0091F4EC89EA9FF001E45EF64FDF01EC9102
:10FCAA00E860EC93EC89A9E0EA9FF001E05EF64F88
:10FCBA00A0E0A08366C0EC89A9E0EA9FF001E05EBB
:10FCCA00F64FDF01EC91EF5FEC93EC89A9E0EA9F34
:10FCDA00F001E05EF64FE081EF93A5E4B1E0EC8934
:10FCEA00F0E0BD01A7E0B0E00E942DDCDB01AE0F21
:10FCFA00BF1F16960E9447DDAF91AE1708F441C0A8
:10FD0A00E4E0E887E2E0EF83EC89EA93A4E00E946A
:10FD1A008D70EC89A9E0EA9FF001E35EF64FE0817D
:10FD2A00EF70EA30D8F4EC89EA9FF001E35EF64F0F
:10FD3A00DF0180E0EFE00E9435DDE7E6EA93ED8936
:10FD4A00E15FEA93EE89A9E0EA9FF001ED5DF64FE3
:10FD5A00DF01ED91FD91DF010E94F12AEEE9F7E062
:10FD6A0060E070E00E9405DDE88DF0E031966F2FCB
:10FD7A00660F660B762F0E9405DD84E00E94FFDA8B
:10FD8A002896B6C0EC89A9E0EA9FF001E45EF64F36
:10FD9A00E081E87089F0EC89EA9FF001E45EF64FB1
:10FDAA00DF01EC91E77FEC93EC89A9E0EA9FF0018F
:10FDBA00E05EF64FA0E0A083A5E4B1E0EC89F0E0B4
:10FDCA00BD01A7E0B0E00E942DDCDB01AE0FBF1F32
:10FDDA0011960E9443DDFF70EE87FF87AE85BF85CF
:10FDEA0000240A160B0608F083C0EC89A9E0EA9FF2
:10FDFA00F001ED5DF64FDF01ED91FD91AE85BF8516
:10FE0A00EA17FB0708F062C0EC89A9E0EA9FF00153
:10FE1A00E05EF64FE081EF93A5E4B1E0EC89F0E013
:10FE2A00BD01A7E0B0E00E942DDCDB01AE0FBF1FD1
:10FE3A0013960E9447DDAF91AE1758F4EC89A9E0FA
:10FE4A00EA9FF001E05EF64FDF01EC91EF5FEC9381
:10FE5A003CC0EC89A9E0EA9FF001E45EF64FE0813C
:10FE6A00E47099F5EC89EA9FF001E45EF64FDF0150
:10FE7A00EC91E460EC93EC89EA93A2E00E948D7025
:10FE8A00EC89A9E0EA9FF001E35EF64FE081EF70AA
:10FE9A00EA30D8F4EC89EA9FF001E35EF64FDF011D
:10FEAA0080E0EFE00E9435DDE5E6EA93ED89E15F67
:10FEBA00EA93EE89A9E0EA9FF001ED5DF64FDF01D2
:10FECA00ED91FD91DF010E94F12A12C0EC89A9E0AF
:10FEDA00EA9FF001E05EF64FA0E0A083EC89A9E07A
:10FEEA00EA9FF001E45EF64FDF01EC91EB7FEC93C1
:10FEFA00D0C0EC89A9E0EA9FF001ED5DF64FA0E0E1
:10FF0A00B0E0A083B183EC89A9E0EA9FF001EF5D3C
:10FF1A00F64FA0E0B0E0A083B183A985A63389F0AB
:10FF2A00A5E4B1E0EC89F0E0BD01A7E0B0E00E94F1
:10FF3A002DDCDB01AE0FBF1F12960E9447DDE07871
:10FF4A0009F4A7C0E885F0E0309709F06CC0E989A8
:10FF5A00E03009F09EC0A5EAB8E0EC89FF276627E1
:10FF6A007727E451FF4F6F4F6BBFE691F0E0AE0F7A
:10FF7A00BF1FEC91E07459F4EC89A9E0EA9FF00103
:10FF8A00E25EF64FDF01EC91E07FEC934BC0EC8927
:10FF9A00A9E0EA9FF001E25EF64FE081EF70EF30F0
:10FFAA0058F4EC89EA9FF001E25EF64FDF0180E047
:10FFBA00EFE00E9435DD36C0E1E0E887EC89A9E090
:10FFCA00EA9FF001E25EF64FDF01EC91E07FEC93ED
:10FFDA00EC89EA93A1E00E948D70EC89A9E0EA9F7E
:10FFEA00F001E35EF64FE081EF70EA30D8F4EC8975
:06FFFA00EA9FF001E35E46
:020000021000EC
:0A000000F64FDF0180E0EFE00E9400
:10000A0035DDE4E6EA93ED89E15FEA93EE89A9E05A
:10001A00EA9FF001ED5DF64FDF01ED91FD91DF0101
:10002A000E94F12A36C0E130A0E0FA0791F5A5EA6C
:10003A00B8E0EC89FF2766277727E451FF4F6F4F17
:10004A006BBFE691F0E0AE0FBF1FEC91E07409F5CB
:10005A00EC89A9E0EA9FF001E25EF64FE081EF70D9
:10006A00EF3058F4EC89EA9FF001E25EF64FDF01C7
:10007A0080E0EFE00E9435DD0CC0E0E0E887EC8923
:10008A00A9E0EA9FF001E25EF64FDF01EC91E07F22
:10009A00EC93AF81A230B1F5AC890E94C461EC89BE
:1000AA00A9E0EA9FF001E35EF64FE081E07419F4FB
:1000BA00A985A63339F5EC89FF2766277727EC52FD
:1000CA00FF4F6F4F6BBF06900B8AEB89A9E0EA9F3F
:1000DA00F001E45EF64FDF01EC91EE7FEC93EB89E1
:1000EA00A9E0EA9FF001E45EF64FDF01E885E770D8
:1000FA00E295E07F0E2EEC91EF78E029EC93AB8944
:10010A000E94C461AF81A23009F046C0E09114098F
:10011A00E770E23068F0EC89A9E0EA9FF001E45E5A
:10012A00F64FE081E295E770AE2FE885EA1709F409
:10013A0033C0EDEAF7E060E070E00E9405DDE88D8B
:10014A00F0E031966F2F660F660B762F0E9405DD61
:10015A00EC8DA9E0EA9FF001E45EF64FE081E295BA
:10016A00E770FF27662777270E9405DDEC89FF27BE
:10017A00662777270E9405DDEAA1FF2766277727EA
:10018A000E9405DDEB8DFF27662777270E9405DD94
:10019A0084E10E94FFDA6896EC89A9E0EA9FF001FF
:1001AA00E45EF64FDF01E885E770E295E07F0E2E08
:1001BA00EC91EF78E029EC93EC89E150EC8B4EC995
:1001CA00E0E0EC8BAC89A03108F05CC2EC89A3E0DA
:1001DA00EA9FF001E551F64FE081E295E770E88782
:1001EA00E0E0EF83EC89EA9FF001E551F64FE08108
:1001FA00E17009F401C1E885F0E0E230A0E0FA0715
:10020A0009F086C0EC89A3E0EA9FF001E551F64FB8
:10021A00E081EC70EC3058F4EC89EA9FF001E5518A
:10022A00F64FDF0182E0E3E00E9435DD70C0A98964
:10023A00A03089F4A5EAB8E0EC89FF27662777277A
:10024A00EE56FD4F6F4F6BBFE691F0E0AE0FBF1F4A
:10025A00EC91E07809F04FC0EC89A3E0EA9FF00145
:10026A00E451F64FE081E07FE03458F4EC89EA9FEC
:10027A00F001E451F64FDF0184E0EFE00E9435DD42
:10028A0039C0E5E0E887E2E0EF83EC89EA93A3E08E
:10029A000E94D470EC89A3E0EA9FF001E451F64F82
:1002AA00E081EF70EA3098F4EC89EA9FF001E451BA
:1002BA00F64FDF0180E0EFE00E9435DDE6E6EA93E3
:1002CA00ED89EA5DEA93A0E0B0E00E94F12AEEEC43
:1002DA00F7E060E070E00E9405DDE88DF0E07896D6
:1002EA006F2F660F660B762F0E9405DD84E00E9451
:1002FA00FFDA28960CC0EC89A3E0EA9FF001E451EA
:10030A00F64FDF01EC91EF70EC93E3E0E88773C0FE
:10031A00E330A0E0FA0709F06EC0A989A03089F499
:10032A00A5EAB8E0EC89FF2766277727EE56FD4F46
:10033A006F4F6BBFE691F0E0AE0FBF1FEC91E07814
:10034A0009F04FC0EC89A3E0EA9FF001E451F64FAF
:10035A00E081E07FE03358F4EC89EA9FF001E45150
:10036A00F64FDF0184E0EFE00E9435DD39C0E2E0BC
:10037A00EF83E4E0E887EC89EA93A4E00E94D47072
:10038A00EC89A3E0EA9FF001E451F64FE081EF70B7
:10039A00EA3098F4EC89EA9FF001E451F64FDF0164
:1003AA0080E0EFE00E9435DDE7E6EA93ED89EA5D59
:1003BA00EA93A0E0B0E00E94F12AEBEDF7E060E0FA
:1003CA0070E00E9405DDE88DF0E078966F2F660FE9
:1003DA00660B762F0E9405DD84E00E94FFDA2896DC
:1003EA000AC0EC89A3E0EA9FF001E451F64FDF016D
:1003FA00EC91EF70EC93ACC0A6EEB1E0EC89F0E0C2
:10040A00EE0FFF1FAE0FBF1F11960E9447DDE87067
:10041A0009F49EC0E885F0E0309709F063C0E989E5
:10042A00E03089F4A5EAB8E0EC89FF276627772748
:10043A00EE56FD4F6F4F6BBFE691F0E0AE0FBF1F58
:10044A00EC91E07859F4EC89A3E0EA9FF001E451D9
:10045A00F64FDF01EC91EF70EC9343C0EC89A3E017
:10046A00EA9FF001E451F64FE081E07FE03F58F463
:10047A00EC89EA9FF001E451F64FDF0184E0EFE0F6
:10048A000E9435DD2EC0E1E0E887EC89A3E0EA9F0F
:10049A00F001E451F64FDF01EC91EF70EC93EC8937
:1004AA00EA93A1E00E94D470EC89A3E0EA9FF001EC
:1004BA00E451F64FE081EF70EA3098F4EC89EA9F54
:1004CA00F001E451F64FDF0180E0EFE00E9435DDF4
:1004DA00E4E6EA93ED89EA5DEA93A0E0B0E00E94DF
:1004EA00F12A36C0E130A0E0FA0791F5A5EAB8E0B2
:1004FA00EC89FF2766277727EE56FD4F6F4F6BBFB4
:10050A00E691F0E0AE0FBF1FEC91E07809F5EC89B7
:10051A00A3E0EA9FF001E451F64FE081E07FE03F7B
:10052A0058F4EC89EA9FF001E451F64FDF0184E0C8
:10053A00EFE00E9435DD0CC0E0E0E887EC89A3E03B
:10054A00EA9FF001E451F64FDF01EC91EF70EC9372
:10055A00AF81A23009F042C0EC89FF2766277727CE
:10056A00A3E0B0E00E942DDCEE59FD4F6F4F6BBF48
:10057A00E691E030D1F0EC89FF2766277727A3E0E0
:10058A00B0E00E942DDCEE59FD4F6F4FEE5FFF4F3A
:10059A006F4F7F4F6BBFE691A0910E09EA23E0935C
:1005AA000E09E0E0E093080919C0EC89FF276627E5
:1005BA007727A3E0B0E00E942DDCEE59FD4F6F4F84
:1005CA00EE5FFF4F6F4F7F4F6BBFE691A0910D0912
:1005DA00EA23E0930D09E0E0E0930709E0911409AA
:1005EA00E770E23068F0EC89A3E0EA9FF001E55198
:1005FA00F64FE081E295E770AE2FE885EA1709F435
:10060A002DC0EAEEF7E060E070E00E9405DDE88DBB
:10061A00F0E078966F2F660F660B762F0E9405DD45
:10062A00EC8DA3E0EA9FF001E551F64FE081E295F7
:10063A00E770FF27662777270E9405DDEC89FF27E9
:10064A00662777270E9405DDEF89FF276627772728
:10065A000E9405DD80E10E94FFDA6496EC89A3E03E
:10066A00EA9FF001E551F64FDF01E885E770E29570
:10067A00E07F0E2EEC91EF78E029EC93EC89EF5FA6
:10068A00EC8BA0CDE091BA08E07421F4A09118098E
:10069A00A03009F018C0E0911609E07431F4E09135
:1006AA001609E064E09316090DC0E0911009E074A0
:1006BA0049F0E0911009EF7BE0931009E0E0E09344
:1006CA0009096AD105C0E0911609E064E0931609A8
:1006DA00E0911409E87009F4B0C0E2E0F8E060E0E3
:1006EA0070E00E9405DD80E00E94FFDA2496E0E0D7
:1006FA00EC8BAC89A73108F060C0EC89A9E0EA9FCD
:10070A00F001E45EF64FE081E17009F452C0ECE0DA
:10071A00F8E060E070E00E9405DDE88DF0E03196D7
:10072A006F2F660F660B762F0E9405DDA5EAB8E0EB
:10073A00EC8DFF2766277727E451FF4F6F4F6BBF7A
:10074A00E691F0E0AE0FBF1FEC91E07411F0E1E02A
:10075A0001C0E0E00E940DDC0E9405DDA1E4B8E0E2
:10076A00E8A1FF2766277727EC5FFE4F6F4F6BBF25
:10077A00E691F0E0EE0FFF1FAE0FBF1FED91FD9166
:10078A00662777270E9405DDECA1A9E0EA9FF00120
:10079A00ED5DF64FDF01ED91FD91AAE0B0E00E9418
:1007AA002DDC662777270E9405DD80E10E94FFDAAB
:1007BA006496EC89EF5FEC8B9CCFAC89A732C0F5CD
:1007CA00EC89A3E0EA9FF001E551F64FE081E17080
:1007DA0059F1E6E2F8E060E070E00E9405DDE88D9C
:1007EA00F0E078966F2F660F660B762F0E9405DD74
:1007FA00A5EAB8E0EC8DFF2766277727EE56FD4F6E
:10080A006F4F6BBFE691F0E0AE0FBF1FEC91E0783F
:10081A0011F0E1E001C0E0E00E940DDC0E9405DD7C
:10082A0088E00E94FFDA2C96EC89EF5FEC8BC5CF4B
:10083A00E0911409E77FE09314090C9494890E94CB
:10084A0078DBE0E05E2F2E2F3E2F0E2F10E01C30BB
:10085A0040F5A8EBB9E0EE27A10FBE1F0E9447DDC5
:10086A00E03009F021E0A9E01A9FF001E45EF64FBA
:10087A00E081F0E00E9404DCE770F070E130A0E073
:10088A00FA0711F451E00BC0E430A0E0FA0711F4C2
:10089A0031E005C0E530A0E0FA0709F401E01F5F86
:1008AA00D6CF10E0183040F5A4ECB9E0EE27A10F3E
:1008BA00BE1F0E9447DDE03009F021E0A9E01A9F3F
:1008CA00F001E45EF64FE081F0E00E9404DCE7709C
:1008DA00F070E130A0E0FA0711F451E00BC0E43007
:1008EA00A0E0FA0711F431E005C0E530A0E0FA070C
:1008FA0009F401E01F5FD6CFE0911009E295EF708D
:10090A00E695E695E170E217A9F0A0E1B9E0E22FD9
:10091A00E170E295E07FEE0FEE0F0E2EEC91EF7B89
:10092A00E029EC93E0E0E0930909E0911609EF7BF6
:10093A00E0931609A5E1B9E0E02FE170EE0FEE0FA2
:10094A000E2EEC91EB7FE029EC93A5E1B9E0E32FC1
:10095A00E170EE0FEE0FEE0F0E2EEC91E77FE0291D
:10096A00EC93A5E1B9E0E22FE170E295E07FEE0FAA
:10097A000E2EEC91EF7DE029EC93A5E1B9E0E52F8D
:10098A00E170E295E07F0E2EEC91EF7EE029EC9388
:10099A000E947FDB269608951A93E2E3F8E060E06E
:1009AA0070E00E9405DD80E00E94FFDA2496ACEC3C
:1009BA00B9E0E0E0F0E00E945BDD10E01731F0F50D
:1009CA00A9E01A9FF001E35EF64FDF01EC91E07FA8
:1009DA00EC93A9E01A9FF001E45EF64FDF01EC9177
:1009EA00EF77EC93A9E01A9FF001E25EF64FDF0180
:1009FA00EC91E07FEC93A9E01A9FF001E45EF64FD8
:100A0A00E081F0E00E9404DCE770F070E130A0E0E1
:100A1A00FA0721F0E430A0E0FA0709F404C0E5304F
:100A2A00A0E0FA0749F4A9E01A9FF001E45EF64F44
:100A3A00DF01EC91EF78EC931F5FC0CF10E01C3020
:100A4A0048F4A8EBB9E0EE27A10FBE1F0E9463DDB0
:100A5A001F5FF5CF10E01031C8F5A3E01A9FF0012F
:100A6A00E451F64FDF01EC91E07FEC93A3E01A9F8B
:100A7A00F001E551F64FDF01EC91EF77EC93A3E03B
:100A8A001A9FF001E451F64FDF01EC91EF70EC93FD
:100A9A00A3E01A9FF001E551F64FE081F0E00E94D1
:100AAA0004DCE770F070E130A0E0FA0721F0E530ED
:100ABA00A0E0FA0749F4A3E01A9FF001E551F64FC6
:100ACA00DF01EC91EF78EC931F5FC5CF10E018308F
:100ADA0048F4A4ECB9E0EE27A10FBE1F0E9463DD23
:100AEA001F5FF5CFE0911009EF7BE0931009E0E07A
:100AFA00E0930909F7C20E947ADB3A2F373310F0E4
:100B0A003C3308F0ADC000E010E0173108F05DC0DA
:100B1A00A9E01A9FF001E15EF64FA0813A1709F0A9
:100B2A0052C0A9E01A9FF001E45EF64FE081F0E0BE
:100B3A000E9404DCE770F070309761F41A9FF001AC
:100B4A00E45EF64FE081E07811F0003009F001C070
:100B5A0005E039C0E230A0E0FA0721F0E330A0E076
:100B6A00FA07B9F4A9E01A9FF001E45EF64FE081B2
:100B7A00E47011F002E00CC0A9E01A9FF001E45EF3
:100B8A00F64FE081E07811F0003009F001C005E08D
:100B9A001AC0E130A0E0FA0751F4A9E01A9FF00167
:100BAA00E45EF64FE081E07809F001E00CC0E43041
:100BBA00A0E0FA0711F4E4E0DEC2E530A0E0FA07AB
:100BCA0011F4E3E0D8C21F5FA0CF10E0103108F0A3
:100BDA0045C0A3E01A9FF001E351F64FA0813A17EE
:100BEA00D9F5A3E01A9FF001E551F64FE081F0E054
:100BFA000E9404DCE770F070309721F0E230A0E048
:100C0A00FA0709F404C0E330A0E0FA0769F4A3E0A4
:100C1A001A9FF001E551F64FE081E07811F00030BB
:100C2A0009F001C005E018C0E130A0E0FA0751F46C
:100C3A00A3E01A9FF001E551F64FE081E07809F050
:100C4A0001E00AC0E430A0E0FA0721F0E530A0E0B4
:100C5A00FA0711F4E3E08FC21F5FB8CFE02F8BC20F
:100C6A00E32FEF501E2F173108F047C0A9E01A9F53
:100C7A00F001E45EF64FE081F0E00E9404DCE770E8
:100C8A00F070309751F41A9FF001E45EF64FE0815C
:100C9A00E07811F0E5E06FC26DC2E230A0E0FA0739
:100CAA0021F0E330A0E0FA07A9F4A9E01A9FF001C5
:100CBA00E45EF64FE081E47011F0E2E05CC2A9E084
:100CCA001A9FF001E45EF64FE081E07811F0E5E06A
:100CDA0052C250C2E130A0E0FA0711F4E1E04BC27F
:100CEA00E430A0E0FA0711F4E4E045C2E530A0E000
:100CFA00FA0711F4E3E03FC233C01751103180F50F
:100D0A00A3E01A9FF001E551F64FE081F0E00E945E
:100D1A0004DCE770F070309751F41A9FF001E55146
:100D2A00F64FE081E07811F0E5E025C223C2E23017
:100D3A00A0E0FA0721F0E330A0E0FA0759F4A3E0B3
:100D4A001A9FF001E551F64FE081E07811F0E5E0F5
:100D5A0012C210C2E130A0E0FA0711F4E1E00BC2BE
:100D6A0009C267971A93FE013896FA93EA93E0E06C
:100D7A00EA93A0E1B0E00E9477D4FE013196FA939B
:100D8A00EA93E0E0EA93A7E0B0E00E9477D4EAE0D1
:100D9A00EC83EF8310E0173108F058C0E12FFF27EA
:100DAA0066277727E45EFE4F6F4F6BBFE691E03010
:100DBA0039F4ED81FE81E070F07EE062F36006C0F6
:100DCA00ED81FE81E070F07EE46FF160ED83FE83D9
:100DDA00A5E4B1E0E12FF0E0BD01A7E0B0E00E9498
:100DEA002DDCE60FF71FFA93EA93FE013396FA9386
:100DFA00EA93A7E00E94A029FE013896FA93EA93A3
:100E0A00EEE3F8E060E070E00E9405DDE12FF0E03B
:100E1A0031966F2F660F660B762F0E9405DD84E0F0
:100E2A000E94C4DA2A96E12FF0E0A0E1B8E30E941A
:100E3A00F2DBEA0FFB1FFA93EA93FE013A96FA9362
:100E4A00EA930E94502CA8951F5FA5CFFE01319608
:100E5A00FA93EA93E0E0EA93A2E0B0E00E9477D442
:100E6A0010E01031E0F5A6EEB1E0E12FF0E0EE0F70
:100E7A00FF1FEA0FFB1FFA93EA93FE013396FA93D8
:100E8A00EA93A2E00E94A029FE013896FA93EA9317
:100E9A00EEE3F8E060E070E00E9405DDE12FF0E0AB
:100EAA0078966F2F660F660B762F0E9405DD84E019
:100EBA000E94C4DA2A96E12FF0E0A0E8B9E30E9482
:100ECA00F2DBEA0FFB1FFA93EA93FE013A96FA93D2
:100EDA00EA93A0E10E94502CA8951F5FC2CF0E94FE
:100EEA0048651881689608951A930A9310E0173195
:100EFA0008F0E1C0E12FF0E0309719F4E2B1E870B0
:100F0A0096C0E130A0E0FA0719F4EEB1E0748FC0A0
:100F1A00E230A0E0FA0719F4E5B1E07188C0E330E5
:100F2A00A0E0FA0719F4E2B1E17081C0E430A0E070
:100F3A00FA0719F4E2B1E0787AC0E530A0E0FA07DE
:100F4A0019F4E4B3E87073C0E630A0E0FA0719F4C4
:100F5A00E5B1E0786CC0E730A0E0FA0719F4E2B135
:100F6A00E07465C0E830A0E0FA0719F4E2B1E27073
:100F7A005EC0E930A0E0FA0719F4E1B3E07457C0A3
:100F8A00EA30A0E0FA0719F4E1B3E07150C0EB309F
:100F9A00A0E0FA0711F4E5B149C0EC30A0E0FA0785
:100FAA0019F4E5B1E07443C0ED30A0E0FA0719F492
:100FBA00EEB1E0713CC0EE30A0E0FA0711F4EEB1F8
:100FCA0035C0EF30A0E0FA0719F4E4B3E0712FC09E
:100FDA00E031A0E0FA0719F4EEB1E47028C0E1317B
:100FEA00A0E0FA0719F4EEB1E87021C0E231A0E0FE
:100FFA00FA0719F4E2B1E0711AC0E331A0E0FA0786
:10100A0019F4EBB1E07813C0E431A0E0FA0711F467
:10101A00E1B30CC0E531A0E0FA0719F4E2B1E470DB
:10102A0006C0E631A0E0FA0719F4E2B1E0720E2F29
:10103A00E8E4F8E060E070E00E9405DDE12FF0E00E
:10104A0031966F2F660F660B762F0E9405DDA9E099
:10105A001A9FF001E45EF64FE081E295E770FF2700
:10106A00662777270E9405DD1A9FF001E45EF64F96
:10107A00E081E170FF27662777270E9405DD0130AE
:10108A0010F0E1E301C0E0E3FF27662777270E941B
:10109A0005DDA9E01A9FF001ED5DF64FDF01ED9144
:1010AA00FD91662777270E9405DD84E10E94FFDA19
:1010BA0068961F5F1CCF0991199108951A9310E041
:1010CA00153080F4E12FF0E0E55EF54F0F01A6E060
:1010DA00B2E0EE27A10FBE1F0E9447DDD001EC93BC
:1010EA001F5FEECF199108950E947ADB3A2F10E024
:1010FA00173110F5A9E01A9FF001E15EF64FA081C1
:10110A003A17C1F4A9E01A9FF001E45EF64FE081B4
:10111A00E295E7700E2F1A9FF001E45EF64FE08128
:10112A00E47031F4013021F0043011F0053011F48B
:10113A00E1E021C01F5FDCCF10E01031D8F4A9E054
:10114A001A9FF001E15EF64FA0813A1789F4A3E0F5
:10115A001A9FF001E551F64FE081E295E7700E2FF4
:10116A00013021F0043011F0053011F4E1E003C040
:10117A001F5FE3CFE0E00E9481DB24960895609729
:10118A001A93FE013196FA93EA93E0E0EA93A2E019
:10119A00B0E00E9477D410E0153088F5A6E0B2E0FE
:1011AA00EE27A10FBE1F0E9463DDFE013196FA935E
:1011BA00EA93E8E6F8E060E070E00E9405DDE12FDE
:1011CA00F0E031966F2F660F660B762F0E9405DDD1
:1011DA0084E00E94C4DA2A96E12FF0E0A0E8BAE39C
:1011EA000E94F2DBEA0FFB1FFA93EA93FE013396A1
:1011FA00FA93EA93A0E10E94502C1F5FCDCF188189
:10120A006196089563970E9478DBA6E2B1E00E9496
:10121A0047DDE07109F483C0A5E2B1E00E9447DD31
:10122A000E2FA6E2B1E00E9447DDEF70EE8B00FFC1
:10123A0004C0E0919307E170F1F401FF04C0E0916A
:10124A009407E170C1F402FF04C0E0919507E170D0
:10125A0091F403FF04C0E0919607E17061F4AE894E
:10126A00A53040F0EE89F0E03197ED56F84FE08175
:10127A00E17009F40AC0A2E3B1E00E9443DDFF7005
:10128A00E093180EF093190E4AC0A1E3B1E00E9450
:10129A0047DDEF83E03081F0AF810E94E03DE0302E
:1012AA0051F0A2E3B1E00E9443DDFF70E093180E13
:1012BA00F093190E34C013C0E091CF03E27021F00D
:1012CA00A091CE03A13008F40AC0A2E3B1E00E94C3
:1012DA0043DDFF70E093180EF093190E20C0A09121
:1012EA00180EB091190E00240A160B0640F4A8E154
:1012FA00BEE0ED91FD913197FE93EE9310C0A6E208
:10130A00B1E00E9447DDE295EF70E695E170EC8B63
:10131A00E03021F0A091610BA13008F404C00E94D2
:10132A007FDB69960895E0E0E093210E0E94C87180
:10133A000E946A39A6E00E94E82AA1E00E94B0C988
:10134A00E8E7F8E060E070E00E9405DD80E00E94D6
:10135A00FFDA249606FF2FC0E0E0E0930D09E09340
:10136A000E092898EDB5E093160EE2E4EEBDEDB550
:10137A00E7FFFDCFEAE0EEBDEDB5E7FFFDCFE09177
:10138A000D09EEBDEDB5E7FFFDCF289A2898EDB51A
:10139A00E093160EE4E4EEBDEDB5E7FFFDCFEAE01B
:1013AA00EEBDEDB5E7FFFDCFE0910E09EEBDEDB55F
:1013BA00E7FFFDCF289A07FF34C0E0E0E2B9E5B1C4
:1013CA00EF70E5B95F98EEB1E378EEB9E1B3EF7883
:1013DA00E1BBE4B3E77EE4BBE0911009EE7FE09362
:1013EA001009ED7FE0931009EB7FE0931009EB7F82
:1013FA00E0931009EF7EE0931009E0911209EB7F68
:10140A00E0931209E77FE0931209EF7EE093120955
:10141A00EF7DE0931209EF7BE0931209EF77E093F7
:10142A001209E0911009EF7DE0931009EF7BE09338
:10143A001009E0910B09EE7FE0930B09EF7DE09331
:10144A000B09E0911209ED7FE0931209E0910B0973
:10145A00E260E0930B09EF77E0930B09EF7EE093EC
:10146A000B092898EDB5E093160EE0E4EEBDEDB554
:10147A00E7FFFDCFEAE0EEBDEDB5E7FFFDCFE09176
:10148A000B09EEBDEDB5E7FFFDCF289A2898EDB51B
:10149A00E093160EE0E4EEBDEDB5E7FFFDCFE6E022
:1014AA00EEBDEDB5E7FFFDCFE0E0EEBDEDB5E7FF40
:1014BA00FDCF289AA298EDB5E093160EE0E4EEBDB2
:1014CA00EDB5E7FFFDCFEAE0EEBDEDB5E7FFFDCFF5
:1014DA00E0911009EEBDEDB5E7FFFDCFA29AA29803
:1014EA00EDB5E093160EE2E4EEBDEDB5E7FFFDCFF4
:1014FA00EAE0EEBDEDB5E7FFFDCFE0911209EEBDE2
:10150A00EDB5E7FFFDCFA29AE0E0EA8BEB8B00FF97
:10151A000FC0E0919307EC7021F452E0E1E0EB8B0D
:10152A0006C0E0919307EC70E43009F451E001C081
:10153A0050E001FF0FC0E0919407EC7021F442E003
:10154A00E1E0EB8B06C0E0919407EC70E43009F41B
:10155A0041E001C040E002FF11C0E0919507EC7044
:10156A0029F4E2E0E88FE1E0EA8B07C0E091950711
:10157A00EC70E43011F4E1E0E88F02C0E0E0E88FBB
:10158A0003FF11C0E0919607EC7029F4E2E0EF8BBB
:10159A00E1E0EA8B07C0E0919607EC70E43011F4C1
:1015AA00E1E0EF8B02C0E0E0EF8BE0E0ED8BAE898B
:1015BA00A530E8F0EE89E1501E2FFF27662777272E
:1015CA00EC56FF4F6F4F6BBFE691E150E8B9E12F40
:1015DA00F0E0ED56F84FE081EC70E43029F4EE8942
:1015EA00ED8BE0E0EE8B02C0E1E0EB8B02C0EFE3B3
:1015FA00E8B9E0E0E88BEF87EE87ED87EC8739E121
:10160A0020E0E0934D0EE887EB87A6E2B1E00E9466
:10161A0047DDE295EF70E695E695E170E98BA4E384
:10162A00B1E00E9447DDE987EA87E0E0E093D8006D
:10163A00ECBDA4E1B0E00E941BDFE0E0E093C10052
:10164A00E093C200609B02C0E1E001C0E0E0EE83EB
:10165A007198689AE0E4E0936A00E0E0E4BD0E94D1
:10166A00DA8FE0E0E0938000E0938500E093840065
:10167A00E8E1E0938900E9E6E0938800E2E0E6BB6E
:10168A00E0936F00E0E0E0937A00F894E0E8E093FA
:10169A006100E6E0E09361007894EAE0E09381007B
:1016AA00E1E8ECBBE1E0E3BF8895A895E0914D0E37
:1016BA00A885EA0FE887E0E0E0934D0EA885A530FB
:1016CA0088F0E885E550E887A4EFB0E1ED91FD9157
:1016DA006D917D91EF5FFF4F6F4F7F4F7E936E93BA
:1016EA00FE93EE93E0E0EB87513089F4489B03C008
:1016FA00E0E0E88B0CC0E989E03039F4A889A2302F
:10170A0020F4E889EF5FE88B02C0E1E0EB87413023
:10171A0089F4499B03C0E0E0EF870CC0E989E03017
:10172A0039F4AF85A23020F4EF85EF5FEF8702C06E
:10173A00E2E0EB87A88DA13089F4799B0DC0E98995
:10174A00E03039F4AE85A23020F4EE85EF5FEE8703
:10175A0002C0E3E0EB8702C0E0E0EE87AF89A13088
:10176A0089F47A9B0DC0E989E03039F4AD85A2305D
:10177A0020F4ED85EF5FED8702C0E4E0EB8702C05D
:10178A00E0E0ED87ED89E03089F0359B03C0E0E0C9
:10179A00EC870CC0E989E03039F4AC85A23020F43A
:1017AA00EC85EF5FEC8702C0E5E0EB87EB89E03080
:1017BA0021F4EA89E03009F44CC0E0E5ECBDE1E04F
:1017CA00EDBDEB89E030D1F0E0911209E260E093DF
:1017DA001209A298EDB5E093160EE2E4EEBDEDB55E
:1017EA00E7FFFDCFEAE0EEBDEDB5E7FFFDCFE09103
:1017FA001209EEBDEDB5E7FFFDCFA29AEA89E03006
:10180A00D1F0E0910B09E068E0930B092898EDB557
:10181A00E093160EE0E4EEBDEDB5E7FFFDCFEAE09A
:10182A00EEBDEDB5E7FFFDCFE0910B09EEBDEDB5DD
:10183A00E7FFFDCF289AAE89A03019F4AD89A03010
:10184A0029F088E592E00197F1F703C085E88A95C7
:10185A00F1F7523089F4489B0DC0E989E03039F438
:10186A00A889A23020F4E889EF5FE88B02C0E1E0A2
:10187A00EB8702C0E0E0E88B423089F4499B0DC057
:10188A00E989E03039F4AF85A23020F4EF85EF5FC3
:10189A00EF8702C0E2E0EB8702C0E0E0EF87A88DA5
:1018AA00A23089F4799B03C0E0E0EE870CC0E98995
:1018BA00E03039F4AE85A23020F4EE85EF5FEE8792
:1018CA0002C0E3E0EB87AF89A23089F47A9B03C0B8
:1018DA00E0E0ED870CC0E989E03039F4AD85A2304B
:1018EA0020F4ED85EF5FED8702C0E4E0EB87AE8977
:1018FA00A13088F0359B0DC0E989E03039F4AC8518
:10190A00A23020F4EC85EF5FEC8702C0E5E0EB87BC
:10191A0002C0E0E0EC87EB89E030D1F0E0911209F7
:10192A00ED7FE0931209A298EDB5E093160EE2E47A
:10193A00EEBDEDB5E7FFFDCFEAE0EEBDEDB5E7FFA1
:10194A00FDCFE0911209EEBDEDB5E7FFFDCFA29AFA
:10195A00EA89E030D1F0E0910B09EF77E0930B09C7
:10196A002898EDB5E093160EE0E4EEBDEDB5E7FF7D
:10197A00FDCFEAE0EEBDEDB5E7FFFDCFE0910B0943
:10198A00EEBDEDB5E7FFFDCF289A313018F13150A1
:10199A002030F9F020E0E0910B09EF7EE0930B098B
:1019AA00E0E5ECBDE1E0EDBD2898EDB5E093160E5B
:1019BA00E0E4EEBDEDB5E7FFFDCFEAE0EEBDEDB543
:1019CA00E7FFFDCFE0910B09EEBDEDB5E7FFFDCFD7
:1019DA00289A20C031E321E0E0910B09E061E0930D
:1019EA000B09E0E5ECBDE1E0EDBD2898EDB5E0932B
:1019FA00160EE0E4EEBDEDB5E7FFFDCFEAE0EEBD81
:101A0A00EDB5E7FFFDCFE0910B09EEBDEDB5E7FFC0
:101A1A00FDCF289A6898E0E0ECBDE091CF03E27030
:101A2A0029F0E79902C0679901C001C002C0E6E047
:101A3A00EB87609B09C0AE81A03019F0EC89E030D9
:101A4A0011F0E7E0EB8702C0E0E0EE83689AEB85ED
:101A5A00E03049F0AA85A13020F0EA85E150EA8712
:101A6A0001C004C002C0E985EA871CCEF894E0E808
:101A7A00E0936100E0E0E09361007894EDBBE093CD
:101A8A008100E0936F00E1E5ECBDE1E0EDBD719A04
:101A9A006898E6E0E093C200E8E9E093C100E0E07C
:101AAA00E093C500E3E0E093C400EDE0E4BDE0E0CC
:101ABA00E093210EADEBB2E00E9443DDDF010E940C
:101ACA005605A0E00E94AE3A0E94F03C07FF03C010
:101ADA000E94486510C006FF0EC010E0103158F48D
:101AEA00A3E01A9FF001E551F64FDF01EC91EF7880
:101AFA00EC931F5FF3CF68D0A2E3B1E00E9443DD0D
:101B0A00FF70E093180EF093190EAB85A73069F4B5
:101B1A00A091180EB091190E1A9730F4EAE0F0E08D
:101B2A00E093180EF093190E0CC0A091180EB09104
:101B3A00190E159730F4E5E0F0E0E093180EF093F3
:101B4A00190EE0E0E0931C0EE3E8F8E060E070E0D4
:101B5A000E9405DDEF85FF27662777270E9405DDAE
:101B6A0084E00E94FFDA2896A0E00E94B0C9A7E0AC
:101B7A000E94E82A0E947139E989E03029F0AB8590
:101B8A00A13010F0A53008F011C0EB85E150EB87C9
:101B9A00AB85B0E0AD56B84FEC91E160EC93AB8504
:101BAA00B0E0AD56B84FEC91E06FEC930C94EF9225
:101BBA00EA93EFB7EA93E0914D0EEF5FE0934D0E93
:101BCA00E991EFBFE991189522970E9478DB20E00E
:101BDA0050E030E0EAD1E0E2FAE0FA93EA93E0E09A
:101BEA00EA93AEE3B0E00E9477D410E0173008F031
